:020000040800F2
:1000000000000220A5B60008A5A50008A7A50008C5
:10001000A9A50008ABA50008ADA5000800000000D8
:10002000000000000000000000000000E184000863
:10003000AFA500080000000081850008E5850008E4
:10004000F5B60008F5B60008F5B60008F5B60008E4
:10005000B1A50008F5B60008F5B60008F5B6000829
:10006000F5B60008B9A50008C3A50008F5B6000854
:10007000CDA50008DDA50008EDA50008FDA5000838
:10008000F5B60008F5B60008F5B60008F5B60008A4
:100090000DA600081DA60008F5B600082DA600084C
:1000A000F5B60008F5B60008F5B60008F5B6000884
:1000B000F5B60008F5B60008F5B60008F5B6000874
:1000C000F5B6000839A6000849A6000859A6000898
:1000D00069A6000879A60008F5B6000889A60008F8
:1000E000F5B60008F5B60008F5B60008F5B6000844
:1000F000F5B6000899A60008F5B60008B1A60008F4
:10010000F5B60008F5B60008F5B60008F5B6000823
:10011000F5B60008F5B60008F5B60008F5B6000813
:10012000C1A60008F5B60008D1A60008E1A600089F
:10013000F1A60008F5B60008F5B60008F5B6000807
:1001400001A7000811A70008F5B6000821A70008BC
:1001500031A7000841A7000851A7000861A70008BF
:1001600071A7000881A70008F5B60008F5B60008D9
:10017000F5B60008F5B60008F5B600080000000066
:08018000F5B60008F5B6000811
:1001A00010B5054C237833B9044B13B10448AFF3B1
:1001B00000800123237010BD980E00200000000075
:1001C000F43B010808B5034B1BB103490348AFF3E7
:1001D000008008BD000000009C0E0020F43B0108D8
:1001E00081F0004102E000BF83F0004330B54FEAE8
:1001F00041044FEA430594EA050F08BF90EA020F55
:100200001FBF54EA000C55EA020C7FEA645C7FEAE7
:10021000655C00F0E2804FEA5454D4EB5555B8BF0A
:100220006D420CDD2C4480EA020281EA030382EA7B
:10023000000083EA010180EA020281EA0303362D0D
:1002400088BF30BD11F0004F4FEA01314FF4801CE0
:100250004CEA113102D0404261EB410113F0004FF2
:100260004FEA03334CEA133302D0524263EB4303A9
:1002700094EA050F00F0A780A4F10104D5F1200E47
:100280000DDB02FA0EFC22FA05F2801841F10001A2
:1002900003FA0EF2801843FA05F359410EE0A5F176
:1002A00020050EF1200E012A03FA0EFC28BF4CF0A7
:1002B000020C43FA05F3C01851EBE37101F000455D
:1002C00007D54FF0000EDCF1000C7EEB00006EEB6A
:1002D0000101B1F5801F1BD3B1F5001F0CD34908F4
:1002E0005FEA30004FEA3C0C04F101044FEA44524B
:1002F00012F5800F80F09A80BCF1004F08BF5FEAD2
:10030000500C50F1000041EB045141EA050130BDB1
:100310005FEA4C0C404141EB0101013C28BFB1F5C3
:10032000801FE9D291F0000F04BF01460020B1FA0E
:1003300081F308BF2033A3F10B03B3F120020CDAE1
:100340000C3208DD02F1140CC2F10C0201FA0CF0BF
:1003500021FA02F10CE002F11402D8BFC2F1200C24
:1003600001FA02F120FA0CFCDCBF41EA0C019040DA
:10037000E41AA2BF01EB0451294330BD6FEA040423
:100380001F3C1CDA0C340EDC04F11404C4F120020E
:1003900020FA04F001FA02F340EA030021FA04F320
:1003A00045EA030130BDC4F10C04C4F1200220FA77
:1003B00002F001FA04F340EA0300294630BD21FAB5
:1003C00004F0294630BD94F0000F83F4801306BF7B
:1003D00081F480110134013D4EE77FEA645C18BF6F
:1003E0007FEA655C29D094EA050F08BF90EA020F06
:1003F00005D054EA000C04BF1946104630BD91EAFE
:10040000030F1EBF0021002030BD5FEA545C05D100
:100410004000494128BF41F0004130BD14F580043F
:100420003CBF01F5801130BD01F0004545F0FE41B3
:1004300041F470014FF0000030BD7FEA645C1ABFE8
:10044000194610467FEA655C1CBF0B46024650EA1F
:10045000013406BF52EA033591EA030F41F400214B
:1004600030BD00BF90F0000F04BF0021704730B5D1
:100470004FF4806404F132044FF000054FF00001A6
:1004800050E700BF90F0000F04BF0021704730B567
:100490004FF4806404F1320410F0004548BF40423C
:1004A0004FF000013EE700BF42004FEAE2014FEA91
:1004B00031014FEA02701FBF12F07F4393F07F4F6C
:1004C00081F06051704732F07F4208BF704793F06F
:1004D0007F4F04BF41F40021704730B54FF4607482
:1004E00001F0004521F000411CE700BF50EA010285
:1004F00008BF704730B54FF000050AE050EA01022E
:1005000008BF704730B511F0004502D5404261EB9D
:1005100041014FF4806404F132045FEA915C3FF4DE
:10052000D8AE4FF003025FEADC0C18BF03325FEA7B
:10053000DC0C18BF033202EBDC02C2F1200300FA2C
:1005400003FC20FA02F001FA03FE40EA0E0021FA51
:1005500002F11444BDE600BF70B54FF0FF0C4CF43F
:10056000E06C1CEA11541DBF1CEA135594EA0C0FF1
:1005700095EA0C0F00F0DEF82C4481EA030621EA2C
:100580004C5123EA4C5350EA013518BF52EA033567
:1005900041F4801143F4801338D0A0FB02CE4FF019
:1005A0000005E1FB02E506F00042E0FB03E54FF049
:1005B0000006E1FB03569CF0000F18BF4EF0010E41
:1005C000A4F1FF04B6F5007F64F5407404D25FEA3D
:1005D0004E0E6D4146EB060642EAC62141EA5551F0
:1005E0004FEAC52040EA5E504FEACE2EB4F1FD0C32
:1005F00088BFBCF5E06F1ED8BEF1004F08BF5FEAB0
:10060000500E50F1000041EB045170BD06F0004661
:1006100046EA010140EA020081EA0301B4EB5C040E
:10062000C2BFD4EB0C0541EA045170BD41F4801106
:100630004FF0000E013C00F3AB8014F1360FDEBF2B
:10064000002001F0004170BDC4F10004203C35DA07
:100650000C341BDC04F11404C4F1200500FA05F38A
:1006600020FA04F001FA05F240EA020001F000422B
:1006700021F0004110EBD37021FA04F642EB0601A1
:100680005EEA430E08BF20EAD37070BDC4F10C04CB
:10069000C4F1200500FA04F320FA05F001FA04F28F
:1006A00040EA020001F0004110EBD37041F100017B
:1006B0005EEA430E08BF20EAD37070BDC4F1200586
:1006C00000FA05F24EEA020E20FA04F301FA05F2EE
:1006D00043EA020321FA04F001F0004121FA04F296
:1006E00020EA020000EBD3705EEA430E08BF20EA66
:1006F000D37070BD94F0000F0FD101F000464000A0
:1007000041EB010111F4801F08BF013CF7D041EA21
:10071000060195F0000F18BF704703F00046520025
:1007200043EB030313F4801F08BF013DF7D043EAF6
:100730000603704794EA0C0F0CEA135518BF95EAAC
:100740000C0F0CD050EA410618BF52EA4306D1D133
:1007500081EA030101F000414FF0000070BD50EA52
:10076000410606BF1046194652EA430619D094EADC
:100770000C0F02D150EA013613D195EA0C0F05D1C6
:1007800052EA03361CBF104619460AD181EA03011A
:1007900001F0004141F0FE4141F470014FF00000D2
:1007A00070BD41F0FE4141F4780170BD70B54FF06D
:1007B000FF0C4CF4E06C1CEA11541DBF1CEA1355ED
:1007C00094EA0C0F95EA0C0F00F0A7F8A4EB0504CF
:1007D00081EA030E52EA03354FEA013100F08880C6
:1007E0004FEA03334FF0805545EA131343EA12638F
:1007F0004FEA022245EA111545EA10654FEA002644
:100800000EF000419D4208BF964244F1FD0404F5FC
:10081000407402D25B084FEA3202B61A65EB030558
:100820005B084FEA32024FF480104FF4002CB6EB15
:10083000020E75EB030E22BFB61A754640EA0C0095
:100840005B084FEA3202B6EB020E75EB030E22BFD5
:10085000B61A754640EA5C005B084FEA3202B6EB16
:10086000020E75EB030E22BFB61A754640EA9C00D5
:100870005B084FEA3202B6EB020E75EB030E22BFA5
:10088000B61A754640EADC0055EA060E18D04FEA63
:10089000051545EA16754FEA06164FEAC30343EA03
:1008A00052734FEAC2025FEA1C1CC0D111F4801FD0
:1008B0000BD141EA00014FF000004FF0004CB6E7C9
:1008C00011F4801F04BF01430020B4F1FD0C88BF68
:1008D000BCF5E06F3FF6AFAEB5EB030C04BFB6EB73
:1008E000020C5FEA500C50F1000041EB045170BD66
:1008F0000EF0004E4EEA113114EB5C04C2BFD4EB93
:100900000C0541EA045170BD41F480114FF0000E16
:10091000013C90E645EA060E8DE60CEA135594EA92
:100920000C0F08BF95EA0C0F3FF43BAF94EA0C0F95
:100930000AD150EA01347FF434AF95EA0C0F7FF40A
:1009400025AF104619462CE795EA0C0F06D152EA5E
:1009500003353FF4FDAE1046194622E750EA410642
:1009600018BF52EA43067FF4C5AE50EA41047FF453
:100970000DAF52EA43057FF4EBAE12E74FEA4102B6
:1009800012F5001215D211D56FF47873B3EB6252E1
:1009900012D94FEAC12343F0004343EA505311F008
:1009A000004F23FA02F018BF404270474FF000009A
:1009B000704750EA013005D111F0004008BF6FF0D8
:1009C000004070474FF00000704700BF4FEA4102FF
:1009D000B2F1E04324BFB3F5001CDCF1FE5C0DD99D
:1009E00001F0004C4FEAC0024CEA5070B2F1004FE7
:1009F00040EB830008BF20F00100704711F0804FEA
:100A000021D113F13872BCBF01F00040704741F4AE
:100A100080114FEA5252C2F11802C2F1200C10FAB2
:100A20000CF320FA02F018BF40F001004FEAC12396
:100A30004FEAD32303FA0CFC40EA0C0023FA02F33A
:100A40004FEA4303CCE77FEA625307D150EA013310
:100A50001EBF4FF0FE4040F44000704701F00040E0
:100A600040F0FE4040F40000704700BF53B94AB95F
:100A7000002908BF00281CBF4FF0FF314FF0FF30A6
:100A800000F074B9ADF1080C6DE904CE00F006F881
:100A9000DDF804E0DDE9022304B070472DE9F047FA
:100AA000089D04468E46002B4DD18A42944669D952
:100AB000B2FA82F252B101FA02F3C2F1200120FA35
:100AC00001F10CFA02FC41EA030E94404FEA1C4883
:100AD000210CBEFBF8F61FFA8CF708FB16E341EA7F
:100AE000034306FB07F199420AD91CEB030306F105
:100AF000FF3080F01F81994240F21C81023E634426
:100B00005B1AA4B2B3FBF8F008FB103344EA0344C9
:100B100000FB07F7A7420AD91CEB040400F1FF33DE
:100B200080F00A81A74240F207816444023840EA1B
:100B30000640E41B00261DB1D4400023C5E9004354
:100B40003146BDE8F0878B4209D9002D00F0EF80D7
:100B50000026C5E9000130463146BDE8F087B3FA0A
:100B600083F6002E4AD18B4202D3824200F2F980F2
:100B7000841A61EB030301209E46002DE0D0C5E9F5
:100B8000004EDDE702B9FFDEB2FA82F2002A40F041
:100B90009280A1EB0C014FEA1C471FFA8CFE012644
:100BA000200CB1FBF7F307FB131140EA01410EFBE8
:100BB00003F0884208D91CEB010103F1FF3802D28F
:100BC000884200F2CB804346091AA4B2B1FBF7F089
:100BD00007FB101144EA01440EFB00FEA64508D9AC
:100BE0001CEB040400F1FF3102D2A64500F2BB80E9
:100BF0000846A4EB0E0440EA03409CE7C6F1200738
:100C0000B34022FA07FC4CEA030C20FA07F401FA7D
:100C100006F31C43F9404FEA1C4900FA06F3B1FB06
:100C2000F9F8200C1FFA8CFE09FB181140EA01416B
:100C300008FB0EF0884202FA06F20BD91CEB010108
:100C400008F1FF3A80F08880884240F28580A8F160
:100C500002086144091AA4B2B1FBF9F009FB1011B2
:100C600044EA014100FB0EFE8E4508D91CEB010150
:100C700000F1FF346CD28E456AD90238614440EAF3
:100C80000840A0FB0294A1EB0E01A142C846A64673
:100C900056D353D05DB1B3EB080261EB0E0101FAFC
:100CA00007F722FA06F3F1401F43C5E90071002659
:100CB0003146BDE8F087C2F12003D8400CFA02FCAF
:100CC00021FA03F3914001434FEA1C471FFA8CFEBF
:100CD000B3FBF7F007FB10360B0C43EA064300FBAF
:100CE0000EF69E4204FA02F408D91CEB030300F14D
:100CF000FF382FD29E422DD9023863449B1B89B204
:100D0000B3FBF7F607FB163341EA034106FB0EF38C
:100D10008B4208D91CEB010106F1FF3816D28B4239
:100D200014D9023E6144C91A46EA004638E72E4605
:100D3000284605E70646E3E61846F8E64B45A9D2FD
:100D4000B9EB020864EB0C0E0138A3E74646EAE76C
:100D5000204694E74046D1E7D0467BE7023B61441A
:100D600032E7304609E76444023842E7704700BF83
:100D7000844641EA000313F003036DD1403A41D3A6
:100D800051F8043B40F8043B51F8043B40F8043B65
:100D900051F8043B40F8043B51F8043B40F8043B55
:100DA00051F8043B40F8043B51F8043B40F8043B45
:100DB00051F8043B40F8043B51F8043B40F8043B35
:100DC00051F8043B40F8043B51F8043B40F8043B25
:100DD00051F8043B40F8043B51F8043B40F8043B15
:100DE00051F8043B40F8043B51F8043B40F8043B05
:100DF00051F8043B40F8043B51F8043B40F8043BF5
:100E0000403ABDD2303211D351F8043B40F8043B94
:100E100051F8043B40F8043B51F8043B40F8043BD4
:100E200051F8043B40F8043B103AEDD20C3205D3A4
:100E300051F8043B40F8043B043AF9D2043208D09C
:100E4000D2071CBF11F8013B00F8013B01D30B880E
:100E500003806046704700BF082A13D38B078DD0EC
:100E600010F003038AD0C3F10403D21ADB071CBFBE
:100E700011F8013B00F8013B80D331F8023B20F828
:100E8000023B7BE7043AD9D3013A11F8013B00F861
:100E9000013BF9D20B7803704B7843708B788370E9
:100EA00060467047000000000000000000000000E5
:100EB0000000000000000000000000000000000032
:100EC000A2EB0300704700BF02780B78012A28BF0D
:100ED0009A42F5D16DE9044540EA0104CDE9026783
:100EE0006FF0000C4FEA447212B380EA010414F070
:100EF000070F6AD100F0070420F0070004F0030593
:100F000021F007014FEAC505F0E8042314F0040FAF
:100F1000F1E804670CFA05F462EA040266EA0406E2
:100F20000AD063EA0403624667EA0407664603E000
:100F3000F0E80423F1E8046782FA4CF582EA06043B
:100F4000A4FA8CF46CBB83FA4CF583EA0705A5FA86
:100F50008CF595B950E9022351E9026782FA4CF504
:100F600082EA0604A4FA8CF483FA4CF583EA0705B6
:100F7000A5FA8CF52543DBD09CB92DBAB5FA85F4DA
:100F800024F0070427FA04F1DDE9026723FA04F3E9
:100F900003F0FF0001F0FF01FDE80445A0EB0100B4
:100FA000704724BAB4FA84F424F0070426FA04F152
:100FB000DDE9026722FA04F202F0FF0001F0FF010E
:100FC000FDE80445A0EB0100704714F0030F3CD18D
:100FD00010F0030428D150F8082B51F8083B82FA8E
:100FE0004CF582EA0305A5FA8CF55DB950F8042C9E
:100FF00051F8043C82FA4CF582EA0305A5FA8CF517
:10100000002DE8D02DBAB5FA85F424F0070423FAB0
:1010100004F122FA04F202F0FF0001F0FF01FDE802
:101020000445A0EB010070474FEAC40420F0030020
:1010300050F8082B21F0030151F8083B0CFA04F496
:1010400062EA040263EA0403C9E710F003041AD059
:10105000A1EB040120F00300E40750F8042B06D0B4
:101060000FD28B785FFAA2F4E41A06D12BB1CB78B9
:101070005FFAB2F4E41A00D11BB920465DF8104BB8
:10108000704701F1040150F8042BCC0721F0030153
:1010900051F8043B48D824D222F07F4482FA4CF520
:1010A00094EA1325A5FA8CF50AD165B951F8043BE9
:1010B00084EA0204B4EB036F0ED150F8042BEBE783
:1010C0004FEA132355E035F07F454DD10878FDE810
:1010D0000445C0F1000070474FEA126203F0FF03BD
:1010E00047E002EA1C4482FA4CF594EA1345A5FA5B
:1010F0008CF50AD165B951F8043B84EA0204B4EBDB
:10110000034F0CD150F8042BEBE74FEA134330E0C8
:1011100015EA1C4528D10B884FEA124229E04FEA14
:10112000124203EA1C4324E002F0FF0482FA4CF569
:1011300094EA1365A5FA8CF50AD165B951F8043B18
:1011400084EA0204B4EB032F09D150F8042BEBE737
:101150004FEA13630DE015F0FF0F05D10B684FEA5E
:10116000122223F07F4304E04FF00000FDE8044525
:10117000704712BA1BBA82FA4CF482EA0304A4FA4A
:101180008CF5B5FA85F402FA04F203FA04F34FEA97
:101190001260FDE80445A0EB1360704708B50B4BE7
:1011A0001A6842F400721A601A6842F480621A6087
:1011B0001A6842F480721A60032000F0C3FD0F2009
:1011C00009F09EF909F072F9002008BD003C0240C8
:1011D000034A1168034B1B780B441360704700BF30
:1011E000B40E002000000020014B1868704700BFBB
:1011F000B40E002038B50446FFF7F6FF0546B4F1FB
:10120000FF3F02D0044B1B781C44FFF7EDFF401B4F
:10121000A042FAD338BD00BF000000204A4B5A68F4
:1012200022F440325A605A6841680A435A600268A0
:10123000536823F48073536002685368016943EA7A
:10124000012353600268536823F0407353600268BF
:10125000536881680B4353600268936823F400630A
:10126000936002689368C1680B439360826A374B4E
:101270009A4257D00268936823F0706393600268C3
:101280009368816A0B4393600268936823F040532C
:10129000936002689368C16A0B4393600268936825
:1012A00023F00203936002689368017E43EA4103DE
:1012B000936090F82030002B3FD00268536843F4CD
:1012C000006353600268536823F46043536001680D
:1012D0004B68426A013A43EA42334B600268D36A80
:1012E00023F47003D3620168CB6AC269013A43EA0E
:1012F0000253CB620268936823F400739360026820
:10130000936890F8301043EA412393600268936831
:1013100023F48063936002689368416943EA812300
:10132000936070470268936823F07063936002686B
:10133000936823F040539360B0E70268536823F446
:1013400000635360CAE700BF002301400100000FA3
:1013500038B310B50446036C43B1236C13F0100F7F
:101360000BD00120002384F83C3010BD08F004FAB3
:101370000023636484F83C30EFE7236C23F4885344
:1013800023F0020343F0020323642046FFF746FFE5
:1013900000206064236C23F0030343F00103236403
:1013A000E0E701207047000030B482B000230193D1
:1013B00090F83C30012B00F0BB80012380F83C30DA
:1013C0000B68092B41D90468E2689BB203EB430325
:1013D0001E3B4FF0070C0CFA03F322EA0303E36011
:1013E0000468E2680B8803EB43031E3B8D6805FA33
:1013F00003F31343E3604B68062B3DD80468626B2C
:1014000003EB8303053B4FF01F0C0CFA03F322EAB6
:10141000030363630468626B4B6803EB8303053B60
:10142000B1F800C00CFA03F3134363630268414B45
:101430009A4251D002683F4B9A4256D0002380F81E
:101440003C30184602B030BC7047046822699BB239
:1014500003EB43034FF0070C0CFA03F322EA0303F8
:101460002361046822690B8803EB43038D6805FA46
:1014700003F313432361BEE70C2B16D805682A6BD0
:1014800003EB8303233B1F2404FA03F322EA030341
:101490002B6305682A6B4B6803EB8303233B0C88A3
:1014A00004FA03F313432B63C0E70568EA6A03EB0E
:1014B0008303413B1F2404FA03F322EA0303EB6294
:1014C0000568EA6A4B6803EB8303413B0C8804FA26
:1014D00003F31343EB62A9E70B68122BAAD1164A58
:1014E000536843F480035360A4E70B68103B012B5F
:1014F000A4D8114A536843F4000353600B68102BBF
:101500009CD10E4B1B6802F1467202F52E3202F29C
:101510008332A2FB03239B0C03EB83035B00019349
:1015200002E0019B013B0193019B002BF9D185E770
:10153000022087E7002001400023014094000020A2
:10154000002800F0A18038B5044690F82030D3B1CF
:101550002268136843F001031360FFF745FE054658
:1015600023685A6812F0010F10D1FFF73DFE401BAF
:101570000A28F5D9636A43F400336362052384F8CB
:101580002030012038BD08F075F9E1E71A6822F033
:1015900002021A60FFF728FE054623685A6812F017
:1015A000020F0DD0FFF720FE401B0A28F5D9636A11
:1015B00043F400336362052384F820300120E1E71F
:1015C000227E012A3DD01A6822F080021A60637ED2
:1015D000012B3BD02268136823F040031360A37EE5
:1015E000012B39D02268136823F020031360E37EB7
:1015F000012B37D02268136843F010031360237F58
:10160000012B35D02268136823F008031360637F31
:10161000012B33D02268136823F004031360A368FE
:10162000E268134322691343626913436268013A13
:1016300021681343CB6100206062012384F82030CD
:10164000A0E71A6842F080021A60C0E722681368B7
:1016500043F040031360C2E72268136843F020039D
:101660001360C4E72268136823F010031360C6E711
:101670002268136843F008031360C8E72268136800
:1016800043F004031360CAE70120704790F820304C
:10169000013BDBB2012B05D9436A43F4802343624B
:1016A0000120704730B5464BD3F8002242F00102CA
:1016B000C3F80022D3F8002222F47C52C3F800229F
:1016C000D3F80022486A42EA0022C3F800224A699D
:1016D00002F01F02012000FA02F2D3F81C026FEAA6
:1016E000020C20EA0200C3F81C02CB69C3B9344BD8
:1016F000D3F80C020CEA0000C3F80C028C8848698D
:10170000CD6844EA0544483043F830408C68088886
:1017100040EA04404C6904F1480E03EBCE035860E4
:10172000CB69012B1ED08B69002B33D12448D0F814
:1017300004320CEA0303C0F804320B698BBB204867
:10174000D0F814320CEA0303C0F814320B6A012BF0
:101750002ED01B4AD2F8003223F00103C2F8003227
:10176000002030BD164BD3F80C021043C3F80C0216
:101770008C8848690D6844EA0544483043F8304095
:1017800088894C698D6840EA0540483403EBC403FE
:101790005860C8E70A48D0F804321343C0F804324E
:1017A000CBE70748D0F814321343C0F81432CDE722
:1017B0000349D1F81C321A43C1F81C22C9E700BF03
:1017C0000064004070B5044690F82050EDB2012D41
:1017D00006D0436A43F4002343620125284670BDC6
:1017E000022380F820300268136823F0010313609D
:1017F000FFF7FAFC064623685B6813F0010F0CD074
:10180000FFF7F2FC831B0A2BF5D9636A43F400331C
:101810006362052384F82030E0E700256562DDE798
:1018200030B590F820C00468A4680CF1FF3C5FFA62
:101830008CFCBCF1010F6BD814F0E05F62D0C4F3F4
:10184000016CBCF1020F05D9436A43F40003436203
:10185000012062E0012404FA0CF41C608B68002B68
:101860003DD10D68CB68046843EA45550CF1180377
:101870001B01E55003680C690CF1180E03EB0E1305
:101880005C600B7D012B35D0D17993791B0443EA41
:101890000163517943EA012314790168234301EB81
:1018A0000C11C1F88C31D17893781B0443EA0163A1
:1018B000517843EA0123117802680B4302EB0C12C2
:1018C000C2F8883102680CF1180C4FEA0C1C52F86F
:1018D0000C3043F0010342F80C3000201DE04C684E
:1018E00043EAC403CC6823430CF1180424010568BF
:1018F0002B51BFE7036803EB0E13596841F4807165
:101900005960C1E7436A43F400134362012004E0D5
:10191000436A43F480234362012030BD90F82030B5
:10192000013BDBB2012B01D90020704703689868A6
:1019300010F0806000D001209A6812F0006F00D093
:1019400001309B6813F0805FEFD00130704790F852
:1019500020C00CF1FF3C5FFA8CFCBCF1010F00F2DF
:10196000958030B451B90468E46814F0030F10D1C5
:10197000436A43F400134362012077E0046824695A
:1019800014F0030F05D1436A43F4001343620120AE
:101990006CE001F11B04240105682C5904F00404D7
:1019A0009460002C64D101F11B04240105682C59BA
:1019B000640D1460046801F11B0C4FEA0C1C54F810
:1019C0000C4004F00204D46004686444646804F0C9
:1019D0000F041461046864446468C4F307249461C8
:1019E000046864446468240C5461026802EB0112C8
:1019F000D2F8B8211A70026802EB0112D2F8B821AD
:101A0000C2F307225A70026802EB0112D2F8B82121
:101A1000C2F307429A70026802EB0112D2F8B821B1
:101A2000120EDA70026802EB0112D2F8BC211A71B0
:101A3000026802EB0112D2F8BC21C2F307225A71EC
:101A4000026802EB0112D2F8BC21C2F307429A717C
:101A5000026802EB0112D2F8BC21120EDA7179B9D8
:101A60000268D36843F02003D360002030BC704785
:101A700001F11B04240105682C59E408546099E71E
:101A80000268136943F020031361EEE7436A43F4ED
:101A9000802343620120704790F82030013BDBB285
:101AA000012B01D90020704721B90368D86800F0E4
:101AB000030070470368186900F00300704790F84E
:101AC0002030013BDBB2012B05D9436A43F480236C
:101AD0004362012070470268536919435161002035
:101AE000704770477047704770477047704770473E
:101AF00070477047704770472DE9F84F05460368F7
:101B00005C69D3F804809F68D3F80CB0D3F810A0B8
:101B1000D3F8189014F001063BD017F0010616D048
:101B200001229A6017F0020F08D117F0040F0CD1B0
:101B300017F0080606D04FF4805608E0FFF7D1FFF3
:101B4000002604E0FFF7D0FF01E04FF4006617F431
:101B5000807F0DD02B684FF480729A6017F4007F5D
:101B600040F0868017F4806F00F0868046F40056BF
:101B700017F4803F0DD02B684FF480329A6017F431
:101B8000003F40F0838017F4802F00F0838046F4FC
:101B9000004614F0080F07D01BF0100F04D046F4D5
:101BA00000762B681022DA6014F0040F02D01BF0CC
:101BB000080F79D114F0020F04D02B68DB6813F002
:101BC000030F78D114F0400F07D01AF0100F04D093
:101BD00046F480662B6810221A6114F0200F02D0A0
:101BE0001AF0080F6BD114F0100F04D02B681B698A
:101BF00013F0030F6AD114F4003F02D018F0100F55
:101C000068D114F4803F02D018F0080F69D114F4A1
:101C1000004F7AD018F0040F74D014F4807F04D0F1
:101C200019F0010F01D046F0010614F4007F04D032
:101C300019F0020F01D046F0020614F4806F04D0B0
:101C400019F0040F01D046F0040614F4006F59D0C7
:101C500019F0700956D0B9F1400F65D058D8B9F1D4
:101C6000200F5ED0B9F1300F42D146F0200644E09B
:101C70002846FFF737FF7BE717F4006F02D046F4E2
:101C8000804675E72846FFF730FF71E72846FFF7E3
:101C90002AFF7EE717F4002F02D046F4803678E75B
:101CA0002846FFF723FF74E72B680822DA602846EE
:101CB000FFF71DFF7EE728460AF0FCFB82E72B6852
:101CC00008221A612846FFF713FF8CE728460AF01E
:101CD000F6FB90E72B6810225A602846FFF709FFB1
:101CE0008FE72B6808225A602846FFF703FF8EE72C
:101CF000B9F1100F01D146F008062A68936923F064
:101D0000700393612B6804225A609EB9BDE8F88F76
:101D1000B9F1500F0BD0B9F1600FEED146F48076D7
:101D2000EBE746F01006E8E746F04006E5E746F048
:101D30008006E2E76B6A1E436E622846FFF7DBFE11
:101D4000E4E70000074AD36823F4E0631B041B0C9C
:101D5000000200F4E060034343F0BF6343F4003348
:101D6000D360704700ED00E000B5194BDB68C3F3AA
:101D70000223C3F1070CBCF1040F28BF4FF0040C81
:101D800003F1040EBEF1060F18D9033B4FF0FF3EDE
:101D90000EFA0CFC21EA0C0199400EFA03F322EA38
:101DA0000303194300280BDB0901C9B200F16040AD
:101DB00000F5614080F800135DF804FB0023E5E7BF
:101DC00000F00F000901C9B2024B1954F4E700BF3B
:101DD00000ED00E014ED00E0002807DB00F01F023A
:101DE000400901239340024A42F82030704700BF67
:101DF00000E100E058B110B5044643791BB101235E
:101E00006371002010BD037107F0E4FDF7E70120C6
:101E1000704770B110B50446037933B102232371C2
:101E2000002020610123237110BD437107F00CFED7
:101E3000F4E7012070474379012B25D010B54FF00E
:101E4000010E80F805E0022303710468236802F0A4
:101E5000100240F6FE7C0CFA02FC23EA0C0C0B6824
:101E600049680B43934043EA0C03236004682368EA
:101E7000C02101FA02F223EA0202226080F804E0A3
:101E800000234371184610BD0220704730B4056826
:101E90002C6824F480242C60046863608368402BE1
:101EA00005D0036899600368DA6030BC7047036846
:101EB0009A600368D960F8E710B40368D9B21039A2
:101EC0000C4AA2FB014212090B4CA25CC2655F29BD
:101ED00009D923F47F7323F0030304338365806DF2
:101EE0005DF8044B704723F47F7323F0030383658D
:101EF000F5E700BFABAAAAAAEC3C0108836A826995
:101F000092B9012B0AD0022B02D00BB100207047EE
:101F1000C36A13F0807F28D100207047C36AB3F1F1
:101F2000C07F24D000207047B2F5005F09D0022B9B
:101F300025D9032B25D1C36A13F0807F23D100203C
:101F40007047032B03D8DFE803F01404140A0020C1
:101F50007047C36A13F0807F0DD100207047C36AB9
:101F6000B3F1C07F09D000207047012070470120E5
:101F70007047012070470120704701207047012001
:101F800070470020704701207047000070B504467C
:101F9000FFF72AF9002C5BD00546022384F8353080
:101FA000002384F834302268136823F0010313609F
:101FB00023681A6812F0010F0AD0FFF715F9431BC6
:101FC000052BF5D920236365032084F8350070BD07
:101FD0001A68204810406168A2680A43E1680A4311
:101FE00021690A4361690A43A1690A43E1690A4315
:101FF000216A0A430243616A04291ED01A602668D6
:10200000756925F00705636A1D43042B07D1A36A90
:102010001D43E36A1BB12046FFF770FF90B975615D
:102020002046FFF749FFE26D3F2393408360002085
:102030006065012384F83530C9E7E16A206B01430C
:102040000A43DBE740236365012084F83500BEE7DF
:102050000120BCE73F8010F038B50446856D90F84C
:10206000340001282BD0012084F8340094F8350086
:10207000C0B2012804D0002384F83430022038BDD7
:10208000022084F83500002060652046FFF7FEFE40
:10209000E26D3F239340AB602268136843F0160360
:1020A0001360236C23B12268136843F008031360A4
:1020B0002268136843F0010313600020DFE7022069
:1020C000DDE770B50446866DFFF78EF894F835307D
:1020D000DBB2022B06D080236365002384F8343002
:1020E000012070BD05462268136823F016031360B3
:1020F0002268536923F080035361236CE3B12268A3
:10210000136823F0080313602268136823F00103A7
:10211000136023681B6813F0010F11D0FFF764F8F8
:10212000431B052BF5D920236365032084F8350074
:10213000002384F83430D4E7A36C002BDFD1E3E72D
:10214000E26D3F239340B360012384F835300020D3
:1021500084F83400C5E790F83530DBB2022B03D0A9
:102160008023436501207047052380F835300268DD
:10217000136823F00103136000207047F0B583B0AB
:10218000044600230193724B1D68724BA3FB053577
:10219000AD0A876D3E68C26D08239340334210D06C
:1021A00003681A6812F0040F0BD01A6822F00402B8
:1021B0001A60C26D08239340BB60436D43F0010376
:1021C0004365E26D01239340334209D0226852698E
:1021D00012F0800F04D0BB60636D43F002036365AF
:1021E000E26D04239340334209D02268126812F052
:1021F000020F04D0BB60636D43F004036365E26DBE
:1022000010239340334224D02268126812F0080F42
:102210001FD0BB6023681A6812F4802F0DD01B6892
:1022200013F4002F04D1236C9BB12046984710E093
:10223000A36C73B1204698470BE01A6812F4807FB4
:1022400003D11A6822F008021A60236C0BB12046F1
:102250009847E26D20239340334255D0226812689C
:1022600012F0100F50D0BB6094F83530DBB2052B64
:102270000ED023681A6812F4802F33D01B6813F431
:10228000002F2AD1636C002B3ED0204698473BE0BC
:102290002268136823F0160313602268536923F041
:1022A00080035361236CA3B12268136823F00803F1
:1022B0001360E26D3F239340BB60012384F8353007
:1022C000002384F83430236D002B3FD020469847FC
:1022D0003CE0A36C002BE7D1EBE7E36BA3B1204616
:1022E000984711E01A6812F4807F09D11A6822F029
:1022F00010021A60012384F83530002384F834304A
:10230000E36B0BB120469847636DFBB1636D13F02F
:10231000010F17D0052384F835302268136823F0A5
:1023200001031360019B01330193AB4204D823687E
:102330001B6813F0010FF5D1012384F83530002319
:1023400084F83430E36C0BB12046984703B0F0BDFD
:1023500094000020B5814E1B90F8350070470000B6
:10236000204BDB6813F0100F07D01F4AD36943F0EE
:102370001003D3611B4B1022DA601A4BDB6813F099
:10238000200F07D0184AD36943F00803D361154BD7
:102390002022DA60134BDB6813F0400F07D0124A9B
:1023A000D36943F00403D3610E4B4022DA600D4B36
:1023B000DB6813F0800F07D00B4AD36943F00203A8
:1023C000D361084B8022DA60064BDB6813F0020F02
:1023D00007D0054AD36943F02003D361014B0222A1
:1023E000DA607047003C0240B80E0020704770472A
:1023F00010B53A4BDB6813F0F20F13D0384B1B7853
:10240000DBB2012B3BD0364B1B78DBB2022B3CD02E
:10241000334B5C69FFF7A4FF2046FFF7E8FF304B22
:1024200000221A702D4BDB6813F0010F13D02B4BD9
:102430000122DA602A4B1B78DBB2934228D0284B6A
:102440001B78DBB2022B41D0254B5869FFF7CEFF3A
:10245000234B00221A70224B1B787BB91F4B1A6941
:1024600022F0FF021A611A6922F080721A611A6959
:1024700022F000721A611A4B00221A7610BD184B16
:10248000DC684FF0FF32DA60C4E7154B1C69C1E726
:10249000134B5A68013A5A605B685BB1104CE068B4
:1024A000FFF7A4FFE3680133E360E068217A00F0FE
:1024B00019F8D0E70A4B4FF0FF34DC6000221A70A5
:1024C00000F03AF82046FFF791FFC4E700F034F837
:1024D000034B1869FFF78AFFBAE700BF003C0240D0
:1024E000B80E002049B1012921D0022902D04FF4B1
:1024F000407C04E04FF4007C01E04FF0000C0D4BF9
:10250000196921F4407119611A6942EA0C021A61D1
:102510001A6922F0F8021A611A6942EAC00040F012
:10252000020018611A6942F480321A6170474FF450
:10253000807CE4E7003C0240164B1B6813F4007FEC
:1025400010D0144B1A6822F400721A601A6842F410
:1025500000621A601A6822F400621A601A6842F473
:1025600000721A600B4B1B6813F4806F10D0094B7C
:102570001A6822F480621A601A6842F480521A6063
:102580001A6822F480521A601A6842F480621A6053
:10259000704700BF003C024000230F2B00F2E48094
:1025A00070B582B060E085685E000324B44025EA1F
:1025B0000405CC68B4402C438460456825EA0205D4
:1025C0004C68C4F300129A402A4342605AE0DC0887
:1025D000083450F8246003F0070295000F22AA4047
:1025E00026EA020E0A69AA4042EA0E0240F82420B6
:1025F0005CE0072200E0002202FA0EF22A430234D5
:102600005A4D45F824205A4A94686FEA0C0224EA8D
:102610000C054E6816F4801F01D04CEA0405544C9A
:10262000A560E46802EA04054E6816F4001F01D0B4
:102630004CEA04054E4CE560646802EA04054E6805
:1026400016F4003F01D04CEA0405494C656024684B
:1026500022404D6815F4803F01D04CEA0402444CFE
:10266000226001330F2B7DD801229A400C6804EAC6
:10267000020C32EA0404F4D14C6804F00304013C77
:10268000012C90D94A6802F00302032A09D0C468D9
:102690005D000322AA4024EA02048A68AA40224379
:1026A000C2604A6802F00302022A90D004684FEA2E
:1026B000430E032202FA0EF224EA02044A6802F0F0
:1026C000030202FA0EF2224302604A6812F4403F0B
:1026D000C7D000220192274A546C44F480445464C9
:1026E000526C02F480420192019A9C08A51C1F4A78
:1026F00052F8255003F003024FEA820E0F2202FA2D
:102700000EF225EA02051C4A90423FF474AF02F52E
:10271000806290421AD002F58062904218D002F591
:102720008062904216D002F58062904214D002F589
:102730008062904212D002F58062904210D002F581
:10274000806290423FF455AF082255E7012253E7DB
:10275000022251E703224FE704224DE705224BE70F
:10276000062249E702B070BD704700BF0038014043
:10277000003C014000380240000002400AB1816183
:10278000704709048161704708B5054B5B690342D6
:1027900000D108BD024B586109F0DCFFF9E700BF2A
:1027A000003C014090F83E30DBB2402B10D0036972
:1027B000B3F5804F1BD0036D002B39D1436CC3F3AD
:1027C000C813026803F0060343F0F0031361704777
:1027D000036D2BB9436C026803F0FE03136170476D
:1027E000436C026843F00103DBB21361704790F859
:1027F0003D30DBB2212B0FD0436C026843F0010364
:10280000DBB21361436B6BB1DB6B5BB10268536886
:1028100043F4006353607047436C026803F0FE03A7
:102820001361EFE7836B33B1DB6B002BEED102E07A
:10283000036D012B00D07047436CC3F3C8130268CB
:1028400003F0060343F0F1031361F4E7436C0268FD
:10285000DBB21361436B3BB1DB6B2BB10268536896
:1028600043F4006353607047836B002BFBD0DB6B3A
:10287000002BF3D1F7E710B48BB090F83E30DAB20A
:10288000C16A046B90F83D30DBB2222B0BD00023E1
:10289000099303685A6909929B690993099B0BB0D4
:1028A0005DF8044B7047036D0BB9402A17D0036DD8
:1028B0001BB90369B3F5404F19D0438D9BB2002B70
:1028C00025D1029303685A6902929A690292029A88
:1028D0001A6842F400721A6000230365DFE7009370
:1028E00003685A6900929B690093009BD7E7002315
:1028F000019303685A6901929A690192019A1A68D0
:1029000042F480721A60036D01330365C7E7438D9B
:102910009BB2012B25D0438D9BB2022B7BD002684A
:10292000136843F48063136003685A6812F4006FFD
:102930000ED011F5803F07D0012905D0082903D01A
:10294000102901D0202903D15A6842F480525A60DC
:102950000023089303685A6908929B690893089BAF
:10296000BAE711F5803F11D0082934D0202932D0A0
:10297000122C2ED0042940D002293ED010293CD060
:102980000268136823F4806313603BE002681368F5
:1029900023F48063136003685A6812F4006F0CD04C
:1029A0001A6822F480621A600023039303685A694C
:1029B00003929B690393039B8EE7002204925A695A
:1029C00004929A690492049A1A6842F400721A6096
:1029D00082E70129CED00268136823F48063136074
:1029E0000023069303685A6906929A690692069A2A
:1029F0001A6842F400721A606EE70268136843F4C2
:102A0000806313600023059303685A6905929B69EC
:102A10000593059B60E704290ED002290CD01029EC
:102A20000AD00268136823F4806313600268136895
:102A300043F40063136004E00268136843F48063A6
:102A4000136003685A6812F4006F0ED011F5803FCE
:102A500007D0012905D0082903D0102901D0202949
:102A600003D15A6842F480525A60002307930368E6
:102A70005A6907929B690793079B2DE7438D9BB289
:102A80005BB1426A036812781A61436A0133436298
:102A9000438D9BB2013B9BB243857047438D9BB2F4
:102AA0005BB103681A69436A1A70436A013343626F
:102AB000438D9BB2013B9BB24385704782B000239C
:102AC00001930E4B1B68DB080D4AA2FB03231B0A74
:102AD00003EB83030193019B013B0193019B33B102
:102AE00003681B6813F4007FF5D1002004E0036C39
:102AF00043F020030364012002B0704794000020DB
:102B000089B5F814C36AB3F52A0F04D0C36AB3F1C8
:102B10002A4F03D070470123C36270470823C36262
:102B2000F8E70000002800F0CC8070B5044690F86B
:102B30003D30002B77D0242384F83D302268136881
:102B400023F0010313602268136843F40043136009
:102B50002268136823F40043136002F045F86268AA
:102B60005A4B9A4264D85A4B98428CBF0023012397
:102B7000002B40F0A8805749A1FB00318B0C256841
:102B80006A6822F03F0242EA91426A6021680A6A5A
:102B900022F03F0266684D4DAE424FD801331343D9
:102BA0000B622168CA6922F44F4222F0FF02666874
:102BB000464B9E424CD8431E7600B3FBF6F30133DE
:102BC00040F6FC70034278D0C3F30B031343CB6190
:102BD00021680B6823F0C003E269206A02431343B3
:102BE0000B6021688B6823F4034323F0FF03226901
:102BF000E068024313438B602168CB6823F0FF0336
:102C00006269A06902431343CB602268136843F0F2
:102C10000103136000202064202384F83D302063EA
:102C200084F83E0070BD80F83C3007F0F9F882E788
:102C3000294B98428CBF0023012399E74FF49675E6
:102C400005FB03F3254DA5FB03539B090133A6E7C1
:102C5000A368BBB9451E06EB460CB5FBFCF5013578
:102C6000C5F30B05B5FA85F56D0945BBC3B9013848
:102C700006EB4603B0FBF3F30133C3F30B0343F45A
:102C80000043A3E7451E06EB860C0CEB8C0CB5FB52
:102C9000FCF50135C5F30B05B5FA85F56D09E4E7DB
:102CA000013806EB860303EB8303B0FBF3F3013338
:102CB000C3F30B0343F4404388E7042386E701236F
:102CC00084E7012070470120ACE700BFA086010027
:102CD0007F841E0083DE1B43FF083D00D34D62103E
:102CE0007047704708B590F83D30DAB2438D9BB21B
:102CF00083B1416A036809781961436A0133436209
:102D0000438D9BB2013B9BB24385438D9BB20BB974
:102D1000292A00D008BD0268536823F480635360F9
:102D200021230363282380F83D30FFF7DAFFF1E722
:102D3000704708B590F83D30DAB2438D9BB283B14D
:102D400003681969436A1970436A01334362438D0A
:102D50009BB2013B9BB24385438D9BB20BB92A2AA0
:102D600000D008BD0268536823F4806353602223B7
:102D70000363282380F83D30FFF7DAFFF1E770475F
:102D800000B583B090F83D3003F02803282B0CD019
:102D90000023019302685169019192690192019A9D
:102DA00080F83C3003B05DF804FB0268536823F4FC
:102DB0008063536011F0040F0BD0002311F0800FDB
:102DC00009D18289002180F83C101946FFF7D7FF0E
:102DD000E8E70123F2E7028BF4E7704708B590F8C3
:102DE0003D30DBB2C26A082A01D0202A01D1282B4B
:102DF00006D0212B1ED003686FF480625A6108BD93
:102E00001A4BC3620268536823F4E063536003689B
:102E10006FF480625A610268136823F48063136060
:102E200000230363202280F83D2080F83E30FFF726
:102E3000D4FFE4E70D4BC36221230363202380F812
:102E40003D30002380F83E300268536823F4E0638D
:102E5000536003686FF480625A610268136823F458
:102E600080631360FFF73DFFC9E700BF0000FFFF6D
:102E7000704708B5C26A90F83D30DBB2212B00D014
:102E800008BD438D9BB263B1426A036812781A6130
:102E9000436A01334362438D9BB2013B9BB243853E
:102EA000EEE7082A04D0202A02D012F5803F19D17B
:102EB0000268536823F4E06353600268136843F4C4
:102EC0000073136000230363202380F83D3090F8E3
:102ED0003E30DBB2402B15D0002380F83E30FFF7A8
:102EE000FFFECDE70268536823F4E06353601123CB
:102EF0000363002380F83E30202380F83D30FFF745
:102F0000EFFEBDE7002380F83E30FFF7B1FFB7E7E3
:102F100008B590F83D30026D9AB9C36C012B08D00A
:102F2000836CC3F3072302681361036D01330365E8
:102F300008BD836C0268DBB21361036D0233036565
:102F4000F6E7DBB2026D012A23D0026D022AEFD12F
:102F5000222B26D0428D92B20AB1212B2AD0428D4B
:102F600092B2002AE4D1212BE2D10268536823F403
:102F7000E06353600268136843F400731360002336
:102F80000363202280F83D2080F83E30FFF770FF79
:102F9000CEE7836C0268DBB21361036D0133036516
:102FA000C6E70268136843F480731360036D01334E
:102FB0000365BDE7426A036812781A61436A013308
:102FC0004362438D9BB2013B9BB24385B0E710B592
:102FD00090F83D30DBB290F83E20D2B2C46A018D49
:102FE00009B9212B04D0212B3BD0402A37D010BD6A
:102FF000082C04D0202C02D014F5803F19D102688F
:10300000536823F4E06353600268136843F4007369
:10301000136000230363202380F83D3090F83E3096
:10302000DBB2402B15D0002380F83E30FFF758FE6E
:10303000DDE70268536823F4E06353601123036300
:10304000002380F83E30202380F83D30FFF748FE13
:10305000CDE7002380F83E30FFF70AFFC7E7222BB9
:10306000C5D1438D9BB22BB90268536823F48063AA
:103070005360BCE790F83E30DBB2402B0CD0426A84
:10308000036812781A61436A01334362438D9BB22D
:10309000013B9BB24385AAE7FFF73AFFA7E708B5D4
:1030A000C26A438D9BB2042B14D0438D9BB2032B79
:1030B00022D0438D9BB2022B39D003681A69436A30
:1030C0001A70436A01334362438D9BB2013B9BB24A
:1030D000438510E00268536823F4806353600368FB
:1030E0001A69436A1A70436A01334362438D9BB283
:1030F000013B9BB2438508BD01684B6823F48063A4
:103100004B60042A06D0022A04D00268136823F414
:103110008063136003681A69436A1A70436A013353
:103120004362438D9BB2013B9BB24385E3E7012A97
:103130000BD0102A09D0042A38D0022A36D00268CF
:10314000136843F40073136004E00268136823F407
:103150008063136003681A69436A1A70426A531CD9
:103160004362438D9BB2013B9BB2438503681B695D
:103170005370436A01334362438D9BB2013B9BB260
:1031800043850268536823F440735360202380F81A
:103190003D3090F83E30DBB2402B0DD0002380F85C
:1031A0003E301223036309F0EDFAA4E702681368C6
:1031B00043F480631360CDE7002380F83E3003635F
:1031C00009F00AFB97E7704790F83D30DBB2222BFD
:1031D00000D0704710B50446438D9BB2032B15D920
:1031E00003681A69436A1A70436A01334362438D64
:1031F0009BB2013B9BB24385438D9BB2032B0FD106
:103200000268536823F48063536009E0C26A022AAB
:1032100001D0012B05D92268536823F480635360E1
:1032200010BDFFF74BFC00282ED12268136823F451
:10323000806313602268536823F4E063536023685B
:103240001A69636A1A70636A01336362638D9BB2A1
:10325000013B9BB26385202384F83D3094F83E30D7
:10326000DBB2402B08D0002384F83E3012232363C6
:10327000204609F087FAD3E7002384F83E30236321
:10328000204609F0A9FACBE72268536823F4E063EB
:10329000536023681A69636A1A70636A0133636250
:1032A000638D9BB2013B9BB26385202384F83D3044
:1032B000002384F83E302046FFF785FFB0E77047D3
:1032C00000B583B000230193806B90F83D20D2B20B
:1032D000324B1B68DB083249A1FB03131B0A03EBCB
:1032E0008303C3EBC3030193019B43B1019B013BE8
:1032F000019303681B6813F4007FF5D103E0036CAE
:1033000043F020030364436B0BB10021D963836B4B
:103310000BB10021D96301680B6823F480630B6053
:1033200000234385436B0BB100211965836B0BB1FF
:103330000021196501680B6823F001030B6090F808
:103340003D30DBB2602B0ED002F02802282A14D0C8
:10335000202380F83D30002380F83E30FFF733FF14
:1033600003B05DF804FB202380F83D30002380F893
:103370003E300364FFF7A3FFF2E70268136843F0EF
:10338000010313600268136843F480631360002331
:103390000363282380F83D30E0E700BF940000205D
:1033A00089B5F81410B5044690F83D30DBB290F8BA
:1033B0003E20D2B2102A36D0402A34D003F0280260
:1033C000282A38D02268526812F4006F07D1602B87
:1033D00005D0202384F83D30002384F83E300023BC
:1033E000236323685A6812F4006F48D05A6822F4A5
:1033F00000625A60626B92F83530DBB2012B20D04C
:10340000444B1365606BFEF7A6FE002849D0226886
:10341000136823F001031360202384F83D30606BB0
:10342000036D98473DE0222BC8D121680A6822F439
:1034300000620A60C2E700232363282384F83D303A
:10344000CFE7A36B334A1A65A06BFEF784FE40B347
:1034500023685A6912F0400F05D01A69636A1A701E
:10346000636A013363622268136823F00103136007
:10347000202384F83D30A06B036D984711E094F849
:103480003D20D2B2602A1FD05A6912F0400F05D0F9
:103490001A69636A1A70636A013363622046FFF730
:1034A00092FE236C13F00F0F04D02268536823F4AC
:1034B000E063536094F83D30DBB2226C12F0040FED
:1034C00001D0282B18D010BD202284F83D200022E6
:1034D00022645A6912F0400F05D01A69636A1A70A3
:1034E000636A013363622268136823F00103136087
:1034F0002046FFF7E4FED4E7074BE3620023236393
:10350000202284F83D2084F83E302046FFF765FCF9
:10351000D9E700BFC13200080000FFFF30B583B01B
:10352000044690F83D50EDB20268536823F4E0631E
:1035300053600023019303685A6901921A6842F0AC
:1035400001021A60019B0268136823F48063136010
:1035500003685A6812F4006F38D0222D21D02A2D2A
:103560001FD0426B1268526892B24285428D92B26D
:103570001AB1026C42F0040202645A6822F400623A
:103580005A60606BFEF7E8FE01281FD0636B444A67
:103590001A65606BFEF7DFFDC0B1606B036D984785
:1035A00014E0A26B1268526892B26285628D92B288
:1035B0001AB1226C42F0040222645A6822F40062BA
:1035C0005A60A06BFEF7C8FE012842D1638D9BB202
:1035D00033B323685A6912F0040F0AD01A69636A78
:1035E0001A70636A01336362638D9BB2013B9BB2C5
:1035F000638523685A6912F0400F0AD01A69636A1A
:103600001A70636A01336362638D9BB2013B9BB2A4
:103610006385638D9BB21BB1236C43F00403236469
:10362000236C13BB2A2D25D094F83D30DBB2282B18
:1036300029D0236B222B01D0222D19D10023236303
:10364000202284F83D2084F83E302046FFF770FBAE
:103650000EE0A36B124A1A65A06BFEF77CFD0028F2
:10366000B4D0A06B036D9847B0E72046FFF79AFEF1
:1036700003B030BD00232363282384F83D30204667
:10368000FFF756FBD0E7074BE362002323632022BA
:1036900084F83D2084F83E302046FFF79EFBE7E7A4
:1036A000C13200080000FFFFF8B504460268556803
:1036B000C66A90F83E30DBB290F83D10C8B2102BCD
:1036C00013D0402B11D0236C002B7AD053690021EA
:1036D00013F0020F78D015F4007F75D0236C03B17E
:1036E00091692046FFF74CFBF8BDD2F818C051692C
:1036F00011F0010705D1B6F52A0FF5D0B6F12A4F22
:10370000F2D017B115F4007F29D111F0080F02D0C3
:1037100015F4007F2AD111F0020F02D015F4007FBA
:1037200028D11CF0040F31D0526812F4006FDBD1A5
:1037300011F0800F05D015F4806F02D011F0040F46
:103740001CD011F0040FCFD015F4007FCCD021286D
:1037500018D0402BC8D12046FFF7DAFBC4E720463B
:10376000FFF7D0F92046FFF71DF8BDE72046FFF729
:103770006DF8B9E72046FFF77EF8B5E72046FFF77A
:1037800026FCB1E72046FFF774FBADE7536813F45E
:10379000006FA9D111F0400F05D015F4806F02D051
:1037A00011F0040F09D011F0040F9DD015F4007F23
:1037B0009AD02046FFF773FC96E72046FFF704FDFA
:1037C00092E79169536983E713F0100F02D015F463
:1037D000007F18D121281AD0292818D013F0400FC3
:1037E00005D015F4806F02D013F0040F28D013F029
:1037F000040F3FF479AF15F4007F3FF475AF204616
:10380000FFF74CF970E72046FFF788FE6CE713F0EE
:10381000800F05D015F4806F02D013F0040F0BD089
:1038200013F0040F3FF460AF15F4007F3FF45CAF7A
:103830002046FFF723F957E72046FFF753FA53E7EF
:103840002046FFF776FA4FE7F8B5044603685D694E
:103850005F6890F83E20D2B215F4807F07D017F44D
:10386000807F3CD06FF480715961012600E0002612
:1038700015F4007F08D017F4807F05D046F00206CB
:1038800023686FF40071596115F4806F19D017F433
:10389000807F16D0638D99B294F83D30DBB2206BF7
:1038A000202A1ED023686FF48061596146F0040617
:1038B000102A01D0402A04D12268136843F400730F
:1038C000136015F4006F08D017F4807F05D046F020
:1038D000080623686FF400625A6186B9F8BD0026B5
:1038E000C6E70029DED1212B05D0292B03D0282BB8
:1038F000D8D12128D6D12046FFF770FAE1E7236C12
:103900001E4326642046FFF74DFDE7E72DE9F0430F
:1039100083B0D0F8008001EBC10300EB8303DA6DC4
:103920005B6D9A4254D807460C469B1A01EBC102C4
:1039300000EB8202926C9A4200D31A4602F103090C
:103940004FEA990915E006F103094FEA990904EBDA
:10395000C40507EB8505E96C3B7C0093B3B2E2B28A
:10396000404603F010FAEB6C3344EB64EB6D3344E8
:10397000EB6508EB441303F510639B699BB24B4561
:1039800012D304EBC40207EB8202D16D536D99424E
:103990000AD24BB15B1A04EBC40207EB8202966CAD
:1039A0009E42D0D31E46CEE704EBC40007EB80074F
:1039B0007A6DFB6D9A420FD804F00F040123A340E7
:1039C000D8F8344824EA0304C8F83448002000E05A
:1039D000012003B0BDE8F0830020FAE770B58AB09B
:1039E000002800F090800546046890F8BD343BB391
:1039F000032385F8BD34E36B13F4807F01D10023EA
:103A00002B61286802F0DAFE2C4654F8106BEC4665
:103A10000FCCACE80F000FCCACE80F0094E803002B
:103A20008CE803002B1D0ECB304602F009FE044645
:103A300058B1022385F8BD34012420460AB070BD78
:103A400080F8BC3407F03CFCD2E70021286803F082
:103A5000B1FB234616E003EBC30205EB8202012112
:103A600082F83D1082F83C30A2F84430002182F800
:103A700040109164D16403EBC30205EB82025165EF
:103A80000133DBB269688B42E5D316E004EBC40373
:103A900005EB8303002283F87D2283F87C4283F8C0
:103AA0008022C3F88822C3F88C2204EBC40305EB00
:103AB0008303C3F894220134E4B2A142E6D82C4631
:103AC00054F8106BEC460FCCACE80F000FCCACE810
:103AD0000F0094E803008CE803002B1D0ECB30464A
:103AE00002F0C8FE044620B1022385F8BD3401244B
:103AF000A3E7002385F83830012385F8BD34286812
:103B000003F015FB99E7012497E7026890F8BC34AD
:103B1000012B19D010B50446012380F8BC34836A08
:103B2000012B09D0206802F043FE206803F0F1FA6F
:103B3000002084F8BC0410BD8369012BF2D0936B84
:103B400043F480339363EDE70220704770B5044679
:103B50000D460068066C00EB411303F530639A686C
:103B60002169012911D038498E4256D03DB905EB63
:103B7000C50304EB8303D3F89432002B5ED0E9B283
:103B8000204607F0E7FB002070BD12F0080F09D0B7
:103B90002E498E42F7D912F4004FF4D04FF4004270
:103BA0009A60F0E712F0200F02D020229A60EAE734
:103BB00012F0280FE7D125498E4206D912F4004FA2
:103BC00003D04FF400429A60DDE705EBC50204EB39
:103BD0008202D2F898121B69C3F31203CB1AC2F8FF
:103BE0009C327DB905EBC50204EB8202D2F8942227
:103BF0006AB105EBC50204EB8202D2F88C120B44C9
:103C0000C2F88C32E9B2204607F0A4FBBBE704F20D
:103C1000C442012103F010FBF4E712F4004F03D07B
:103C20004FF400429A60AEE712F0200F01D020223C
:103C30009A60E9B2204607F08DFBA4E704F2C44283
:103C4000002103F0F9FA9AE70A31544F0A30544F31
:103C500038B5044603681D6C03EB4113D3F8081B09
:103C60000E4A954207D903F5306311F4004F02D094
:103C70004FF400429A60204607F064FB074B9D42D8
:103C800002D92369012B01D0002038BD04F2C442BF
:103C90000121206803F0D0FAF6E700BF0A30544F44
:103CA00090F8BC34012B0DD010B50446012380F8E8
:103CB000BC3480F83810006803F01BFA002084F848
:103CC000BC0410BD0220704738B505468C4611F083
:103CD000800F29D101F00F0E0EEBCE04A40004F5E5
:103CE0001E740444211D0EEBCE0E00EB8E0E002040
:103CF0008EF87D020CF00F0C81F800C0CA600B71C9
:103D00004A780AB1A1F808C0022B1DD095F8BC343E
:103D1000012B1CD0012385F8BC34286802F083FEF7
:103D2000002085F8BC0438BD01F00F0000EBC00195
:103D3000890038312944043100EBC00005EB8000D4
:103D4000012480F83D40D5E700234B71DEE70220D7
:103D5000E9E710B504460A4611F0800F20D101F0C2
:103D60000F0000EBC0039B0003F51E732344191DD5
:103D700000EBC00004EB8000002380F87D3202F0ED
:103D80000F020A7094F8BC34012B19D0012384F877
:103D9000BC34206802F096FE002084F8BC0410BDFC
:103DA00001F00F0000EBC0039B0038332344191DC2
:103DB00000EBC00004EB8000012380F83D30DEE71B
:103DC0000220ECE710B501F00F0404EBC4018900F8
:103DD00001F51E710144043104EBC40C00EB8C0CA2
:103DE000CCF88C22CCF894320023CCF89C328CF89E
:103DF0007D328CF87C420369012B06D064B9DAB2BB
:103E0000006802F0CFFE002010BD04EBC40C00EBF4
:103E10008C0CCCF89022F1E7DAB2006802F0CAFF0D
:103E2000F1E701F00F0101EBC10100EB8101D1F8D5
:103E30009C02704710B501F00F0404EBC401890027
:103E400038310144043104EBC40C00EB8C0CCCF889
:103E50004C20CCF854300023CCF85C3001238CF893
:103E60003D308CF83C400369012B06D064B9DAB2CE
:103E7000006802F097FE002010BD04EBC40C00EBBC
:103E80008C0CCCF85020F1E7DAB2006802F092FF17
:103E9000F1E738B501F00F054268954239D804467C
:103EA0000B4611F0800F1FD101EBC101890001F514
:103EB0001E710144043103EBC30300EB83030022B2
:103EC00083F87D2201238B700D7094F8BC34012B94
:103ED00021D0012384F8BC34206803F0AFF88DB101
:103EE000002084F8BC0438BD05EBC50189003831D9
:103EF0000144043105EBC50300EB8303012283F881
:103F00003D20DFE704F2C442217C206803F094F9ED
:103F1000E6E70120E7E70220E5E701F00F0342684A
:103F2000934231D810B5044611F0800F1ED103EB37
:103F3000C301890001F51E710144043103EBC30282
:103F400000EB8202002082F87D0200228A700B7052
:103F500094F8BC34012B19D0012384F8BC342068B8
:103F600003F099F8002084F8BC0410BD03EBC301F2
:103F7000890038310144043103EBC30200EB8202B3
:103F8000012082F83D00E0E7012070470220ECE7C5
:103F900008B511F0800F0CD101F00F0101EBC10148
:103FA000890001F51E7101440431006802F08CFEA5
:103FB00008BD01F00F0101EBC10189003831014456
:103FC0000431F2E72DE9F04F83B004460568284636
:103FD00003F0ECF810B103B0BDE8F08F064620689E
:103FE00003F0B3F80028F6D005F50067BB68C3F30B
:103FF0000D23C4F8FC34206803F0A7F810F0020F7A
:1040000004D02268536903F002035361206803F06F
:104010009CF810F0100F13D02268936923F010035E
:104020009361D5F8208008F00F09C8F34343022BB1
:104030004BD0062B6FD02268936943F01003936135
:10404000206803F082F810F4002F76D1206803F086
:104050007CF810F4802F40F0E080206803F075F8C1
:104060000028C0F26381206803F06FF810F4006F3D
:1040700009D0BB6813F0010F40F0708122685369CA
:1040800003F400635361206803F05FF810F4805F6D
:1040900040F06881206803F058F810F4005F40F0A9
:1040A000B581206803F051F810F0080F40F0C68188
:1040B000206803F04AF810F0800F00F0D981AB6956
:1040C00023F08003AB610126C2E147F6F07318EAE2
:1040D000030FB0D04FEA181B4FEAC903019309EB55
:1040E000C90A04EB8A0AC8F30A12DAF88C122846C5
:1040F00002F07AFFCBF30A0BDAF88C325B44CAF891
:104100008C32019B4B4404EB8303D3F89C325B4419
:10411000CAF89C328FE7082204F2C441284602F014
:1041200063FFC8F30A1809EBC90204EB8202D2F854
:104130009C324344C2F89C327DE7206803F009F8C2
:104140008046B14635E005EB49130122C3F8082B40
:1041500049462046FFF7FAFC3CE005EB49130822EC
:10416000C3F8082B49462046FFF772FD35E009EBFE
:10417000C90304EB830393F87F32012B41D005EB95
:1041800049130222C3F8082B1AF0200F04D005EBC4
:1041900049132022C3F8082B1AF4005F05D005EB61
:1041A00049134FF40052C3F8082B09F101094FEAF3
:1041B0005808B8F1000F3FF449AF18F0010FF4D0E0
:1041C0005FFA89FB5946206802F0D3FF824610F05F
:1041D000010FB8D11AF0080FBFD11AF0100F04D098
:1041E00005EB49131022C3F8082B1AF0020FCBD0AD
:1041F0006B6913F0800FBAD07B6843F480637B60F7
:10420000B5E709EBC90304EB8303002283F87F229F
:104210005946204607F0F0F8B1E7206802F0A1FF08
:104220008046B14625E05946204607F09FF81AF02F
:10423000080F04D005EB49130822C3F808291AF027
:10424000100F04D005EB49131022C3F808291AF007
:10425000400F04D005EB49134022C3F808291AF097
:10426000020F40D11AF0800F5BD109F101094FEA2A
:104270005808B8F1000F3FF4F0AE18F0010FF4D079
:104280005FFA89FB5946206802F07CFF824610F0F5
:10429000010FCCD009F00F03012101FA03F27B6B6F
:1042A00023EA02037B6305EB4913C3F8081923696A
:1042B0008B42B8D109EBC90304EB8303996CDA6C28
:1042C0000A44DA64B9F1000FADD109EBC90304EB7C
:1042D00083035B6D002BA6D104F2C4420121206848
:1042E00002F0AAFF9FE74946284602F06DFA09EB63
:1042F000C90304EB830393F83F30012B05D005EB92
:1043000049130222C3F80829ACE709EBC90304EBFF
:104310008303002283F83F205946204607F072F8B5
:10432000EDE749462046FFF7F1FA9EE77B6823F068
:1043300001037B6094F8F434012B08D0204607F089
:1043400055F82268536903F0004353618BE600215E
:1043500084F8F414204600F041F9F2E7204607F013
:104360002DF88BE67B6823F001037B601021206829
:1043700002F02AFA1AE005EB46134FF67F31C3F834
:104380000819D3F8002922F40012C3F80029C3F851
:10439000081BD3F8002B22F40012C3F8002BD3F82B
:1043A000002B42F00062C3F8002B01366368B34271
:1043B000E1D8FB6943F00113FB61236BDBB1D7F854
:1043C000843043F00B03C7F884307B6C43F00B035D
:1043D0007B64D5F8003823F4FE63C5F8003804F296
:1043E000C442217C206802F027FF2268536903F44D
:1043F000805353614EE67B6943F4005343F02B0333
:104400007B613B6943F00B033B61E2E7206802F00C
:1044100002FF206802F0F6FAE060266800F0DEFB9A
:104420000146227B304602F051F9204606F0AFFFEC
:104430002268536903F40053536132E6204606F0C4
:10444000A0FF2268536903F00803536130E6013688
:104450006368B3420CD906EBC60304EB830393F8FD
:104460007F32012BF3D1F1B22046FFF791FDEEE749
:10447000206802F06AFE10F4801F27D1206802F045
:1044800064FE10F4001F5BD0012328E0013663684E
:10449000B3421DD905EB4613D3F8002906EBC6033A
:1044A00004EB830393F84030012BEFD1002AEDDABF
:1044B00006EBC60304EB8303012283F83F2066F07A
:1044C0007F01C9B22046FFF763FDDFE70126DEE783
:1044D0002268536903F480135361CFE701336268A4
:1044E0009A4228D905EB4312D2F8001B03EBC30212
:1044F00004EB820292F88022012AEFD10029EDDA42
:1045000001F48031D4F8FC2402F001029142E5D19B
:1045100003EBC30204EB8202012182F87F12AA6935
:1045200042F08002AA616A6912F0800FD6D17B68DE
:1045300043F400737B602268536903F400135361F2
:10454000206802F002FE10F0804F10D1206802F0C7
:10455000FCFD10F0040F3FF43EAD23685D6815F0DC
:10456000040F0DD1226853682B43536033E5204676
:1045700006F04EFF2268536903F080435361E5E77C
:10458000204606F04BFFEDE710B40468606A31B9CD
:1045900040EA0240A06200205DF8044B70478C4660
:1045A000A36A00EB1340002308E003F1400104EB91
:1045B0008101496800EB11400133DBB20CF1FF319E
:1045C0008B42F2D340EA02400CF13F0104EB81013F
:1045D0004860E0E7036859620020704770470000B8
:1045E000002800F0E08170B582B00446036813F043
:1045F000010F3BD09F4B9B6803F00C03042B2CD086
:104600009C4B9B6803F00C03082B21D06368B3F527
:10461000803F4FD0B3F5A02F52D0964B1A6822F4AA
:1046200080321A601A6822F480221A606368002BB4
:1046300050D0FCF7D9FD05468E4B1B6813F4003FA4
:1046400014D1FCF7D1FD401B6428F5D90320B1E15A
:10465000884B5B6813F4800FD8D0864B1B6813F42B
:10466000003F03D06368002B00F09F81236813F0A4
:10467000020F54D07F4B9B6813F00C0F3ED07D4B44
:104680009B6803F00C03082B33D0E368002B68D041
:10469000794B01221A60FCF7A7FD0546754B1B6894
:1046A00013F0020F54D1FCF79FFD401B0228F5D9EF
:1046B00003207FE16F4A136843F480331360B5E74A
:1046C0006C4B1A6842F480221A601A6842F48032F5
:1046D0001A60ABE7FCF788FD0546664B1B6813F4D0
:1046E000003FC3D0FCF780FD401B6428F5D90320B0
:1046F00060E1604B5B6813F4800FC6D15D4B1B68B3
:1047000013F0020F03D0E368012B40F05081594AA7
:10471000136823F0F803216943EAC1031360236897
:1047200013F0080F42D063696BB3534B0122C3F8F7
:10473000802EFCF759FD05464E4B5B6F13F0020FC0
:1047400034D1FCF751FD401B0228F5D9032031E19B
:10475000484A136823F0F803216943EAC103136050
:10476000DDE7454B00221A60FCF73EFD0546414B54
:104770001B6813F0020FD2D0FCF736FD401B022855
:10478000F5D9032016E13C4B0022C3F8802EFCF73C
:104790002BFD0546374B5B6F13F0020F06D0FCF77D
:1047A00023FD401B0228F5D9032003E1236813F001
:1047B000040F77D02F4B1B6C13F0805F33D1002395
:1047C00001932C4B1A6C42F080521A641B6C03F05C
:1047D00080530193019B0125284B1B6813F4807FB4
:1047E00023D0A368012B34D0052B38D0214B1A6F6E
:1047F00022F001021A671A6F22F004021A67A368F6
:10480000002B3DD0FCF7F0FC06461A4B1B6F13F053
:10481000020F46D1FCF7E8FC801B41F28833984236
:10482000F3D90320C6E00025D6E7144A136843F401
:1048300080731360FCF7D8FC0646104B1B6813F41A
:10484000807FCED1FCF7D0FC801B0228F5D9032055
:10485000B0E0084A136F43F001031367CFE7054B3D
:104860001A6F42F004021A671A6F42F001021A67C7
:10487000C5E700BF0038024000004742007000401A
:10488000FCF7B2FC0646524B1B6F13F0020F08D028
:10489000FCF7AAFC801B41F288339842F3D903202D
:1048A00088E0EDB9A369002B00F08380484A926844
:1048B00002F00C02082A51D0022B17D0454B0022DF
:1048C0001A66FCF791FC0446414B1B6813F0007F0D
:1048D00042D0FCF789FC001B0228F5D9032069E0CF
:1048E0003B4A136C23F080531364DBE7394B0022FF
:1048F0001A66FCF779FC0546354B1B6813F0007F00
:1049000006D0FCF771FC401B0228F5D9032051E0CA
:10491000E369226A1343626A43EA8213A26A520875
:10492000013A43EA0243E26A43EA0263284A5360D7
:10493000284B01221A66FCF757FC0446244B1B68DF
:1049400013F0007F06D1FCF74FFC001B0228F5D9BD
:1049500003202FE000202DE000202BE0012B2BD0A6
:104960001B4B5B6803F48001E269914226D103F09E
:104970003F02216A8A4223D1616A47F6C0721A4017
:10498000B2EB811F1ED103F44031A26A5208013AF2
:10499000B1EB024F18D103F07063E26AB3EB026F20
:1049A00014D1002006E001207047012002E0012020
:1049B00000E0002002B070BD0120FBE70120F9E714
:1049C0000120F7E70120F5E70120F3E70120F1E7F7
:1049D000003802400000474208B5254B9B6803F0B1
:1049E0000C03042B3FD0082B3FD1214B5A6802F017
:1049F0003F025B6813F4800F12D01D4B5968C1F35E
:104A000088111C480023A1FB0001FCF72FF8184B6C
:104A10005B68C3F3014301335B00B0FBF3F025E0B7
:104A2000134B5968C1F3881C4FEA4C11B1EB0C00D1
:104A30006EEB0E0E4FEA8E1343EA90638101091A62
:104A400063EB0E03DB0043EA5173C90011EB0C0C5E
:104A500043F10003990200234FEA8C2041EA9C5164
:104A6000FCF704F8D3E7034800E0034808BD00BFA3
:104A700000380240001BB7000024F400002800F0BA
:104A80009B8070B50D4604464F4B1B6803F007032F
:104A90008B4208D2CBB24C4A1370136803F0070361
:104AA0008B4240F08B80236813F0020F17D013F075
:104AB000040F04D0454A936843F4E053936023689D
:104AC00013F0080F04D0414A936843F460439360A5
:104AD0003E4A936823F0F003A1680B439360236878
:104AE00013F0010F32D06368012B21D09A1E012AE6
:104AF00025D9364A126812F0020F61D033498A680C
:104B000022F0030213438B60FCF76EFB06462F4B2B
:104B10009B6803F00C036268B3EB820F16D0FCF7BE
:104B200063FB801B41F288339842F0D9032042E0B6
:104B3000264A126812F4003FE0D101203BE0234AEC
:104B4000126812F0007FD9D1012034E01E4B1B689F
:104B500003F00703AB4207D9EAB21B4B1A701B687C
:104B600003F00703AB422DD1236813F0040F06D0E6
:104B7000164A936823F4E053E1680B43936023687B
:104B800013F0080F07D0114A936823F4604321699A
:104B900043EAC1039360FFF71FFF0C4B9B68C3F30D
:104BA00003130B4AD35CD8400A4B18600A4B1868B1
:104BB00005F0A6FC002070BD012070470120FAE737
:104BC0000120F8E70120F6E7003C024000380240EF
:104BD000803D01089400002004000020014B18686B
:104BE000704700BF9400002008B5FFF7F7FF044BA3
:104BF0009B68C3F38223034AD35CD84008BD00BF3F
:104C000000380240903D010808B5FFF7E7FF044B6C
:104C10009B68C3F34233034AD35CD84008BD00BF4E
:104C200000380240903D01080F2303600B4B9A6847
:104C300002F0030242609A6802F0F00282609A6811
:104C400002F4E052C2609B68DB0803F4E0530361A6
:104C5000034B1B6803F007030B60704700380240EA
:104C6000003C024030B583B00446036813F0050FE2
:104C700006D1236813F0020F2ED1002003B030BDFF
:104C80004A4B00229A66FCF7AFFA0546484B1B6870
:104C900013F0006F06D0FCF7A7FA431B022BF5D9DF
:104CA0000320EBE76268A3681B0743EA8213404ACC
:104CB000C2F884303D4B01229A66FCF795FA05460E
:104CC0003B4B1B6813F0006FD3D1FCF78DFA431BED
:104CD000022BF5D90320D1E700230193344B1A6C42
:104CE00042F080521A641B6C03F080530193019BC5
:104CF000304A136843F480731360FCF775FA054675
:104D00002C4B1B6813F4807F06D1FCF76DFA431B14
:104D1000022BF5D90320B1E7254B1B6F13F4407329
:104D200014D0E26802F440729A420FD0204B1A6FFE
:104D300022F440721D490120C1F8400E0020C1F844
:104D4000400E1A671B6F13F0010F13D1E36803F4D1
:104D50004072B2F5407F1ED0154A936823F4F813D1
:104D6000936013490B6FE268C2F30B0213430B67A6
:104D7000002083E7FCF738FA05460D4B1B6F13F054
:104D8000020FE3D1FCF730FA401B41F2883398421E
:104D9000F3D9032072E706498A6822F4F81223F057
:104DA000704323F4407313438B60DAE700004742FB
:104DB000003802400070004098B110B504464379B5
:104DC0005BB1022363712268136843F0040313602C
:104DD000012363710020A06010BD037105F0B4F9D8
:104DE000EFE70120704738B504460268D36823F026
:104DF000A003D360FCF7F8F905462368DB6813F0DD
:104E0000200F07D1FCF7F0F9401BB0F57A7FF4D9F9
:104E1000032000E0002038BD70B50368DA6812F0A6
:104E2000400F02D00025284670BD0446DA6842F0E3
:104E30008002DA60FCF7D8F9064600252368DB68B3
:104E400013F0400FEFD1002DEDD1FCF7CDF9831B0E
:104E5000B3F57A7FF2D9042363770125EEE7026880
:104E6000D36823F08003D36003689B6813F0200F9E
:104E700001D00020704710B50446FFF7B4FF10B111
:104E800004236377012010BD002841D010B50446EB
:104E9000437FE3B1022363772368CA225A622368FF
:104EA00053225A622046FFF7B7FFA0B158B92268D3
:104EB000136C23F4802313642268136CA1690B43E1
:104EC0001364012363772368FF225A6210BD0377BE
:104ED00005F06CF9DEE72268936823F4E00323F021
:104EE0004003936021688A686368206903436069AE
:104EF000034313438B602368E2681A6122681369D5
:104F0000A16843EA014313612046FFF7A8FFCDE7FC
:104F1000012070472DE9F04782B0054688461746C4
:104F20001E46FCF761F90A9B1B1A03EB0609FCF706
:104F30005BF982462B4B1B68C3F3CB3309FB03F3AE
:104F400001932B689C6838EA04030CBF4FF0010CF6
:104F50004FF0000CBC4540D0B6F1FF3FF1D0FCF75C
:104F600043F9A0EB0A0048450AD2B9F1000F07D077
:104F7000019A02B14A46019B013B01939146E0E749
:104F80002A68536823F0E00353606B68B3F5827FAF
:104F90000BD0AB6AB3F5005F14D0012385F8513014
:104FA000002385F85030032018E0AB68B3F5004FBC
:104FB00002D0B3F5806FECD12A68136823F0400368
:104FC0001360E6E72A68136823F4005313602A6825
:104FD000136843F400531360DFE7002002B0BDE81C
:104FE000F08700BF9400002010B584B00446164B33
:104FF0001868164BA3FB0030400D4FF47A7303FB87
:1050000000F003906368B3F5827F0BD0039BBBB1C4
:10501000039B013B039323689B6813F0800FF5D13A
:1050200000200EE000920B46002280212046FFF770
:1050300071FF30B1636D43F020036365032000E02E
:10504000002004B010BD00BF94000020819F5E16B8
:1050500000285AD010B50446436A33B94368B3F503
:10506000827F05D00023C36102E000230361436116
:105070000023A36294F85130002B40D0022384F81F
:1050800051302268136823F040031360636803F40F
:105090008273A26802F404421343E26802F40062DD
:1050A0001343226902F002021343626902F0010213
:1050B0001343A26902F400721343E26902F038025A
:1050C0001343226A02F080021343A26A02F40052E0
:1050D000216813430B60638B03F00403626A02F0E0
:1050E0001002216813434B602268D36923F40063E4
:1050F000D36100206065012384F8513010BD84F82D
:105100005030204605F0BEF8B8E7012070472DE981
:10511000F04383B01F460A9D90F85030012B00F0F9
:105120001081044688469146012380F85030FCF7F0
:105130005BF8064694F85130DBB26268012B0AD066
:10514000B2F5827F40F0E380A268002A40F0E98057
:10515000042B40F0E880B8F1000F00F0E680B9F1D0
:10516000000F00F0E480002F00F0E38094F851304D
:10517000DBB2042B02D0052384F851300023636591
:10518000C4F83890E787A787C4F83080E786A786F9
:105190002364636423681A6812F0400F03D11A680D
:1051A00042F040021A60E368B3F5006F11D0636803
:1051B0000BB1012F0BD1226B236812781A73236B6A
:1051C00001332363E38E9BB2013B9BB2E38601274D
:1051D0006BE063680BB1012F0BD1226B236812883F
:1051E000DA60236B02332363E38E9BB2013B9BB2F5
:1051F000E38601271CE023689A6812F0010F0ED0A5
:10520000E28F92B25AB1DA68A36B1A80A36B0233B1
:10521000A363E38F9BB2013B9BB2E3870127FBF7BC
:10522000E3FF801BA84203D3B5F1FF3F40F083802A
:10523000E38E9BB21BB9E38F9BB2002B53D0236844
:105240009A6812F0020FD6D0E28E92B2002AD2D023
:10525000002FD0D0226B1288DA60236B02332363D5
:10526000E38E9BB2013B9BB2E3860027C3E7236832
:105270009A6812F0010F0ED0E28F92B25AB1DA683A
:10528000A36B1A70A36B0133A363E38F9BB2013B43
:105290009BB2E3870127FBF7A7FF831BAB4202D337
:1052A000B5F1FF3F49D1002D49D0E38E9BB213B930
:1052B000E38F9BB2BBB123689A6812F0020FD6D07D
:1052C000E28E92B2002AD2D0002FD0D0226B127878
:1052D0001A73236B01332363E38E9BB2013B9BB2B2
:1052E000E3860027C3E7324629462046FFF77CFEC7
:1052F00048B9A36863B901932368DA6801929B688F
:105300000193019B04E020236365012000E002205B
:10531000012384F85130002384F8503003B0BDE8F5
:10532000F0830220F4E70220F2E70120F0E70120F9
:10533000EEE70120ECE70320EAE70320E8E703209B
:10534000E6E70220EAE7704730B585B00446026818
:1053500051689368C3F3801013F0400F05D113F028
:10536000010F02D011F0400F69D113F0020F02D0EB
:1053700011F0800F67D1C3F3401513F0200F03D154
:1053800010B913F4807F61D011F0200F5ED078B196
:1053900094F85100C0B203285AD0606D40F0040068
:1053A000606500200090D0680090906800900098A0
:1053B00065B1606D40F0010060650020029090686A
:1053C0000290106820F040001060029A13F4807F71
:1053D00009D0636D43F008036365002303932368DA
:1053E0009B680393039B636D002B2FD02268536847
:1053F00023F0E0035360012384F8513011F0030FD0
:105400002ED02268536823F003035360E36C4BB142
:10541000154A1A65E06CFCF79EFE18B1636D43F007
:1054200040036365A36C8BB10F4A1A65A06CFCF74F
:1054300092FE58B1636D43F04003636506E0236C50
:105440002046984702E0636C2046984705B030BD7F
:1054500000230193D368019393680193019BF5E7BF
:105460002046FFF770FFF1E76D54000808B5806B28
:105470000023C387C386FFF766FF08BD30B4036A05
:1054800023F001030362036A4268846924F0730411
:105490000D682C4323F0020C8B6843EA0C03104D7B
:1054A000A84203D005F58065A84205D123F0080382
:1054B000CD682B4323F00403094DA84203D005F522
:1054C0008065A84205D122F440724D692A438D6956
:1054D0002A43426084614A684263036230BC704779
:1054E0000000014030B4036A23F480730362036A4E
:1054F0004268C46924F0730C0C6844EA0C0523F478
:1055000000738C6843EA0423114CA04203D004F5D5
:105510008064A04206D123F40063CC6843EA0423EC
:1055200023F480630A4CA04203D004F58064A042B7
:1055300007D122F440524C6942EA04128C6942EAD3
:1055400004124260C5614A68C263036230BC70479E
:105550000000014030B4036A23F480530362036AFD
:105560004468C26922F4E6420D6842EA052223F447
:1055700000538D6843EA0533094DA84203D005F571
:105580008065A84204D124F480444D6944EA85141E
:105590004460C2614A680264036230BC704700BF65
:1055A0000000014010B4036A046A24F0010404629C
:1055B000846924F0F00C4CEA021223F00A030B4336
:1055C000826103625DF8044B704710B4046A24F0F2
:1055D000100404628469036A24F4704C4CEA0232B9
:1055E00023F0A00343EA0113826103625DF8044BD8
:1055F0007047836823F070030B4343F00703836015
:105600007047000090F83D30DBB2012B37D1022308
:1056100080F83D300268D36843F00103D36003682B
:10562000194A934220D0B3F1804F1DD0A2F57C429D
:10563000934219D002F58062934215D002F5806240
:10564000934211D002F5784293420DD002F5705288
:10565000934209D0A2F59432934205D01A6842F0E1
:1056600001021A60002070479A6802F00702062AB9
:1056700007D01A6842F001021A600020704701202A
:1056800070470020704700BF00000140704770471E
:105690007047704710B5044603681A6912F0020F8C
:1056A00011D0DA6812F0020F0DD06FF002021A6109
:1056B0000123037703689B6913F0030F70D0FFF792
:1056C000E7FF0023237723681A6912F0040F12D032
:1056D000DA6812F0040F0ED06FF004021A61022390
:1056E000237723689B6913F4407F5FD02046FFF740
:1056F000CFFF0023237723681A6912F0080F12D016
:10570000DA6812F0080F0ED06FF008021A61042355
:1057100023772368DB6913F0030F4ED02046FFF791
:10572000B7FF0023237723681A6912F0100F12D0F5
:10573000DA6812F0100F0ED06FF010021A61082311
:1057400023772368DB6913F4407F3DD02046FFF7C1
:105750009FFF0023237723681A6912F0010F03D0FB
:10576000DA6812F0010F36D123681A6912F0800F3F
:1057700003D0DA6812F0800F34D123681A6912F06E
:10578000400F03D0DA6812F0400F32D123681A6953
:1057900012F0200F03D0DA6812F0200F30D110BDC4
:1057A000FFF775FF204607F059F88AE72046FFF714
:1057B0006EFF204607F052F89BE72046FFF767FF91
:1057C000204607F04BF8ACE72046FFF760FF204685
:1057D00007F044F8BDE76FF001021A61204604F0BB
:1057E000F9FBC1E76FF080021A61204600F000FB70
:1057F000C3E76FF040021A612046FFF74AFFC5E792
:105800006FF020021A61204600F0F1FAC7E70000AD
:105810000368304A904212D0B0F1804F0FD0A2F509
:105820007C4290420BD002F58062904207D002F594
:105830008062904203D002F57842904203D123F077
:1058400070034A681343234A90422AD0B0F1804F34
:1058500027D0A2F57C42904223D002F5806290428C
:105860001FD002F5806290421BD002F57842904230
:1058700017D002F57052904213D002F58062904228
:105880000FD002F5806290420BD0A2F59832904280
:1058900007D002F58062904203D002F58062904208
:1058A00003D123F44073CA68134323F080034A6989
:1058B000134303608B68C3620B688362054B984295
:1058C00003D003F58063984201D10B690363012380
:1058D000436170470000014040B310B5044690F8A2
:1058E0003D30F3B1022384F83D30214651F8040BDA
:1058F000FFF78EFF012384F8463084F83E3084F8A9
:105900003F3084F8403084F8413084F8423084F8E5
:10591000433084F8443084F8453084F83D3000202A
:1059200010BD80F83C3004F061FFDBE701207047D8
:1059300040B310B5044690F83D30F3B1022384F82B
:105940003D30214651F8040BFFF762FF012384F834
:10595000463084F83E3084F83F3084F8403084F894
:10596000413084F8423084F8433084F8443084F87D
:10597000453084F83D30002010BD80F83C30FFF702
:1059800085FEDBE70120704730B4036A23F0100383
:105990000362036A4468826922F4E6420D6842EABF
:1059A000052223F020038D6843EA0513114DA84218
:1059B00003D005F58065A84206D123F08003CD68A9
:1059C00043EA051323F040030A4DA84203D005F52E
:1059D0008065A84207D124F440644D6944EA8504F7
:1059E0008D6944EA8504446082614A688263036287
:1059F00030BC70470000014038B590F83C30012BB6
:105A000066D004460D46012380F83C300C2A5AD853
:105A1000DFE802F0075959591B595959305959595A
:105A200044000068FFF72AFD2268936943F00803E9
:105A300093612268936923F0040393612268936958
:105A400029690B43936100203EE00068FFF79CFF4B
:105A50002268936943F4006393612268936923F495
:105A60008063936122689369296943EA0123936102
:105A7000002029E00068FFF735FD2268D36943F074
:105A80000803D3612268D36923F00403D361226839
:105A9000D36929690B43D361002015E00068FFF743
:105AA00059FD2268D36943F40063D3612268D36946
:105AB00023F48063D3612268D369296943EA01230F
:105AC000D361002000E00120002384F83C3038BD81
:105AD0000220FCE710B4846824F47F4C42EA0322DD
:105AE0000A4342EA0C0282605DF8044B704790F86A
:105AF0003C30012B78D010B50446012380F83C30AF
:105B0000022380F83D300268936823F47F4323F03A
:105B1000770393600B68602B4CD029D8402B54D06E
:105B20000CD9502B22D1CA6849680068FFF73AFDAA
:105B300050212068FFF75DFD002005E0202B0DD0EF
:105B400009D9302B0AD00120012384F83D300023ED
:105B500084F83C3010BD0BB1102B05D119462068DC
:105B6000FFF747FD0020EFE70120EDE70120EBE71D
:105B7000B3F5805F34D0B3F5005F0CD1CB684A68D1
:105B800089680068FFF7A6FF2268936843F48043A2
:105B900093600020D8E7702B24D1CB684A688968CD
:105BA0000068FFF797FF2268936843F077039360DC
:105BB0000020C9E7CA6849680068FFF706FD602150
:105BC0002068FFF716FD0020BEE7CA684968006834
:105BD000FFF7E8FC40212068FFF70BFD0020B3E74A
:105BE0000020B1E70120AFE70220704701F01F015C
:105BF000012303FA01FC036A23EA0C030362036A2C
:105C000002FA01F10B4303627047000010B504462D
:105C10000846002942D194F83E30DBB2013B18BF60
:105C20000123002B6ED1002851D1022384F83E308D
:105C3000012201462068FFF7D9FF2368334A9342C7
:105C400003D002F58062934203D15A6C42F40042C1
:105C50005A6423682D4A934249D0B3F1804F46D00D
:105C6000A2F57C42934242D002F5806293423ED03C
:105C700002F5806293423AD002F57842934236D0E0
:105C800002F57052934232D0A2F5943293422ED054
:105C90001A6842F001021A60002032E0042908D09C
:105CA00008290DD094F84130DBB2013B18BF012325
:105CB000B7E794F83F30DBB2013B18BF0123B0E7F0
:105CC00094F84030DBB2013B18BF0123A9E7042858
:105CD00005D0082807D0022384F84130A8E7022322
:105CE00084F83F30A4E7022384F84030A0E79A68A4
:105CF00002F00702062A07D01A6842F001021A6071
:105D0000002010BD0120FCE70020FAE70000014060
:105D100090F83C30012B3DD010B4012380F83C308A
:105D2000022380F83D3003685A689C6822F0700CAA
:105D30000A6842EA0C025A600368174A93421AD072
:105D4000B3F1804F17D0A2F57C42934213D002F5F5
:105D5000806293420FD002F5806293420BD002F52D
:105D60007842934207D002F57052934203D0A2F5D5
:105D70009432934204D124F080044A6814439C6016
:105D8000012380F83D30002380F83C3018465DF850
:105D9000044B7047022070470000014090F83C30EF
:105DA000012B22D0012380F83C30CB6823F44073D0
:105DB0008A68134323F480634A68134323F400631F
:105DC0000A68134323F480530A69134323F40053EE
:105DD0004A69134323F48043CA6913430268536436
:105DE000002380F83C301846704702207047704707
:105DF0007047026802F10C0353E8003F23F0C00330
:105E00000C3242E800310029F3D1202380F83D30E4
:105E10007047026802F10C0353E8003F23F49073CB
:105E20000C3242E800310029F3D1026802F1140378
:105E300053E8003F23F00103143242E80031002907
:105E4000F3D1036B012B05D0202380F83E300023D3
:105E500003637047026802F10C0353E8003F23F02C
:105E600010030C3242E800310029F3D1ECE790F83E
:105E70003D30DBB2212B01D0022070478368B3F59F
:105E8000805F17D0036A5A1C02621A7803685A604E
:105E9000C38C9BB2013B9BB2C3844BB90268D368ED
:105EA00023F08003D3600268D36843F04003D360DB
:105EB000002070470369002BE4D1036A1B88026845
:105EC000C3F308035360036A02330362E0E7000090
:105ED00038B504460268136923F44053C1680B4384
:105EE000136183680269134342691343C2691A4309
:105EF0000168CB6823F4164323F00C031343CB60F3
:105F00000268536923F4407381690B43536103684A
:105F1000314A934206D002F58062934202D0FEF7E6
:105F200063FE01E0FEF770FEE369B3F5004F29D090
:105F30000021031849411B1841F10001C90041EA41
:105F40005371DB00181863684FEA83024FEA9373BA
:105F500041F10001FAF78AFD204DA5FB00325109FD
:105F6000642303FB11031B013233A5FB03235B09ED
:105F700003F0F00202EB011203F00F032168134457
:105F80008B6038BD0023021843EB0301121841F166
:105F90000001C90041EA5271D200101841F100011C
:105FA000626892185B41FAF761FD0C4DA5FB003267
:105FB0005109642303FB1103DB003233A5FB0323E8
:105FC0005B095A0002F4F87202EB011203F00703B6
:105FD000216813448B60D4E7001001401F85EB510A
:105FE00058B310B5044690F83D300BB3242384F821
:105FF0003D302268D36823F40053D3602046FFF776
:1060000067FF2268136923F4904313612268536980
:1060100023F02A0353612268D36843F40053D3600A
:1060200000202064202384F83D3084F83E3010BDE9
:1060300080F83C3004F06CFFD8E7012070477047CF
:1060400008B50168CA6822F04002CA60202280F8C0
:106050003D20FFF7F4FF002008BD7047704710B5E2
:10606000846B23685A6994F83D30DBB2212B10D041
:1060700023685A6902F0400294F83E30DBB2222BCA
:1060800011D0236C43F010032364204606F03EFD3C
:1060900010BD02F08002002AEAD00023E3842046EB
:1060A000FFF7A7FEE4E7002AEBD00023E3852046B4
:1060B000FFF7AFFEE5E708B5806B0023C385C38417
:1060C00006F024FD08BD90F83E30DBB2222B67D1EC
:1060D0008368B3F5805F4DD0826AB3F5805F04D0EA
:1060E000002B54D10369002B51D103685B681370F6
:1060F000836A01338362C38D9BB2013B9BB2C3852C
:10610000002B4FD100B583B00268D36823F0200381
:10611000D3600268D36823F48073D3600268536944
:1061200023F001035361202380F83E30036B012BE1
:1061300033D100230363026802F10C0353E8003FEC
:1061400023F010030C3242E800310029F3D1036838
:106150001A6812F0100F06D0002201921A680192FC
:106160005B680193019B818D06F09AFC002003B0CF
:106170005DF804FB0269002AAED1826A03685B689D
:10618000C3F308031380836A02338362B3E70368AF
:106190005B6803F07F031370AAE7FFF75EFFE5E794
:1061A000022070470020704730B583B00446026873
:1061B0001368D068516913F00F0505D113F0200F53
:1061C00002D010F0200F19D12DB111F0010119D119
:1061D00010F4907F16D1216B01297DD013F0800F30
:1061E00003D010F0800F40F0158113F0400F03D062
:1061F00010F0400F40F0128103B030BD2046FFF791
:1062000062FFF9E713F0010F06D010F4807F03D08E
:10621000226C42F00102226413F0040F04D019B181
:10622000226C42F00202226413F0020F04D019B172
:10623000226C42F00402226413F0080F07D010F021
:10624000200F00D119B1226C42F008022264226CA6
:10625000002AD1D013F0200F02D010F0200F29D146
:1062600023685B6903F04003226C12F0080F00D131
:1062700063B32046FFF7CDFD23685B6913F0400F41
:1062800020D0226802F1140353E8003F23F04003BA
:10629000143242E800310029F3D1A36B73B1614A93
:1062A0001A65A06BFBF757FF0028A5D0A06B036D04
:1062B0009847A1E72046FFF706FFD1E7204606F002
:1062C00025FC99E7204606F021FC95E7204606F0DC
:1062D0001DFC002323648FE713F0100F3FF47EAF03
:1062E00010F0100F3FF47AAF00230193136801936D
:1062F00053680193019B536913F0400F50D0A26B78
:1063000013685B689BB2002B3FF476AFA18D994276
:106310007FF672AFE385D369B3F5807F37D022680B
:1063200002F10C0353E8003F23F480730C3242E87F
:1063300000310029F3D1226802F1140353E8003F31
:1063400023F00103143242E800310029F3D122681E
:1063500002F1140353E8003F23F04003143242E8F3
:1063600000310029F3D1202384F83E300023236339
:10637000226802F10C0353E8003F23F010030C32B3
:1063800042E800310029F3D1A06BFBF79AFEA18D02
:10639000E38D9BB2C91A89B2204606F081FB2BE738
:1063A000A18DE38D9BB2C91A89B2E38D9BB2002BFC
:1063B0003FF422AF00293FF41FAF226802F10C0323
:1063C00053E8003F23F490730C3242E80030002879
:1063D000F3D1226802F1140353E8003F23F00103D4
:1063E000143242E800300028F3D1202384F83E30F4
:1063F00000232363226802F10C0353E8003F23F0DB
:1064000010030C3242E800300028F3D1204606F099
:1064100047FBF1E62046FFF72AFDEDE62046FFF7B1
:106420000FFEE9E6B760000808B5806B036B012B2F
:1064300002D0FFF713FE08BD818D490806F030FB3E
:10644000F9E708B50346806B1B681B6813F4807F6F
:106450002BD10023C385026802F10C0353E8003FEF
:1064600023F480730C3242E800310029F3D1026832
:1064700002F1140353E8003F23F00103143242E811
:1064800000310029F3D1026802F1140353E8003F00
:1064900023F04003143242E800310029F3D12023D5
:1064A00080F83E30036B012B05D0036B012B0FD01E
:1064B000FFF7D3FD08BD026802F10C0353E8003F6B
:1064C00023F010030C3242E800310029F3D1ECE74D
:1064D000818D06F0E5FAEDE730B583B0044613464A
:1064E0008162828500250564222280F83E20826B2D
:1064F0002048D063A26B20481064A26B1F48D06470
:10650000A26B156520680A46011DA06BFBF7A4FD70
:10651000019523681A6801925B680193019B84F8D6
:106520003C5023695BB1226802F10C0353E8003F41
:1065300043F480730C3242E800310029F3D1226821
:1065400002F1140353E8003F43F00103143242E820
:1065500000310029F3D1226802F1140353E8003F0F
:1065600043F04003143242E800310029F3D1002007
:1065700003B030BD43640008296400085F60000870
:1065800090F83E30DBB2202B29D110B582B0044602
:1065900039B342B390F83C30012B27D0012380F867
:1065A0003C300363FFF798FFF0B9236B012B01D058
:1065B000012019E00023019323681A6801925B68A7
:1065C0000193019B226802F10C0353E8003F43F062
:1065D00010030C3242E800310029F3D104E002201C
:1065E0007047012000E0012002B010BD0220FBE74F
:1065F00082B000230193019B01330193019A0F4B59
:106600009A4215D80369002BF5DA00230193036938
:1066100043F001030361019B01330193019A074B8E
:106620009A4208D8036913F0010FF4D1002000E06A
:10663000032002B070470320FBE700BF400D0300BA
:1066400084B010B5044603A880E80E00089B012B17
:106650001FD1A36B23F48033A363E36823F4840383
:1066600023F04003E360E36823F44013E3600F9BEF
:10667000012B09D02046FFF7BBFF069B012B1BD047
:10668000BDE8104004B07047E36843F48013E36052
:10669000F0E7E36843F04003E3602046FFF7A8FF1C
:1066A0000C9B23B9A36B43F48033A363E5E7A36B8F
:1066B00023F48033A363E0E7A36843F00603A360F9
:1066C000A36843F02003A360DAE70000022A0AD09F
:1066D0000921C26822F47052C260C36843EA812370
:1066E000C36000207047234B0B44234A93422FD9A9
:1066F000224B0B44224A93422CD9A1F57403A3F5F3
:106700001053204A934227D9A1F18373A3F5E7439D
:106710001D4A934222D31D4B0B441D4A93421FD95D
:106720001C4B0B441C4A93421CD31C4B0B441C4A6D
:10673000934219D3A1F1B773A3F55853194A934261
:1067400014D3194B0B44194A934211D20721C0E7C5
:106750000F21BEE70E21BCE70D21BAE70C21B8E7F7
:106760000B21B6E70A21B4E70921B2E70821B0E717
:106770000621AEE7405327FFFF340C00401E1BFFED
:106780003F420F007F4F120020D6130060B6E5FE97
:106790005FE3160000D3CEFE40771B00C05BB3FE64
:1067A000C091210020753800E05459FEE09C410062
:1067B000836843F00103836000207047836823F0FF
:1067C000010383600020704782B000230193019B86
:1067D00001330193019A0F4B9A4215D80369002B9C
:1067E000F5DA00230193890141F020010161019B49
:1067F00001330193019A074B9A4208D8036913F0B9
:10680000200FF4D1002000E0032002B070470320E5
:10681000FBE700BF400D030082B000230193019B02
:1068200001330193019A0E4B9A4213D80369002B4E
:10683000F5DA0023019310230361019B01330193D7
:10684000019A074B9A4208D8036913F0100FF4D14C
:10685000002000E0032002B070470320FBE700BFE8
:10686000400D0300D0F800381943C0F8001800208C
:106870007047000084B02DE9F041044607A880E885
:106880000E00002306E003F1400204EB8202002127
:10689000516001330E2BF6D9119F27BBD4F8043871
:1068A00043F00203C4F80438A36B43F40013A3635A
:1068B000A36B23F40023A363A36B23F48023A363BC
:1068C0000023C4F8003E04F50065D4F80038C4F88D
:1068D00000380C9B012B14D1099B6BB90021204679
:1068E000FFF7C0FF11E0A36B23F40013A363A36BB6
:1068F00043F40023A363E3E701212046FFF7B2FF3F
:1069000003E003212046FFF7ADFF10212046FFF7EB
:106910005BFF804608B14FF001082046FFF77CFF7F
:1069200008B14FF0010800232B616B61EB610AE0B5
:10693000C3B94FF00060C2F8000900220A614FF6A7
:106940007F328A6001330799994210D904EB4312D0
:1069500002F51061D2F800090028E9DB0020C2F836
:106960000009EAE74FF09040C2F80009E5E700238C
:106970000AE0C3B14FF0904CC2F800CB0022026194
:106980004FF67F3282600133994211D904EB4312F2
:1069900002F53060D2F8006B002EEADB4FF0000CFD
:1069A000C2F800CBEAE74FF0006CC2F800CBE5E795
:1069B0002B6923F480732B610023A3616FF0804364
:1069C00063610A9B1BB9A36943F01003A361A26929
:1069D0000B4B1343A3610D9B1BB1A36943F0080349
:1069E000A361012F04D04046BDE8F04104B07047D8
:1069F000A36943F0804343F00403A361F3E700BFBE
:106A000000383C80D0F8083813F0060307D0022B7A
:106A100007D0062B01D00F207047022070470020BE
:106A200070470220704710B591F800C04B78012BD9
:106A300023D000F5006ED0F81C380CF00F040122B2
:106A4000A24043EA0243C0F81C3800EB4C10D0F8D7
:106A5000003B13F4004F0ED1D0F8003BCA68C2F3DC
:106A60000A02097942EA8142134343F0805343F416
:106A70000043C0F8003B002010BDD0F81C280CF0EB
:106A80000F0E03FA0EF39BB21343C0F81C3800EB51
:106A90004C10D0F8003913F4004FECD1D0F8003985
:106AA000CA68C2F30A02097942EA814242EA8C5C6E
:106AB00043EA0C0343F0805343F40043C0F8003929
:106AC000D9E7000030B40B784A78012A26D000EBD1
:106AD0004313D3F8002B002A52DBD0F83C480A7845
:106AE00002F00F024FF0010C0CFA02F224EA02420B
:106AF000C0F83C28D0F81C28097801F00F010CFAE6
:106B000001FC22EA0C42C0F81C28D3F8001B234ADF
:106B10000A40C3F8002B002030BC704700EB431341
:106B2000D3F80029002A1EDBD0F83C580A7802F07E
:106B30000F02012404FA02F292B225EA0202C0F81E
:106B40003C28D0F81C28097801F00F018C40A4B231
:106B500022EA0404C0F81C48D3F80019104A0A407D
:106B6000C3F80029D7E7D3F8002942F00062C3F840
:106B70000029D3F8002942F08042C3F80029D3E766
:106B8000D3F8002B42F00062C3F8002BD3F8002B9F
:106B900042F08042C3F8002B9FE700BF0078F3EF7C
:106BA000007833EC70B40B784C78012C29D000EBD2
:106BB000431000F530631C69E40CE4041C611C699B
:106BC00024F0FF5424F4C0141C618C690CB1CC680F
:106BD0008C61CC68CC611C6944F400241C611C6984
:106BE000CD69C5F3120C44EA0C041C61012A66D07D
:106BF000D0F8003B43F00443C0F8003B002070BCD9
:106C000070478C696CBB00EB4314D4F8105925F025
:106C1000FF5525F4C015C4F81059D4F8105945F49F
:106C20000025C4F81059D4F81059ED0CED04C4F83F
:106C30001059012A34D000EB4313D3F8002942F055
:106C40000442C3F800298B69002BD7D0D0F8343820
:106C50000A7802F00F0101228A401343C0F8343849
:106C6000CCE700EB431404F510642569ED0CED044A
:106C70002561256925F0FF5525F4C0152561CD68EE
:106C80008E69AE4200D98D61256945F400252561E4
:106C900025698E69C6F3120C45EA0C052561C8E723
:106CA0004A691AB100EB4311C1F8142900EB4310F3
:106CB000D0F8002942F00442C0F800299EE70A6992
:106CC000002A95D05A6193E710B483B0024600239E
:106CD0000193487801280BD00B7802EB4313D3F8CB
:106CE000000B00282DDB002003B05DF8044B70473B
:106CF0000B7802EB4313D3F80049002C01DB002092
:106D0000F2E7D3F8004944F00064C3F800490B7877
:106D100002EB4313D3F8004944F08044C3F8004920
:106D2000019B01330193019C42F210739C42DBD81A
:106D30000B7802EB4313D3F80039002BF0DB002073
:106D4000D2E7D3F8000B40F00060C3F8000B0B78DB
:106D500002EB4313D3F8000B40F08040C3F8000B64
:106D6000019B01330193019842F21073984208D8B5
:106D70000B7802EB4313D3F8003B002BF0DB002031
:106D8000B2E70120B0E710B59DF8084084B903339D
:106D90004FEA930E4FF0000C08E000EB023303F5CE
:106DA000805351F8044B1C600CF1010CF445F4D3F2
:106DB000002010BDF0B583B00B784C78012C33D097
:106DC00000EB431303F5306CDCF81040E40CE404F2
:106DD000CCF81040DCF8104024F0FF5424F4C01428
:106DE000CCF810408C69002C40F0C780DCF81040D3
:106DF000CD68C5F312052C43CCF81040DCF81040E8
:106E000044F40024CCF81040012A00F0D0800A7924
:106E1000012A00F0D380D3F8002B42F00442C3F8DB
:106E2000002B002003B0F0BD8C6984BB00EB431441
:106E3000D4F8105925F0FF5525F4C015C4F81059A1
:106E4000D4F8105945F40025C4F81059D4F8105955
:106E5000ED0CED04C4F81059012A4CD000EB43139B
:106E6000D3F8004944F00444C3F800490C79012CDC
:106E70006AD08B69002BD4D0D0F834380A7802F06D
:106E80000F0101228A401343C0F83438C9E700EBF0
:106E90004314D4F81059ED0CED04C4F81059D4F88B
:106EA000105925F0FF5525F4C015C4F81059D4F831
:106EB00010698D69CF683D44013DB5FBF7F5494F39
:106EC00007EAC5453543C4F81059D4F810598E69FE
:106ED000C6F312063543C4F8105904F510640D7951
:106EE000012DB9D1256925F0C0452561256945F0F9
:106EF00000552561B0E74A691AB100EB4314C4F8A4
:106F000014290A79012A08D000EB4313D3F8002989
:106F100042F00442C3F8002983E7D0F8082812F4AD
:106F2000807F08D100EB4311D1F8002942F00052D4
:106F3000C1F80029E8E700EB4311D1F8002942F03D
:106F40008052C1F80029DFE7D0F8084814F4807FA8
:106F50000CD1D3F8004944F00054C3F80049009222
:106F60000B8B0A780969FFF70EFF5AE7D3F800493F
:106F700044F08054C3F80049F1E7CD682C44013C4B
:106F8000B4FBF5F4A4B204FB05F5CD61DCF81050B8
:106F9000144E06EAC4442C43CCF81040DCF81040F0
:106FA000CD69C5F312052C43CCF810402CE70A69D3
:106FB000002A3FF42CAFCCF8142028E7D0F808289A
:106FC00012F4807F06D1D3F8002B42F00052C3F8B0
:106FD000002B20E7D3F8002B42F08052C3F8002B9F
:106FE00019E700BF0000F81F00B583B084460846CB
:106FF0004FEA920E02F00302002305E00CF58051E7
:10700000096840F8041B01337345F7D39AB10CF5B6
:10701000805CDCF8003001934FF0000C5FFA8CF3D9
:10702000D900019BCB4000F8013B0CF1010C013A67
:1070300092B2002AF2D103B05DF804FB0B784A78D3
:10704000012A14D000EB4310D0F8002B002A06DBF5
:107050002BB1D0F8003B23F08043C0F8003BD0F8C0
:10706000003B43F40013C0F8003B0020704700EBE6
:107070004310D0F80029002A06DB2BB1D0F80039E4
:1070800023F08043C0F80039D0F8003943F40013EE
:10709000C0F80039E9E70B784A78012A0ED000EBF6
:1070A0004310D0F8003B23F40013C0F8003B0B79E9
:1070B000023BDBB2012B15D90020704700EB4310D7
:1070C000D0F8003923F40013C0F800390B79023BE3
:1070D000DBB2012BF0D8D0F8003943F08053C0F870
:1070E0000039E9E7D0F8003B43F08053C0F8003B9B
:1070F000E2E7D0F8003823F4FE63C0F80038D0F897
:107100000038090101F4FE611943C0F8001800209D
:107110007047D0F8003E23F00303C0F8003ED0F8DB
:10712000043823F00203C0F8043800207047D0F878
:10713000003E23F00303C0F8003ED0F8043843F0CB
:107140000203C0F80438002070474269806910408B
:107150007047D0F8183800F50060C0691840000C7E
:107160007047D0F8183800F50060C069184080B248
:10717000704700EB4111D1F8082B00F50060406921
:107180001040704710B4D0F81048D0F8343801F0EF
:107190000F02D340DB01DBB2234300EB411000F5CB
:1071A0001060806818405DF8044B7047406900F03B
:1071B0000100704738B50546C36823F0C043C3607B
:1071C000012913D019BBC36843F08043C360002476
:1071D0000120FAF70FF801342846FFF7E7FF08B15E
:1071E000312CF5D9322C14D0002038BDC36843F0BF
:1071F0000053C36000240120F9F7FCFF0134284646
:10720000FFF7D4FF0128EDD0312CF4D9EAE70120B3
:10721000EBE70120E9E7D0F8003923F4FF6323F01E
:107220000703C0F80039D0F8043843F48073C0F87D
:10723000043800207047000010B4046C154B9C42C9
:1072400003D9D0F8003B002B16DB0024C0F8104B0C
:10725000D0F8104B44F40024C0F8104BD0F8104B79
:1072600044F01804C0F8104BD0F8104B44F0C04460
:10727000C0F8104B012903D000205DF8044B704783
:10728000C0F8142BD0F8003B43F08023C0F8003B3B
:10729000F2E700BF0A30544F10B5D0F8D43203F1F2
:1072A000B00250F822408CB100EB820043687BB101
:1072B00094F80002FF280DD09B6894F80122214623
:1072C0009847FF2384F80032002010BD0320FCE71C
:1072D0000020FAE70020F8E70A23038000487047FF
:1072E00084000020F8B506460F4F8221384600F092
:1072F0001FFC05460121384600F01AFC0446812196
:10730000384600F015FC0DB11022AA711CB14022C4
:1073100022710022627118B1402202710022427172
:10732000432333800048F8BD40000020F8B50646EE
:107330000F4F8221384600F0FBFB054601213846FD
:1073400000F0F6FB04468121384600F0F1FB0DB158
:107350001022AA711CB1402222710022627118B160
:107360004022027100224271432333800048F8BD5D
:1073700040000020F8B506460F4F8221384600F045
:10738000D7FB05460121384600F0D2FB0446812197
:10739000384600F0CDFB0DB11022AA711CB10022BD
:1073A00022710222627118B100220271022242711E
:1073B000432333800048F8BD4000002038B5D0F8A2
:1073C000D432B03350F8235095B1044604F077F826
:1073D000C5F80C02D4F8D432B03304EB83046368EC
:1073E000DB6805F50371D5F804029847002038BD25
:1073F0000320FCE738B5D0F8C852D0F8D432B03307
:1074000050F8234084B301F00F0303EB830200EB39
:10741000820292694AB103EBC30C05EB8C05AD6C9B
:10742000B2FBF5FC05FB1C2292B10023C4F8143218
:10743000D0F8D432B03300EB830043681B69ABB1A2
:107440000A4604F50471D4F808029847002038BDB4
:1074500003EB830300EB830300249C612346224655
:1074600004F076F82046F2E70320F0E70020EEE78C
:10747000F0B583B0D0F8D43203F1B00250F82270E6
:1074800000228DF80720ADF80420002F7BD00446A1
:107490000D46097811F0600634D0202E6CD1EA88B0
:1074A0002AB311F0800F07D16B7887F80032EA8891
:1074B0003F2A13D8D2B212E0B03300EB83035B68EB
:1074C0009B68394668789847EA88072A28BF0722C8
:1074D0003946204600F0DCFE002651E0402287F8C5
:1074E00001223946204600F0E8FE002648E0B0338D
:1074F00000EB830463689B680022294668789847FC
:1075000000263DE06F780B2F31D8DFE807F0063911
:107510003030303030303030162690F89C32DBB2CC
:10752000032B04D0294600F040FB032628E002226A
:1075300001A900F0ADFE3E4622E090F89C32DBB29D
:10754000032B04D0294600F030FB032618E001226B
:107550000DF1070100F09CFE12E090F89C32DBB2C6
:10756000032B0DD0294600F020FB032608E0294616
:1075700000F01BFB032603E0294600F016FB032660
:10758000304603B0F0BD0326FAE738B50446812142
:1075900003F0BEFF002525870121204603F0B8FF38
:1075A000A4F878518221204603F0B2FFA4F84C5091
:1075B000A4F84E50D4F8D43203F1B00254F822208B
:1075C0009AB1B03304EB83035B685B689847D4F8E7
:1075D000D432B03354F8230003F07CFFD4F8D43213
:1075E000B03344F82350C4F8BC52002038BD70B505
:1075F00004464FF4077003F069FF002849D00546A0
:107600004FF4077200210BF0E1FFD4F8D432B0330D
:1076100044F82350C4F8BC52237C002B41D14FF4D2
:10762000007302228121204603F067FF012626878E
:107630004FF4007302223146204603F05EFFA4F8A7
:1076400078611023A4F84E300823032282212046BB
:1076500003F053FF0123A4F84C300026C5F8046260
:10766000D4F8D432B03304EB83035B681B689847CB
:10767000C5F81462C5F81862D5F8042262B3257CF7
:107680001DBB4FF400730121204603F069FF28461B
:1076900070BDD4F8D432B033002244F82320022540
:1076A000F5E7402302228121204603F026FF012630
:1076B0002687402302223146204603F01EFFA4F80D
:1076C00078611023A4F84E30BEE740230121204604
:1076D00003F046FF0025DAE70225D8E739B1D0F8F4
:1076E000D432B03300EB83004160002070470320A8
:1076F0007047D0F8D432B03350F823302BB1C3F8F0
:107700000812C3F810220020704703207047D0F8F9
:10771000D432B03350F823301BB1C3F80412002028
:1077200070470320704710B5D0F8D432B03350F80A
:10773000232092B1047C44B94FF40073D2F80422A0
:10774000012103F00DFF204610BD4023D2F8042292
:10775000012103F005FF0024F5E70324F3E798B1C6
:1077600008B503460020C3F8B802C3F8C402C3F842
:10777000D00209B1C3F8B412012183F89C121A7027
:10778000184603F051FE08BD0320704710B582B0C3
:107790000023ADF8063089B10446C0F8B812CB6AB0
:1077A00023B10DF106009847C4F8D002D4F8D832BE
:1077B0000133C4F8D832002002B010BD0320FBE72B
:1077C00008B503F092FE08BD08B5D0F8B83213B181
:1077D0001B68984708BD0020FCE708B5D0F8B83210
:1077E0005B68984700B908BD0320FCE738B504463C
:1077F00000F2AA25284600F0C4F90123C4F8943207
:10780000B4F8B032C4F8983294F8AA1201F01F0309
:10781000012B0DD0022B10D02BB101F0800120469E
:1078200003F07EFE03E02946204600F07FFB38BDD2
:107830002946204600F0B5FBF9E72946204600F02E
:10784000F2FBF4E7F8B50446012380F89C320023EC
:10785000C0F894324360C0F8A43280F8A032D0F867
:10786000B832DBB15B68DBB1002198470746C8B985
:10787000402300221146204603F03FFE0126A4F8D3
:1078800064614025C4F860512B46002280212046C7
:1078900003F033FEA68425623846F8BD0027E7E7EB
:1078A0000027E5E70327E3E701740020704790F81D
:1078B0009C32DBB280F89D32042380F89C32002099
:1078C000704790F89C32DBB2042B01D00020704747
:1078D00090F89D32DBB280F89C32F7E708B590F85B
:1078E0009C32DBB2032B01D0002008BDD0F8B832A7
:1078F000002BF9D0DB69002BF6D09847F4E708B5E8
:10790000D0F8D432AE3350F823205AB190F89C32DC
:10791000DBB2032B01D0002008BD136A23B19847C6
:107920000020F9E70320F7E70020F5E708B5D0F8D5
:10793000D432AE3350F823205AB190F89C32DBB2E7
:10794000032B01D0002008BD536A23B198470020C3
:10795000F9E70320F7E70020F5E70020704708B5B6
:10796000012380F89C32D0F8B83223B15B680179EA
:10797000984710B908BD0020FCE70320FAE7002073
:1079800070470020704738B504460D46002943D1A2
:107990001346D0F89422032A01D0084638BDD0F807
:1079A0005C11D0F86021914212D890F8AA3203F00D
:1079B0001F03012B17D0022B1CD0284694F89C32B1
:1079C000DBB2032B1BD0204600F08EFC2846E5E7F7
:1079D000891AC0F85C118A4228BF0A46194600F08D
:1079E0007BFC2846DAE790F8AE12FFF7C8FF0028C4
:1079F000E9D1E3E790F8AE12FFF7C3FFF7E700F134
:107A0000AE0354F823301A69002ADCD0C4F8D4023B
:107A10001B6920469847D6E701F07F01FFF7B1FFC9
:107A200090B994F89C32DBB2032BB7D100F1AE03CE
:107A300054F823309A69002AB0D0C4F8D4029B6964
:107A4000294620469847A9E70020A7E738B504460D
:107A50000D4600294BD11346D0F89422022A07D0B4
:107A600094F8A00218B1002384F8A032284638BD4B
:107A7000C269016A8A420ED88A4218D094F89C32B0
:107A8000DBB2032B27D08021204603F049FD20469E
:107A900000F035FCE4E7521AC261194600F005FC1B
:107AA00000231A461946204603F05AFDD8E7836999
:107AB0009942E3D8D0F898229342DFD200221146AF
:107AC00000F0F3FB0021C4F898120B460A4620464A
:107AD00003F046FDC4E7D4F8B832DA68002AD2D001
:107AE0000022C4F8D422DB6820469847CBE741F057
:107AF0008001FFF746FF90B994F89C32DBB2032B6C
:107B0000B5D100F1AE0354F823305A69002AAED043
:107B1000C4F8D4025B69294620469847A7E70020AD
:107B2000A5E703780A8813440B800378184470474C
:107B3000428803789A4218D930B583B004460D467E
:107B4000ADF806306288BDF806309A420AD90DF1C8
:107B50000601FFF7E6FF4378052BF3D18378AB42AC
:107B6000F0D100E0002003B030BD00207047034694
:107B7000002002E00130C0B201331A78002AF9D1A6
:107B800070470B7803704B7843708B78CA7843EA60
:107B9000022343800B794A7943EA022383808B795D
:107BA000CA7943EA0223C380704710B50446802196
:107BB00003F0B6FC0021204603F0B2FC10BD30B546
:107BC00083B004460D460023ADF806304A88130AF8
:107BD000013B062B00F2AB80DFE803F0041F33A962
:107BE000A98D9A00D0F8B4321B680DF10601007C13
:107BF0009847EA88002A00F0A380BDF80630002BE1
:107C000000F099809A4228BF1A46ADF80620014636
:107C1000204600F03DFB03B030BD037C43B9D0F8F3
:107C2000B8329B6A0DF10600984702234370E0E7E3
:107C3000D0F8B832DB6A0DF1060098470223437092
:107C4000D7E7D2B2052A52D8DFE802F003101D2A86
:107C50003744D0F8B4325B6823B10DF10601007CE3
:107C60009847C6E72946FFF7A0FFD4E7D0F8B4321B
:107C70009B6823B10DF10601007C9847B9E72946BE
:107C8000FFF793FFC7E7D0F8B432DB6823B10DF1FB
:107C90000601007C9847ACE72946FFF786FFBAE764
:107CA000D0F8B4321B6923B10DF10601007C98476E
:107CB0009FE72946FFF779FFADE7D0F8B4325B695B
:107CC00023B10DF10601007C984792E72946FFF7A2
:107CD0006CFFA0E7D0F8B4329B6923B10DF1060127
:107CE000007C984785E72946FFF75FFF93E7294621
:107CF000FFF75BFF8FE7037C33B9D0F8B8325B6BDB
:107D00000DF10600984774E72946FFF74EFF82E71A
:107D1000037C43B9D0F8B8321B6B0DF106009847CD
:107D20000723437065E72946FFF73FFF73E72946BE
:107D3000FFF73BFF6FE729462046FFF736FF6AE76C
:107D4000204600F0D1FA66E738B504468B88FBB9C7
:107D5000CB88EBB94B887F2B1AD803F07F0590F8BE
:107D60009C32DBB2032B0CD080F89E52294603F0E4
:107D7000E7FB204600F0B8FA35B1022384F89C32C4
:107D800009E0FFF712FF06E0012384F89C3202E0CD
:107D90002046FFF70AFF38BD70B504460E468D78C1
:107DA0002F4B1D70012D10D890F89C32DBB2022BA6
:107DB0000FD0032B26D0FFF7F8FE294B1978204669
:107DC000FFF70BFD0325284670BDFFF7EEFE0325E8
:107DD000F9E7A5B145602946FFF7F6FC054638B13D
:107DE00031462046FFF7E1FE022384F89C32EAE7A1
:107DF000204600F079FA032384F89C32E3E700F090
:107E000073FAE0E7CDB141688D4225D0C9B2FFF7E2
:107E1000E4FC134B197861602046FFF7D5FC05465A
:107E2000B0B131462046FFF7C0FE21792046FFF76A
:107E3000D4FC022384F89C32C5E7022380F89C32EC
:107E400045602946FFF7C9FC204600F04DFABAE725
:107E5000204600F049FAB6E700F046FA0025B2E7FE
:107E6000D80E002008B5CB88012B0BD190F89C329E
:107E7000DBB2022B09D9032B09D10122011D00F02D
:107E800007FA01E0FFF791FE08BD5BB213B9FFF7F7
:107E90008CFEF9E70146002341F8083F012200F07B
:107EA000F7F9F1E708B590F89C32013B022B12D8A4
:107EB000CB88022B0CD10123C360D0F8A4320BB1C4
:107EC0000323C360022200F10C0100F0E1F908BDB8
:107ED000FFF76BFEFBE7FFF768FEF8E708B54B8896
:107EE000012B04D0022B07D0FFF75FFE08BDC0F8BE
:107EF000A43200F0F9F9F9E78B881B0A80F8A03268
:107F000000F0F2F9F2E708B590F89C32013B022B41
:107F100009D84B88012B00D008BD0023C0F8A4323B
:107F200000F0E2F9F8E7FFF740FEF5E738B50C7826
:107F300004F06004202C06D0402C04D06CB1FFF774
:107F400034FE002407E0D0F8D432AE3350F82330AA
:107F50009B6898470446204638BD4D78092D1DD8AA
:107F6000DFE805F012191C161C08051C0F0BFFF7A3
:107F700026FEF0E7FFF7E8FEEDE7FFF70DFF04460A
:107F8000E9E7FFF76FFFE6E7FFF78CFF2C46E2E734
:107F9000FFF7A4FFDFE7FFF7B6FFDCE7FFF705FE1B
:107FA000D9E770B505460C460B7803F06003202B2B
:107FB00007D0402B05D023B1FFF7F7FD0026304650
:107FC00070BD95F89C32013B022B26D821790129FE
:107FD00005D921462846FFF7E8FD0026EFE72846A9
:107FE000FFF7CDFC68B900F1AE0255F82220916888
:107FF00089B1C5F8D40293682146284698470646B9
:1080000000E00326E388002BD9D1002ED7D12846E3
:1080100000F06AF9D3E70326F4E721462846FFF784
:10802000C4FD0026CBE72DE9F04106460D468B88BE
:10803000DFB20C7804F06004202C08D0402C06D06D
:10804000DCB1FFF7B2FD00242046BDE8F0813946DF
:108050003046FFF796FC0446002840F0F880C6F84A
:10806000D40200F1AE0356F823309B68002BEBD00E
:108070002946304698470446E6E791F80180B8F172
:10808000010F31D0B8F1030F05D0B8F1000F67D060
:10809000FFF78BFDD8E790F89C32DBB2022B04D0BF
:1080A000032B12D0FFF781FDCEE70FB1802F04D153
:1080B00029463046FFF779FDC6E7394603F030FA26
:1080C0008021304603F02CFABEE74B8823B91FB15C
:1080D000802F01D0CB881BB1304600F005F9B3E703
:1080E000394603F01DFAF7E790F89C32DBB2022B19
:1080F00004D0032B12D0FFF758FDA5E70FB1802F56
:1081000004D129463046FFF750FD9DE7394603F07C
:1081100007FA8021304603F003FA95E74B88002BDD
:1081200092D117F07F0F17D1304600F0DDF83946B5
:108130003046FFF726FC002886D1C6F8D40200F1AD
:10814000AE0256F822209268002A00F0828029466A
:1081500030469047044677E7394603F0E9F9E3E70C
:1081600090F89C22D2B2022A05D0032A27D0FFF72A
:108170001CFD444668E70FB1802F13D113F0800F28
:1081800014D107F07F0707EB8707B90001F5A87145
:108190003144043100230B600222304600F078F8AD
:1081A000444651E7FFF701FD44464DE707F07F07DE
:1081B00007EB8707B900103131440431EAE75BB2BD
:1081C000002B1FDB07F00F0202EB820200EB8202A2
:1081D000B2F864211AB3002B25DB07F07F0303EB11
:1081E00083039C0004F5A874344404340FB1802F39
:1081F00022D10023236002222146304600F048F8B5
:10820000444621E707F00F0202EB820200EB8202F4
:10821000928C002ADFD1FFF7C8FC444614E7FFF731
:10822000C4FC444610E707F07F0303EB83039C0084
:10823000103434440434D9E73946304603F028F981
:1082400010B101232360D6E700232360D3E7002485
:10825000FAE60446F8E6D0B170B50D461646044677
:10826000FFF785FC431C5B009BB233802B7003231C
:108270006B70022307E0EA5401345A1CD2B2002189
:10828000A9540233DBB22278002AF4D170BD7047C2
:1082900008B513460222C0F894228361C3610A46DE
:1082A000002103F055F9002008BD08B513460A4621
:1082B000002103F04DF9002008BD08B51346032244
:1082C000C0F89422C0F85831C0F85C310A46002149
:1082D00003F046F9002008BD08B513460A46002100
:1082E00003F03EF9002008BD08B50422C0F894222E
:1082F00000231A46194603F02BF9002008BD08B5E3
:108300000522C0F8942200231A46194603F028F9E2
:10831000002008BD842801D003307047002070473A
:1083200008B500F039FD002008BD2DE9F04387B005
:1083300004460F464569BDB18669AEB1D0F80480E8
:10834000D0F80090B0F90800FFF7E4FF029601951D
:1083500000903B4622694946404600F0ADFC05903E
:10836000059807B0BDE8F08365682668D4F81080EA
:10837000B4F90800FFF7CEFF05AB019300903B4630
:108380001FFA88F23146284600F0D1FC0128E7D0D8
:108390000020E6E708B500B9012000F047FE002004
:1083A00008BD00F1080343604FF0FF328260C360F4
:1083B0000361002303607047002303617047436833
:1083C0004B609A688A605160996008610368013364
:1083D0000360704730B40D68B5F1FF3F11D000F174
:1083E00008031C465B681A68AA42FAD963684B60A6
:1083F00099608C606160086103680133036030BC80
:1084000070470469F2E70369416882688A604168DD
:1084100051605A68824206D0002202611A68013A0D
:108420001A601868704782685A60F5E782B00023C6
:1084300001930D4B1B68B3F1FF3F08D04FF0500381
:1084400083F31188BFF36F8FBFF34F8FFEE74FF0B9
:10845000500383F31188BFF36F8FBFF34F8F019BDE
:10846000002BFCD002B07047900000200848006844
:10847000006880F308884FF0000080F3148862B62B
:1084800061B6BFF34F8FBFF36F8F00DF00BF0000F7
:1084900008ED00E0DFF80C00016841F470010160B4
:1084A0007047000088ED00E04FF0807340F8043C16
:1084B00021F0010140F8081C054B40F80C3C40F845
:1084C000202C6FF0020340F8243C4438704700BF72
:1084D0002D840008000000000000000000000000E3
:1084E000074B19680868B0E8F04F80F30988BFF3BC
:1084F0006F8F4FF0000080F311887047AFF300805A
:10850000205D00204FF0500383F31188BFF36F8F7D
:10851000BFF34F8F0B4A136801331360012B00D058
:1085200070474FF0E023D3F8043D13F0FF0FF7D06E
:108530004FF0500383F31188BFF36F8FBFF34F8F5A
:10854000FEE700BF90000020094B1B6843B94FF0C5
:10855000500383F31188BFF36F8FBFF34F8FFEE794
:10856000013B034A13600BB983F31188704700BFC6
:10857000900000200000000000000000000000004B
:10858000EFF30980BFF36F8F154B1A681EF0100FC1
:1085900008BF20ED108A20E9F04F10602DE9090096
:1085A0004FF0500080F31188BFF34F8FBFF36F8FF0
:1085B00000F062FD4FF0000080F3118809BC1968DB
:1085C0000868B0E8F04F1EF0100F08BFB0EC108A3A
:1085D00080F30988BFF36F8F704700BFAFF300804F
:1085E000205D002008B54FF0500383F31188BFF3DE
:1085F0006F8FBFF34F8F00F011FC28B14FF0E023D5
:108600004FF08052C3F8042D002383F3118808BD76
:108610004FF0E022002313619361054B1B6805496D
:10862000A1FB03139B09013B5361072313617047AF
:1086300094000020D34D62104FF0E023D3F8002DBA
:108640003D4B9A421CD04FF0E023D3F8002D3B4B1A
:108650009A421ED030B583B0394B1A78D2B201920B
:10866000FF221A701B78DBB28DF803309DF80330BF
:1086700003F05003334A1370334B07221A601BE098
:108680004FF0500383F31188BFF36F8FBFF34F8F09
:10869000FEE74FF0500383F31188BFF36F8FBFF3F2
:1086A0004F8FFEE7284A1368013B13609DF80330A3
:1086B0005B00DBB28DF803309DF8033013F0800FC0
:1086C000F0D1214B1B68032B08D04FF0500383F3EC
:1086D0001188BFF36F8FBFF34F8FFEE71B021A4A5B
:1086E000136003F4E0631360019BDBB2144A137060
:1086F0004FF0E024D4F8203D43F47003C4F8203D4B
:10870000D4F8203D43F07043C4F8203DFFF780FFCC
:1087100000250E4B1D60FFF7BDFED4F8343F43F03B
:108720004043C4F8343FFFF7A1FE00F0A5FCFFF77B
:108730007DFE284603B030BD71C20F4170C20F41AB
:1087400000E400E0D90E0020DC0E002090000020A4
:10875000134A12F0070F1FD0D11D21F00701C1F5F8
:108760009C43203313440A460E48026000214160B6
:108770001344083B23F007030B480360596019605A
:10878000991A51601360094B1960094B1960094B24
:108790004FF000421A60704744F62063E4E700BFE0
:1087A000E40E0020185D0020E00E00200C5D00208B
:1087B000085D0020045D0020164B1A461B688342AA
:1087C000FBD3516802EB010C844509D0416800EBF2
:1087D000010C634509D00360904219D010607047C6
:1087E0004068014451601046F0E710B40A4C246818
:1087F000A3420BD05B681944416013681B68036097
:10880000904200D010605DF8044B70470460F7E7B9
:10881000704700BF185D0020E00E002070B50546CF
:1088200000F0F4FA364B1B68A3B1364B1B681D42AF
:108830004ED135B1083515F0070F02D025F00705E8
:108840000835002D46D0304B1B68AB4251D32F4A20
:10885000146804E0FFF77CFFE7E722461C466368E4
:10886000AB4202D22368002BF7D1254B1B68A342F1
:1088700041D0166808362368136063685B1B102BB1
:1088800010D9601910F0070F08D04FF0500383F390
:108890001188BFF36F8FBFF34F8FFEE743606560B2
:1088A000FFF78AFF626818490B689B1A0B6018492A
:1088B00009688B4201D216490B60124B1B681343A7
:1088C000636000232360134A13680133136002E0DE
:1088D000002600E0002600F02DFB16F0070F0CD05C
:1088E0004FF0500383F31188BFF36F8FBFF34F8FA7
:1088F000FEE70026EFE70026EDE7304670BD00BF3B
:10890000E00E0020045D0020085D0020185D0020BE
:108910000C5D0020105D0020002834D038B50446DE
:10892000A0F1080550F8043C174A1268134208D118
:108930004FF0500383F31188BFF36F8FBFF34F8F56
:10894000FEE750F8081C41B14FF0500383F3118843
:10895000BFF36F8FBFF34F8FFEE723EA020340F8A8
:10896000043C00F053FA54F8041C084A13680B4402
:1089700013602846FFF720FF054A13680133136090
:1089800000F0D8FA38BD7047045D0020085D002073
:10899000145D0020084B1B681B6823B9074B4FF080
:1089A000FF321A607047044B1B68DB68DB685A684B
:1089B000024B1A60704700BF245D0020F85D002064
:1089C0002DE9F04707469846089DDDF824900A9C5B
:1089D000266B02F18042013A06EB820626F007067A
:1089E00000293AD08E464FF0000CBCF11F0F0BD877
:1089F0001EF80C2004EB0C0383F834201EF80C3016
:108A000013B10CF1010CF0E7002384F85330062D6C
:108A100000D90625E56265654FF0000AC4F858A044
:108A2000201DFFF7C9FC04F11800FFF7C5FC246105
:108A3000C5F10705A5616462C4F85CA084F860A074
:108A4000424639463046FFF72FFD2060B9F1000F4E
:108A500001D0C9F80040BDE8F087002384F8343025
:108A6000D5E7000038B5002407E004EB840293004A
:108A70000E481844FFF795FC0134062CF5D90C4D2F
:108A80002846FFF78EFC0B4C2046FFF78AFC0A486D
:108A9000FFF787FC0948FFF784FC0948FFF781FCD2
:108AA000084B1D60084B1C6038BD00BF2C5D0020CA
:108AB000CC5D0020E05D0020045E0020305E0020E0
:108AC0001C5E0020245D0020285D002010B50446B7
:108AD000FFF718FD214A136801331360204B1B6810
:108AE0005BB1204B1B686BB91D4B1B68DA6AE36AEC
:108AF0009A4207D81A4B1C6004E0194B1C6013689B
:108B0000012B28D0184A136801331360E06A01234F
:108B10008340164A11680B43136000EB8000211D4F
:108B2000134B03EB8000FFF74AFCFFF70DFD0D4BE5
:108B30001B687BB10A4B1B68DA6AE36A9A4209D266
:108B40004FF0E0234FF08052C3F8042DBFF34F8F56
:108B5000BFF36F8F10BDFFF785FFD3E7B85D00202F
:108B6000205D0020185E0020C45D0020C85D00204C
:108B70002C5D002010B5044690F8613063B1012BE4
:108B800011D0022B0ED04FF0500383F31188BFF3A6
:108B90006F8FBFF34F8FFEE7006BFFF7BDFE2046E0
:108BA000FFF7BAFE10BDFFF7B7FEFBE70F4B1B68E0
:108BB000D3B110B5FFF7A6FC0D4BDB68DC68201DB8
:108BC000FFF721FC0B4A1368013B1360074A136847
:108BD000013B1360FFF7B8FC2046FFF7CBFF034BC8
:108BE0001B68002BE6D110BD704700BFBC5D0020A4
:108BF000305E0020B85D002008B5FFF7D7FF074BB7
:108C00001B68012BF9D94FF0E0234FF08052C3F8D5
:108C1000042DBFF34F8FBFF36F8FEEE72C5D002065
:108C200070B504460D461D4B1E681D4B1868043078
:108C3000FFF7E9FB50B91A4B1B68DA6A012303FA04
:108C400002F218490B6823EA02030B60B4F1FF3FFC
:108C50000DD03444124B1B685C60A64210D9124BF5
:108C600018680F4B19680431FFF7B4FB70BD002D75
:108C7000EFD00B4B196804310C48FFF7A0FBF5E768
:108C80000B4B1868064B19680431FFF7A3FB094B1F
:108C90001B68A342EAD9074B1C60E7E7445E00204B
:108CA000205D0020C85D0020285D00201C5E0020A3
:108CB000245D0020F85D002030B587B00B9C7CB1AE
:108CC0000C9DB5B164250495049D642D1AD04FF018
:108CD000500383F31188BFF36F8FBFF34F8FFEE70D
:108CE0004FF0500383F31188BFF36F8FBFF34F8FA3
:108CF000FEE74FF0500383F31188BFF36F8FBFF38C
:108D00004F8FFEE7049D0C9D2C63022485F8614083
:108D100000240394029505AC01940A9C0094FFF78B
:108D20004FFE0C98FFF7D2FE059807B030BD2DE935
:108D3000F04385B00746884614461E469000FFF76C
:108D40006DFD00B381466420FFF768FD0546B0B1B4
:108D5000C0F83090E5B1002385F8613003930295A7
:108D60000D9B01930C9B00933346224641463846A7
:108D7000FFF726FE2846FFF7A9FE012005E048463A
:108D8000FFF7CAFDE6E74FF0FF3005B0BDE8F0831E
:108D90004FF0FF30F9E7000010B588B000240594CB
:108DA000069407AA06A905A800F006FF059B0293F2
:108DB000069B019300942346079A0E490E48FFF73D
:108DC0007BFF0E4B186090B14FF0500383F3118876
:108DD000BFF36F8FBFF34F8F094B4FF0FF321A6015
:108DE000084B01221A60084B1C60FFF725FC08B0F5
:108DF00010BD00BFF43C0108F98B0008F45D0020B1
:108E0000F85D0020185E0020445E0020024A1368CE
:108E100001331360704700BFC05D0020F8B53A4BC6
:108E20001B68002B69D1394B1D6801351D60C5B920
:108E3000374B1B681B6843B14FF0500383F3118815
:108E4000BFF36F8FBFF34F8FFEE7314A1168314B8D
:108E5000186810601960304A136801331360FFF717
:108E600099FD2E4B1B68AB423DD900272C4B1B684C
:108E7000DB6A03EB83039A002A4B9B58012B00D932
:108E80000127294B1B68002B3CD001273AE0012722
:108E90001F4B1B681B6843B31D4B1B68DB68DC68FA
:108EA00063689D4226D3261D3046FFF7ACFAA36ABD
:108EB0001BB104F11800FFF7A6FAE36A01229A40F9
:108EC0001A49086802430A6003EB83039A0031469B
:108ED00014481044FFF773FAE26A114B1B68DB6A0F
:108EE0009A42D4D2D4E70027D2E70C4B4FF0FF329E
:108EF0001A60BBE7094A1360B8E70D4A13680133EB
:108F0000136000273846F8BDC05D0020445E002095
:108F1000245D0020285D0020FC5D0020F85D00201D
:108F2000205D00202C5D0020485E0020C85D0020F0
:108F3000005E002038B5354B1B6843B94FF0500335
:108F400083F31188BFF36F8FBFF34F8FFEE7FFF7F7
:108F5000D9FA2E4B1A68013A1A601B68002B4FD1C0
:108F60002B4B1B680BB900244BE00024294B1B68DA
:108F70001BB3284BDB68DC6804F11800FFF743FAE9
:108F8000251D2846FFF73FFAE06A01238340224A65
:108F900011680B43136000EB800029461F4B03EB65
:108FA0008000FFF70CFAE26A1D4B1B68DB6A9A42ED
:108FB000DCD31C4B01221A60D8E70CB1FFF7EAFCA6
:108FC000194B1C6884B9174B1C68D4B14FF0E023CF
:108FD0004FF08052C3F8042DBFF34F8FBFF36F8F54
:108FE00001240EE0013C07D0FFF718FF0028F9D05C
:108FF0000C4B01221A60F5E70B4B00221A60E2E7E6
:109000000024FFF7A1FA204638BD00BFC05D002054
:10901000B85D0020045E0020C85D00202C5D0020AB
:10902000205D0020485E0020005E002010B5A8B141
:109030000446104B1B6843B14FF0500383F3118873
:10904000BFF36F8FBFF34F8FFEE7FFF7DFFE002107
:109050002046FFF7E5FDFFF76DFF48B94FF0E0232D
:109060004FF08052C3F8042DBFF34F8FBFF36F8FC3
:1090700010BD00BFC05D0020204B1B681BB1204B02
:1090800001221A6070471E4B00221A601D4B1B689C
:10909000B3FA83F3DBB2C3F11F0303EB83018A004E
:1090A00019498A5842B94FF0500383F31188BFF32E
:1090B0006F8FBFF34F8FFEE7134903EB83008200EE
:1090C0000A4450684068506003EB830C4FEA8C02FE
:1090D00008321144884209D003EB83039A000A4BFB
:1090E00013445B68DA68094B1A607047406862464F
:1090F0009100054A0A445060EEE700BFC05D0020C1
:10910000485E0020C85D00202C5D0020205D00200E
:109110000369C268934204D88068801A0344581EC9
:1091200070479B1A581E70472DE9F843044688463D
:109130001646C5688768A7EB0509914509D94068B7
:109140002844F7F715FEBFF35F8F3544E560BDE8AF
:10915000F88340684A462844F7F70AFEED1B354479
:109160002A4608EB09016068F7F702FEBFF35F8F3C
:10917000E560ECE72DE9F843064688461746C568E2
:109180004FF000091AE0641B621EB3685C1B944236
:1091900028BF1446BC4228BF3C4670682246414660
:1091A0002844F7F7E5FDA144A0443F1B2544B368DC
:1091B000AB420BD0BFF35F8FF5604FB13469A5426E
:1091C000E1D3B268641B1444621EDEE70025F1E7B8
:1091D0004846BDE8F883000010B5154CA8220021D0
:1091E00020460AF0F3F9032323616361114AA26167
:1091F000114BE3614FF4806323620023A362636237
:10920000E36222660D4A62661022A2662367E36665
:109210006367BFF35F8F06E0C3F10F020849895C03
:10922000034AD15401330F2BF6D9BFF35F8F10BD22
:109230004C5E0020FC3C0108045F0020F45E00202E
:10924000083D0108F8B50F461646184B451C05EBBE
:10925000450503EBC50500EB400003EBC000C46A05
:10926000012C11D0022C1CD014B100242046F8BDD2
:109270002846FFF74DFF8642F8D832463946284641
:10928000FFF752FF3446F1E72846FFF741FF344627
:10929000864228BF0446224639462846FFF744FF47
:1092A000E4E72846FFF766FF0446DFE74C5E002050
:1092B000F8B504460D461646094B1B786BB1EFF323
:1092C00011874FF0200181F311883246294620464C
:1092D000FFF7B8FF87F31188F8BDFFF77DFFEEE7D2
:1092E0004C5E002008B5FFF777FF08BD10B50446B7
:1092F0008268531C4068834205D820688154A3606B
:10930000E3680133E360A26863689A4200D010BD4D
:1093100021682069FFF7CCFFA368984203D04FF083
:10932000FF33E360F3E70023A360F0E72DE9F84F94
:1093300081460F4615461E46DDF828A00B9A0B46BF
:109340004FF0010803E0B3FBF5F308F10108AB426D
:10935000F9D2B04500D2B04612F0010B18D1BAF1E3
:10936000000F15D012F0020F02D0BEB1202400E091
:109370002024BAF1000F0BD0C24509D90AF1FF3AF7
:1093800021464846FFF7B2FFD9F80C30002BF0DA3F
:10939000D9F80C30002B25DB012404E03024E8E769
:1093A000013E05FB04F4012EFAD8B7FBF4F39D420D
:1093B000F7D900E01C46B7FBF4F304FB1377124A1D
:1093C000D15C4846FFF792FFD9F80C30002B03DB45
:1093D000B4FBF5F3AC42EDD2BBF1000F02D0BAF111
:1093E000000F01D1BDE8F88FBAF1000FFAD0C245E5
:1093F000F8D90AF1FF3A20214846FFF777FFD9F85C
:109400000C30002BF0DAEDE71C3D01082DE9F047A8
:1094100082B007468846154699460A9EDDF82CA07C
:1094200081EAE17CACEBE17C012402E09CFBF5FCF1
:1094300001346545FADD4C4500D24C4636B1B8F1F1
:10944000000F02DB1AF0040F00D0013E1AF0020FE9
:1094500002D0B9F1000F03D01AF0010F00D1AEB95C
:10946000FB68002B0FDBB8F1000F1CDB1AF0040FB8
:1094700020D1FB68002B06DB0AF00303022B1ED071
:10948000FB68002B2DDA02B0BDE8F087002EE7D094
:10949000A642E5D9013E20213846FFF727FFFB68A9
:1094A000002BF3DADCE7C8F100082D213846FFF77E
:1094B0001DFFDEE72B213846FFF718FFD9E7B9F18A
:1094C000000FDDD1002EDBD0002ED9D0A642D7D997
:1094D000013E30213846FFF709FFFB68002BF3DA25
:1094E000CEE7CDF804A000964B462A4641463846C2
:1094F000FFF71CFFC7E70000F0B599B006460C4621
:10950000154603AB13934023149300231593179030
:1095100016938AE00020012211E040F0010001349E
:109520000CE040F00200013408E040F00400013497
:1095300004E040F00800013400E0002212B3237878
:10954000233B0D2BF9D801A151F823F033950008E6
:109550003B9500083B9500083B9500083B950008AB
:109560003B9500083B9500083B9500082B950008AB
:109570003B9500081B9500083B9500083B950008AB
:10958000239500082378A3F13001C9B2092907D82F
:10959000013402EB820203EB4203A3F13002F1E754
:1095A0002E2B02D00023217813E00134002305E0A4
:1095B000013403EB830301EB4303303B2178A1F13A
:1095C000300C5FFA8CFCBCF1090FF1D9EBE714F811
:1095D000011F6C29FBD06829F9D025296DD020D333
:1095E00078291ED858291CD35839202919D8DFE8E2
:1095F00001F03D18181818181818181818112718FD
:109600001818181818181818181857181848183251
:1096100018183D002B681A1D2A60197813A8FFF747
:1096200065FE0134169B002B4CDB14F8011B00294E
:1096300048D025293FF46EAF13A8FFF757FEF1E796
:1096400029680F1D2F600968019000920A2213A853
:10965000FFF7DCFEE5E729680F1D2F600968019020
:1096600000920A2213A8FFF761FEDAE729680F1DAE
:109670002F60096801900092102213A8FFF756FE90
:10968000CFE72B681A1D2A601F6817F8011B0029F5
:10969000C7D013A8FFF72AFE169B002BF5DAC0E708
:1096A0002B681A1D2A601968002301930823009370
:1096B000102213A8FFF73AFEB3E7252113A8FFF7FE
:1096C00015FEAEE7169B002B05DD159A32B9159AEB
:1096D000169B13441693169819B0F0BD03A9304693
:1096E000FFF7E6FDF3E700BF0EB400B582B003ABB1
:1096F00053F8041B019301AAFFF7FEFE02B05DF8C8
:1097000004EB03B07047000000B585B00023009360
:109710000193029303931548154A02604FF40032F7
:10972000426083600361037680F82030C362114A8F
:109730008262C3600122C26180F830304261F7F773
:1097400007FE68B9102300930123019300230293BD
:1097500069460648F7F728FE28B905B05DF804FB0E
:1097600000F044FCEEE700F041FCF6E70463002063
:10977000002001400100000F0268184B9A4200D0FF
:10978000704710B582B0044600230193144A516C0F
:1097900041F480715164526C02F480720192019A1A
:1097A0001048114A026043608360C3604FF48062D6
:1097B00002614FF4006242614FF400528261C36162
:1097C00003624362F8F7E2FB20B9064BA3639C6394
:1097D00002B010BD00F00AFCF7E700BF0020014016
:1097E000003802404C6300207064024008B50E4807
:1097F0000E4B03600323436000238360C3604FF478
:10980000102202614FF400124261037643768376A0
:109810000122C27603774277F7F792FE00B908BDBE
:1098200000F0E4FBFBE700BFB063002000640040F1
:1098300008B50E480E4B036003234360002383608A
:10984000C3604FF4102202614FF4001242610376AC
:10985000437683760122C27603774277F7F770FE6C
:1098600000B908BD00F0C2FBFBE700BFD8630020D1
:109870000068004010B58AB0002305930693079353
:10988000089309930368454A934204D0444A93429B
:109890003CD00AB010BD434A136801331360012B5A
:1098A00027D000240194404B1A6B42F008021A633F
:1098B0001B6B03F008030193019B03230593022212
:1098C000069208930923099305A93848F8F764FE1E
:1098D000224605211420F8F747FA1420F8F77CFAFD
:1098E000224605211520F8F73FFA1520F8F774FAFB
:1098F000CFE7002300932C4B1A6C42F000721A64DD
:109900001B6C03F000730093009BCAE700230293D3
:10991000254B1A6C42F080621A641B6C03F0806362
:109920000293029B1F4A136801331360012B28D056
:10993000002404941C4B1A6B42F002021A631B6B46
:1099400003F002030493049B602305930223069310
:10995000032308930923099305A91548F8F71CFE6A
:10996000224605214020F8F7FFF94020F8F734FAA5
:10997000224605214120F8F7F7F94120F8F72CFAA3
:1099800087E700230393084B1A6C42F000721A64B5
:109990001B6C03F000730393039BC9E70064004052
:1099A00000680040AC63002000380240000C024018
:1099B0000004024008B50548054B0360F8F71AFAA1
:1099C00000B908BD00F012FBFBE700BF00640020F7
:1099D000003002400268094B9A4200D0704782B0C2
:1099E00000230193064B1A6B42F480521A631B6BDF
:1099F00003F480530193019B02B070470030024092
:109A00000038024000B583B00023009301930C4856
:109A10000C4B0360F8F7FDF958B90023009301934C
:109A2000102269460648F8F706FA28B903B05DF82F
:109A300004FB00F0DBFAF0E700F0D8FAF6E700BF2D
:109A4000086400200074004000B589B0002303932F
:109A500004930593069307930268134B9A4202D02E
:109A600009B05DF804FB0021019103F5E2331A6CA3
:109A700042F000521A641A6C02F000520192019AEC
:109A800002911A6B42F001021A631B6B03F001038F
:109A90000293029B202303930323049303A9034807
:109AA000F8F77AFDDCE700BF0074004000000240D8
:109AB00010B582B0002400943A4B1A6B42F4800235
:109AC0001A631A6B02F480020092009A01941A6BD6
:109AD00042F400121A631B6B03F400130193019B01
:109AE000224605210C20F8F73FF90C20F8F774F90D
:109AF000224605210D20F8F737F90D20F8F76CF90B
:109B0000224605210E20F8F72FF90E20F8F764F908
:109B1000224605210F20F8F727F90F20F8F75CF906
:109B2000224605212F20F8F71FF92F20F8F754F9C6
:109B3000224605213820F8F717F93820F8F74CF9B4
:109B4000224605213A20F8F70FF93A20F8F744F9B0
:109B5000224605213B20F8F707F93B20F8F73CF9AE
:109B6000224605213C20F8F7FFF83C20F8F734F9AD
:109B7000224605214420F8F7F7F84420F8F72CF99D
:109B8000224605214520F8F7EFF84520F8F724F99B
:109B9000224605214620F8F7E7F84620F8F71CF999
:109BA00002B010BD0038024008B501F01BFB0120D7
:109BB000FEF7F0FBFBE70000034B0360034B0B6079
:109BC00080231360704700BF2066002020640020BF
:109BD00010B588B00DF1040C074C0FCCACE80F00A9
:109BE00094E807008CE80700002101A8FEF79DFB20
:109BF000024B186008B010BD0C3C01081C6400202A
:109C00002DE9F0438FB0002409940A940B940C942E
:109C10000D9400945F4B1A6B42F002021A631A6BA8
:109C200002F002020092009A01941A6B42F0400284
:109C30001A631A6B02F040020192019A02941A6BA5
:109C400042F001021A631A6B02F001020292029AB8
:109C500003941A6B42F008021A631A6B02F00802AE
:109C60000392039A04941A6B42F004021A631A6B6B
:109C700002F004020492049A05941A6B42F4807272
:109C80001A631A6B02F480720592059A06941A6B95
:109C900042F020021A631A6B02F020020692069A22
:109CA00007941A6B42F080021A631A6B02F080026A
:109CB0000792079A08941A6B42F010021A631B6B02
:109CC00003F010030893089B334F22464021384687
:109CD000F8F754FD314E012210213046F8F74EFDC1
:109CE000DFF8C080012211464046F8F747FD4023C7
:109CF000099301250A950B940C9409A93846F8F7A5
:109D00004BFC082309934FF40419CDF828900B95C8
:109D100009A93846F8F740FC09950A940B9509A95A
:109D20003046F8F739FC102309930A950B95022762
:109D30000C9709A93046F8F72FFC30230993CDF88A
:109D400028900B9409A91648F8F726FC09950A955E
:109D50000B950C9709A94046F8F71EFC22460521F1
:109D60000920F8F701F80920F8F736F8224605210E
:109D70000A20F7F7F9FF0A20F8F72EF82246052106
:109D80001720F7F7F1FF1720F8F726F80FB0BDE816
:109D9000F08300BF0038024000180240000002407B
:109DA000000802400004024008B50B480B4B03605A
:109DB0000B4B436000238360C3604FF48042026119
:109DC00043618361C3610362F8F7ACFE00B908BD6B
:109DD00000F00CF9FBE700BF44670020005800408A
:109DE000801A060008B50B480B4B03600B4B436011
:109DF00000238360C3604FF480420261436183614A
:109E0000C3610362F8F78EFE00B908BD00F0EEF8FA
:109E1000FBE700BF98670020005C0040801A060046
:109E20002DE9F0418AB00023059306930793089328
:109E3000099303685D4A934205D05D4A934269D015
:109E40000AB0BDE8F081044600250095594E336BF9
:109E500043F020033363336B03F020030093009B34
:109E6000032305931222069208930423099305A95C
:109E70005148F8F791FB0195336C43F48003336448
:109E8000336C03F480030193019B4C484C4B0360FB
:109E90004FF0606343608560C5604FF48063036189
:109EA00045618561C56105624562F8F76FF858BB89
:109EB000424BA3639C634348434B03604FF0606392
:109EC0004360402383600023C3604FF480620261DB
:109ED00043618361C36103624362F8F757F8B0B925
:109EE000384B63639C63002205212120F7F73CFF78
:109EF0002120F7F771FF002205212220F7F734FF18
:109F00002220F7F769FF9BE700F070F8D0E700F038
:109F10006DF8E5E700250295264C236B43F004031A
:109F20002363236B03F004030293029B0395236BCB
:109F300043F001032363236B03F001030393039BAB
:109F40004FF4007305934FF01208CDF818800327E3
:109F500008970426099605A91C48F8F71DFB4FF43D
:109F600080730593CDF8188007950897099605A981
:109F70001748F8F711FB0495236C43F4000323649E
:109F8000236C03F400030493049B2A460521482014
:109F9000F7F7EAFE4820F7F71FFF2A460521492078
:109FA000F7F7E2FE4920F7F717FF49E700580040AE
:109FB000005C00400038024000140240846600202B
:109FC00040600240E4660020B860024000080240A1
:109FD0000000024008B50268034B9A4200D008BD59
:109FE000F7F7F6F8FBE700BF0020004072B6FEE787
:109FF00000B595B03022002108A809F0E7FA002347
:10A00000039304930593069307930193204A116CDD
:10A0100041F080511164126C02F080520192019A59
:10A0200002931C4B1A6842F480421A601B6803F4C6
:10A0300080430293029B012308934FF480330993DA
:10A0400002230E934FF480020F9206221092A82250
:10A05000119212930723139308A8FAF7C1FA98B93B
:10A060000F23039302230493002305934FF4A0537B
:10A0700006934FF480530793052103A8FAF7FEFCDB
:10A0800020B915B05DF804FBFFF7B0FFFFF7AEFF96
:10A09000003802400070004000B583B0F7F77EF84A
:10A0A000FFF7A6FFFFF7ACFDFFF702FDFFF72CFB64
:10A0B000FFF79CFBFFF7BCFB00F09CF800F052FDA3
:10A0C00000F0A8FD00F0EAFE00F02EF800F054F8D1
:10A0D00000F0B8FC00F08EFE00F0C6FE00F0FEFEC0
:10A0E00000F002FEFFF760FEFFF77CFE00F0A6F82E
:10A0F000FFF760FCFFF786FC01F01AFE064B0093A9
:10A10000064B074A07490020FFF7EEFAFFF760FD0C
:10A11000FEF706F9FEE700BF783D0108383D01086B
:10A120003C3D0108443D010808B50548054B036066
:10A13000FAF742FE00B908BDFFF758FFFBE700BF82
:10A14000EC670020000806500268094B9A4200D0D4
:10A15000704782B000230193064B5A6B42F04002D5
:10A160005A635B6B03F040030193019B02B070479D
:10A17000000806500038024008B50A480A4B036040
:10A18000002343607C22826040F67F42C26003610C
:10A1900043618361FAF778FE00B908BDFFF726FF37
:10A1A000FBE700BFFC6700200028004000B585B039
:10A1B0000023009301930293039302680A4B9A428F
:10A1C00002D005B05DF804FB02230093074B039314
:10A1D0006846FAF747FD20B9054B0122C3F83C2E2B
:10A1E000EFE7FFF703FFF7E70028004000031E003A
:10A1F0000000474208B50F480F4B03604FF48273CD
:10A20000436000238360C360022202610122426135
:10A210004FF4007282611022C26103624362836262
:10A220000A23C362FAF714FF00B908BDFFF7DEFE88
:10A23000FBE700BF9C6900200030014008B50F48D3
:10A240000F4B03604FF48273436000238360C3604D
:10A2500002220261012242614FF4007282613822BF
:10A26000C2610362436283620A23C362FAF7F0FEAB
:10A2700000B908BDFFF7BAFEFBE700BFF469002094
:10A28000003800402DE9F0438BB0044600230593CD
:10A2900006930793089309930368774A934206D07D
:10A2A000764A934200F082800BB0BDE8F08300252F
:10A2B0000095734B5A6C42F480525A645A6C02F403
:10A2C00080520092009A01951A6B42F002021A63C2
:10A2D0001A6B02F002020192019A02951A6B42F087
:10A2E00001021A631B6B03F001030293029B182304
:10A2F00005934FF00209CDF818904FF00108CDF802
:10A300001C80032608960527099705A95D48F8F7DC
:10A3100043F980230593CDF81890CDF81C8008965A
:10A32000099705A95848F8F737F95848584B03607A
:10A330004FF0C06343608560C5604FF48063036184
:10A3400045618561C5610562042343628662C56219
:10A350000563F7F71BFE18BB4C4BE3649C634D4849
:10A360004D4B03604FF0C063436040238360002384
:10A37000C3604FF48062026143618361C361036221
:10A380004362F7F703FE70B9424BA3649C6300225B
:10A3900005212320F7F7E8FC2320F7F71DFD83E7CD
:10A3A000FFF724FED8E7FFF721FEEDE70025039530
:10A3B000334B1A6C42F480421A641A6C02F48042E5
:10A3C0000392039A04951A6B42F002021A631B6B04
:10A3D00003F002030493049B4FF4604305930223AC
:10A3E0000693032608960523099305A92548F8F73F
:10A3F000D3F82A482A4B036045608560C5604FF456
:10A400008063036145618561C56105620423436220
:10A410008662C5620563F7F7B9FD30BB1F4BE36485
:10A420009C632048204B03600023436040228260ED
:10A43000C3604FF48062026143618361C361036260
:10A440000422426203228262C3620363F7F79EFD25
:10A4500070B9144BA3649C63002205212420F7F7F4
:10A4600083FC2420F7F7B8FC1EE7FFF7BFFDD5E714
:10A47000FFF7BCFDEDE700BF0030014000380040B1
:10A480000038024000040240000002401C68002026
:10A49000106402407C68002058640240DC680020A0
:10A4A000586002403C6900207060024010B582B0E4
:10A4B00000240094114B5A6C42F480425A645A6C46
:10A4C00002F480420092009A01941A6C42F0805289
:10A4D0001A641B6C03F080530193019B22460F21E9
:10A4E0006FF00100F7F740FC224606210420F7F741
:10A4F0003BFC0420F7F770FC02B010BD00380240AE
:10A5000030B589B0044600230193214B1A6C42F404
:10A5100080721A641B6C03F480730193019B02A97F
:10A5200003A8FAF781FB069BCBB9FAF75DFB03465C
:10A530001848A0FB03239B0C013B1748174A0260F5
:10A5400040F2E732C26043600023036183608361AD
:10A55000FBF7C2F9054630B1284609B030BDFAF71D
:10A5600043FB4300E4E70C48FBF74CF805460028A2
:10A57000F2D12D20F7F730FC0F2C01D90125EBE7A4
:10A58000002221462D20F7F7EFFB054B1C60E3E787
:10A590000038024083DE1B434C6A0020002000404C
:10A5A00004000020FEE7FEE7FEE7FEE7FEE7704757
:10A5B00008B5F7F71DFF08BD08B50820F8F7E4F85F
:10A5C00008BD08B51020F8F7DFF808BD08B5024847
:10A5D000F7F7D4FD08BD00BFC06C002008B50248E5
:10A5E000F7F7CCFD08BD00BF8466002008B502481F
:10A5F000F7F7C4FD08BD00BFDC68002008B50248BD
:10A60000F7F7BCFD08BD00BF3C69002008B5024853
:10A61000F7F772FA08BD00BFB063002008B5024822
:10A62000F7F76AFA08BD00BFB063002008B5202024
:10A63000F8F7AAF808BD000008B50248F9F734F8A1
:10A6400008BD00BF4467002008B50248F9F7FCF8D0
:10A6500008BD00BF4467002008B50248FAF774FE41
:10A6600008BD00BF9C69002008B50248FAF76CFEDF
:10A6700008BD00BFF469002008B50248FBF794FD4F
:10A6800008BD00BFE06D002008B50248FBF78CFD57
:10A6900008BD00BF246E002008B50348FAF7FAFF92
:10A6A0000248FAF7F7FF08BDB86B00204C6A00209B
:10A6B00008B50248F7F762FD08BD00BFE466002058
:10A6C00008B50248F7F75AFD08BD00BF1C68002016
:10A6D00008B50248F7F752FD08BD00BF206D002005
:10A6E00008B50248F7F74AFD08BD00BF7C680020A6
:10A6F00008B50248F7F742FD08BD00BF4C630020D3
:10A7000008B50248F7F7F8F908BD00BFD863002084
:10A7100008B50248F7F7F0F908BD00BFD86300207C
:10A7200008B50248F9F74EFC08BD00BF9081002033
:10A7300008B50248F7F722FD08BD00BF006C0020F5
:10A7400008B50248F7F71AFD08BD00BF806D00206C
:10A7500008B50248F7F712FD08BD00BF606C002085
:10A7600008B50248FBF720FD08BD00BF686E002059
:10A7700008B50248F8F798FF08BD00BF98670020A9
:10A7800008B50248F9F760F808BD00BF98670020D7
:10A7900010B503460C4A0D490D48006840B10C48FD
:10A7A00000680344521A934206D8094A136010BD48
:10A7B0000748084C0460F2E708F010FC0C23036023
:10A7C0004FF0FF30F3E700BF000002200050000010
:10A7D000946A0020F0980020034AD2F8883043F4AD
:10A7E0007003C2F88830704700ED00E000B587B014
:10A7F00003682C4A934218D02B4A934224D02B4A08
:10A8000093422ED02A4A934238D02A4A934218D1F2
:10A8100000230593284B5A6C42F400325A645B6C57
:10A8200003F400330593059B0BE000230193224BB7
:10A830005A6C42F001025A645B6C03F0010301930D
:10A84000019B07B05DF804FB002302931A4B1A6CBE
:10A8500042F004021A641B6C03F004030293029B8F
:10A86000EFE700230393144B1A6C42F008021A64BA
:10A870001B6C03F008030393039BE2E7002204929E
:10A880000D4B596C41F0020159645B6C03F00203FB
:10A890000493049B0F212D20F7F766FA2D20F7F77C
:10A8A0009BFACEE70000014000080040000C004089
:10A8B00000040140004401400038024070B58CB0F3
:10A8C00000230793089309930A930B930368514A53
:10A8D00093420DD0504A934222D0504A93423AD0EC
:10A8E0004F4A934251D04F4A934279D00CB070BD39
:10A8F000002301934C4B1A6B42F010021A631B6B3E
:10A9000003F010030193019B4FF4D44307930223F8
:10A91000089301230B9307A94448F7F73DFEE5E7A9
:10A9200000230293404B1A6B42F008021A631B6B20
:10A9300003F008030293029B4FF480430793022322
:10A9400008930122099203220A920B9307A938481F
:10A95000F7F722FECAE700230393334B1A6B42F04A
:10A9600080021A631B6B03F080030393039B4FF475
:10A97000E053079302230893012209920A930B9351
:10A9800007A92C48F7F708FEB0E700240494264BEB
:10A990001A6B42F480721A631A6B02F4807204928A
:10A9A000049A05941A6B42F004021A631B6B03F0BD
:10A9B00004030593059BC0230793022608960325ED
:10A9C0000B9507A91C48F7F7E7FD40230793089666
:10A9D00009940A940B9507A91848F7F7DDFD85E758
:10A9E00000230693104B1A6B42F020021A631B6B74
:10A9F00003F020030693069B40230793022308934A
:10AA0000012209920A9303230B9307A90C48F7F735
:10AA1000C3FD6BE70000014000080040000C00404F
:10AA20000004014000440140003802400010024090
:10AA3000000C0240001C02400020024000080240BE
:10AA40000014024010B596B000241294139414948C
:10AA500015941094119409940A940B940C940D94E9
:10AA60000E940F942022214601A808F0AFFD3B4828
:10AA70003B4B0360A7234360846044F61F63C360BD
:10AA8000046144618461FAF727FF00284BD14FF439
:10AA90008053129312A93148FBF729F8002845D1B9
:10AAA0002E48FAF745FF002843D100231093119355
:10AAB00010A92A48FBF72CF900283DD160230993FF
:10AAC00000220A920B920C920D920E920F9209A9FB
:10AAD0002248FAF791FF002831D1042209A91F4822
:10AAE000FAF78AFF70BB082209A91C48FAF784FF0D
:10AAF00058BB0C2209A91948FAF77EFF40BB002376
:10AB0000019302930393049305934FF4005206922A
:10AB1000089301A91148FBF741F9E0B90F48FFF785
:10AB2000CDFE16B010BDFFF761FAB0E7FFF75EFA91
:10AB3000B6E7FFF75BFAB8E7FFF758FABEE7FFF7AB
:10AB400055FACAE7FFF752FACDE7FFF74FFAD0E719
:10AB5000FFF74CFAD3E7FFF749FADFE7986A0020DE
:10AB60000000014000B58FB000230A930B930C93B3
:10AB70000D93089309930193029303930493059310
:10AB8000069307932148224A0260A722426083600D
:10AB90004FF6FF72C26003618361FAF79DFE28BB26
:10ABA0004FF480530A930AA91848FAF7A0FF00BB94
:10ABB0001648FAF7BDFEF8B900230893099308A9CF
:10ABC0001248FBF7A5F8D0B9602301930023029344
:10ABD00003930593082201A90C48FAF70DFF88B9E1
:10ABE0000A48FFF76BFE0FB05DF804FBFFF7FEF9B4
:10ABF000D6E7FFF7FBF9DBE7FFF7F8F9DCE7FFF74C
:10AC0000F5F9E1E7FFF7F2F9EAE700BF286B00206A
:10AC10000008004000B58FB000230A930B930C93FB
:10AC20000D9308930993019302930393049305935F
:10AC3000069307932A482B4A0260436083604FF6CD
:10AC4000FF72C26003618361FAF746FE002831D1CA
:10AC50004FF480530A930AA92148FAF748FF60BBD2
:10AC60001F48FAF765FE58BB00230893099308A90B
:10AC70001B48FBF74DF830BB602301930022029282
:10AC80000392059201A91648FAF7B6FEF0B904221C
:10AC90000DEB02011248FAF7AFFED0B9082201A964
:10ACA0000F48FAF7A9FEB8B90D48FFF707FE0FB035
:10ACB0005DF804FBFFF79AF9CAE7FFF797F9CFE7CA
:10ACC000FFF794F9D0E7FFF791F9D5E7FFF78EF991
:10ACD000DDE7FFF78BF9E1E7FFF788F9E4E700BF6D
:10ACE000706B0020000C004010B596B00024129448
:10ACF0001394149415941094119409940A940B9439
:10AD00000C940D940E940F942022214601A808F073
:10AD10005DFC3648364B0360A7234360846044F6ED
:10AD20001F63C360046144618461FAF7D5FD0028A4
:10AD300044D14FF48053129312A92C48FAF7D7FE4E
:10AD400000283ED12948FAF7F3FD00283CD1002322
:10AD50001093119310A92548FAF7DAFF002836D18D
:10AD60006023099300220A920B920C920D920E928C
:10AD70000F9209A91D48FAF73FFE58BB042209A902
:10AD80001A48FAF739FE40BB082209A91748FAF712
:10AD900033FE28BB0023019302930393049305938E
:10ADA0004FF400520692089301A91048FAF7F6FFF3
:10ADB000C8B90E48FFF782FD16B010BDFFF716F9AF
:10ADC000B7E7FFF713F9BDE7FFF710F9BFE7FFF7A4
:10ADD0000DF9C5E7FFF70AF9D0E7FFF707F9D3E761
:10ADE000FFF704F9D6E7FFF701F9E2E7B86B0020B7
:10ADF0000004014000B589B000230193029303933E
:10AE000004930593069307931548164A0260A722F8
:10AE10004260836041F28732C26003618361FAF766
:10AE20005BFDA0B90E48FAF783FD98B96023019342
:10AE3000002202920392059201A90948FAF7DCFD6B
:10AE400058B90748FFF73AFD09B05DF804FBFFF772
:10AE5000CDF8E7E7FFF7CAF8E8E7FFF7C7F8F0E74C
:10AE6000E06A00200044014008B50A480A4B03602C
:10AE70004FF46123436000238360C36003610C22AD
:10AE800042618361C361FBF7ABF800B908BDFFF70E
:10AE9000ADF8FBE7E06D00200010014008B50C485C
:10AEA0000C4B03600C4B43604FF4805383600023D2
:10AEB000C3604FF4806202610C2242618361C3610E
:10AEC000FBF78EF800B908BDFFF790F8FBE700BF6D
:10AED000246E002000480040A086010008B50A4802
:10AEE0000A4B03604FF4E133436000238360C36087
:10AEF00003610C2242618361C361FBF771F800B901
:10AF000008BDFFF773F8FBE7686E002000140140EE
:10AF10002DE9F0418CB00446002307930893099370
:10AF20000A930B9303689D4A93420AD09C4A93422A
:10AF300000F082809B4A934200F0C3800CB0BDE8D1
:10AF4000F08100250095984B5A6C42F010025A642B
:10AF50005A6C02F010020092009A01951A6B42F0AE
:10AF600002021A631A6B02F002020192019A029520
:10AF70001A6B42F001021A631B6B03F00103029388
:10AF8000029B802307934FF00208CDF8208003270F
:10AF90000A9707260B9607A98448F7F7FDFA4FF49E
:10AFA00000730793CDF8208009950A970B9607A99F
:10AFB0007F48F7F7F1FA7F487F4B03604FF000635B
:10AFC000436040238360C5604FF480630361456143
:10AFD0008561C5614FF4403303624562F6F7D6FFE1
:10AFE00020BB744B63639C637448754B03604FF0E4
:10AFF0000063436000238360C3604FF4806202619A
:10B0000043618361C3614FF4403202624362F6F7E9
:10B01000BDFF70B9694BA3639C6300220521252005
:10B02000F6F7A2FE2520F6F7D7FE87E7FEF7DEFF4C
:10B03000D7E7FEF7DBFFEDE7002503955A4B1A6CC7
:10B0400042F480221A641A6C02F480220392039A5A
:10B0500004951A6B42F004021A631B6B03F004039D
:10B060000493049B4FF44063079302230893032344
:10B070000A9307230B9307A95248F7F78DFA524812
:10B08000524B03604FF0006343608560C5604FF42E
:10B090008063036145618561C56105624562F6F7BC
:10B0A00075FF58B9484BA3639C63002205212720F4
:10B0B000F6F75AFE2720F6F78FFE3FE7FEF796FFDA
:10B0C000F0E700250595384B5A6C42F020025A648F
:10B0D0005A6C02F020020592059A06951A6B42F00E
:10B0E00040021A631B6B03F040030693069B4FF468
:10B0F000844307930223089303260A9608230B939D
:10B1000007A93348F7F748FA3248334B03604FF04A
:10B11000206343608560C5604FF4806303614561CF
:10B120008561C5614FF40033036204234362866284
:10B13000C5620563F6F72AFF50BB264BA3639C63E9
:10B140002648274B03604FF0206343604023836011
:10B150000023C3604FF48062026143618361C36175
:10B160004FF4003202620422426203228262C3620E
:10B170000363F6F70BFF70B9184B63639C630022FF
:10B1800005214720F6F7F0FD4720F6F725FED5E626
:10B19000FEF72CFFD1E7FEF729FFEDE70010014095
:10B1A0000048004000140140003802400004024002
:10B1B00000000240606C0020B8640240006C002077
:10B1C0008864024000080240C06C002028600240F1
:10B1D00000180240206D002040640240806D002075
:10B1E000A064024008B500220F491048FCF7B7FAE6
:10B1F00070B90F490D48FCF7C9FA60B90D490B4801
:10B20000FCF76CFA50B90948FCF7DAFA48B908BDFE
:10B21000FEF7ECFEEDE7FEF7E9FEEFE7FEF7E6FEF0
:10B22000F1E7FEF7E3FEF2E7AC000020AC6E002091
:10B230000800002098000020002070470020704780
:10B2400008B5034B1B680BB108889847002008BD60
:10B250008C81002038B50C46074D01462846FCF786
:10B2600056FA2846FCF75FFA044B1B680BB120889E
:10B270009847002038BD00BFAC6E002088810020B8
:10B2800010B5064C002206492046FCF732FA054963
:10B290002046FCF73CFA002010BD00BFAC6E002039
:10B2A0008879002088710020024B1860024B1960D9
:10B2B000024870478C81002088810020887100201E
:10B2C00030B589B000230393049305930693079345
:10B2D0000368B3F1A04F01D009B030BD002501953E
:10B2E000164C236B43F001032363236B03F001032C
:10B2F0000193019B4FF4E053039302230493032330
:10B3000006930A23079303A90D48F7F745F9636BE2
:10B3100043F0800363630295636C43F4804363648A
:10B32000636C03F480430293029B2A460521432069
:10B33000F6F71AFD4320F6F74FFDCDE7003802403F
:10B340000000024008B500F2C441D0F80805FCF73F
:10B350004DFA08BD08B501EBC10300EB8303D3F838
:10B360008C22D0F80805FCF70EFB08BD08B501EBF0
:10B37000C10300EB8303DA6CD0F80805FCF766FB29
:10B3800008BD08B5D0F80805FCF7A8FA08BD10B547
:10B390000446C3683BB1022B01D1012104E0FEF752
:10B3A00025FE012100E00021D4F80805FCF77CFA15
:10B3B000D4F80805FCF746FA10BD000010B50446A5
:10B3C000D0F80805FCF773FA2268D2F8003E43F083
:10B3D0000103C2F8003E236A23B1034A136943F014
:10B3E0000603136110BD00BF00ED00E008B5D0F802
:10B3F0000805FCF766FA08BD08B5D0F80805FCF7A3
:10B4000095FA08BD08B5D0F80805FCF778FA08BD2C
:10B4100008B5D0F80805FCF7A0FA08BD08B5D0F8C3
:10B420000805FCF79CFA08BD02780AB100207047B5
:10B4300010B503461548C0F80835C3F8C8024FF0E8
:10B44000A0430360042343600222C260002303611F
:10B450008261C36103624362C3620363F8F7BEFAA9
:10B4600080B90A4C80212046F9F7B4F84022002127
:10B470002046F9F789F8802201212046F9F784F85F
:10B48000002010BDFEF7B2FDEBE700BF9081002069
:10B49000D0F8C83211F0800F08D101F07F0101EB24
:10B4A000C10103EB810191F87E02704701F07F0139
:10B4B00001EBC10103EB810191F83E00704708B533
:10B4C000D0F8C802F8F7ADFC08BD0000004870478E
:10B4D0009C8600207047032805D8DFE800F00504AB
:10B4E0000205012070470320704708B5D0F8C80254
:10B4F000F8F70BFBFFF7EFFF08BD08B594461A46B7
:10B500006346D0F8C802F8F7DFFBFFF7E4FF08BD99
:10B5100008B5D0F8C802F8F71CFCFFF7DCFF08BD3F
:10B5200008B5D0F8C802F8F7B4FCFFF7D4FF08BD9F
:10B5300008B5D0F8C802F8F7F0FCFFF7CCFF08BD5B
:10B5400008B5D0F8C802F8F7ABFBFFF7C4FF08BD99
:10B5500008B5D0F8C802F8F76DFCFFF7BCFF08BDCE
:10B5600008B5D0F8C802F8F72DFCFFF7B4FF08BD06
:10B5700012230B8000487047C800002004230B8072
:10B5800000487047DC000020002393421ED200B523
:10B5900010E00CF1370C01F813C000014FEA430C26
:10B5A0000CF1010C4FF0000E01F80CE00133DBB29E
:10B5B000934209D24FEA107CB0F1204FE9D20CF14E
:10B5C000300C01F813C0E8E75DF804FB7047000099
:10B5D00038B50B4BD3F8100AD3F8144AD3F8183AFD
:10B5E000C01800D138BD074D0822A91CFFF7CCFFB9
:10B5F000042205F112012046FFF7C6FFF2E700BF63
:10B600000070FF1FE000002008B51A230B80FFF731
:10B61000DFFF014808BD00BFE000002008B50A4672
:10B6200028B905490548FCF716FE034808BD02493C
:10B630000248FCF710FEF8E7BC880020983D01089E
:10B6400010B50A46034C21460348FCF704FE204689
:10B6500010BD00BFBC880020AC3D010808B50A46FB
:10B6600028B905490548FCF7F6FD034808BD02491D
:10B670000248FCF7F0FDF8E7BC880020BC3D01085B
:10B6800008B50A4628B905490548FCF7E4FD034812
:10B6900008BD02490248FCF7DEFDF8E7BC8800203F
:10B6A000C83D0108DFF834D00D480E490E4A00238A
:10B6B00002E0D458C4500433C4188C42F9D30B4A66
:10B6C0000B4C002301E013600432A242FBD3FFF7CE
:10B6D00083F807F089FCFEF7DFFC704700000220CA
:10B6E00000000020940E0020C8550108980E00208C
:10B6F000EC980020FEE700001A4BD3ED0A7A1A4BB3
:10B70000C3ED007A9FED197AF4EEC77AF1EE10FAE4
:10B7100005DD77EEC77A164BC3ED037A70479FEDD0
:10B72000137AF4EEC77AF1EE10FA0ED89FED117A83
:10B73000F4EEC77AF1EE10FA07DB9FED0C7A77EEA4
:10B74000C77A0B4BC3ED037A70479FED087A77EE0B
:10B75000C77A9FED097A77EE877A054BC3ED037AB6
:10B76000704700BF048B0020BC8A00202C70B442BC
:10B77000C48A0020D48FB3C20000B443000000008C
:10B78000F8B54B4B1C68E37A012B03D0E37A032B0B
:10B790005FD0F8BD474B01221A70A37A934226D09E
:10B7A000032B50D0022BF1D1B4F9020007EE900A1E
:10B7B000F8EEE77A17EE900AF4F776FE3AA3D3E9AB
:10B7C0000023F4F7C9FE06460F463A4DD5F80100AE
:10B7D000F4F76AFE32463B46F4F708FDF5F7F6F853
:10B7E000C5F801000223AB720523EB72CEE7B4F972
:10B7F000023007EE103AB8EEC77ADFED2F6A27EE77
:10B80000267A2C4BD3F8012007EE902A37EE277AC0
:10B8100017EE102AC3F80120B4F9062007EE902A8B
:10B82000F8EEE77A67EEA67AD3F8052007EE102A3D
:10B8300077EE877A17EE902AC3F805200522DA7290
:10B8400003229A72A2E71B4B0422DA7203229A7235
:10B850009CE7B4F9023007EE903AF8EEE77A9FEDF4
:10B86000177A67EE877A134BD3F8012007EE102A78
:10B8700077EE877A17EE902AC3F80120B4F90620F4
:10B8800007EE902AF8EEE77A9FED0B7A67EE877A5B
:10B89000D3F8052007EE102A77EE877A17EE902A64
:10B8A000C3F8052075E700BF9A9999999999B93F0E
:10B8B000348B0020408B0020CDCCCC3D0AD7233CDC
:10B8C00000B583B01A4B1B68B3F90830B3F5967F07
:10B8D00002DC184B1B787BB90020164B1870164BF6
:10B8E0001873164B1874164B1870164B0093164BA2
:10B8F000164A1749FDF7F8FE0D4B1B68B3F90830DF
:10B9000013F5FA7F02DB03B05DF804FB0123094A5B
:10B9100013700B4A13700F4B5A6A074B1A60094B8E
:10B9200000930D4B0D4A0E490020FDF7DDFEEAE7BE
:10B93000348B0020388B0020F08A0020C48A00203D
:10B94000408B0020783D0108D83D0108DC3D01080E
:10B95000E43D0108048B0020383D01083C3D01080E
:10B96000043E010808B51F4805F006FD1E4B18608F
:10B9700004F0E2F91D4B18601D4805F0DFFB1D4B7C
:10B9800018601D4805F036FA1C4B18600D211C4844
:10B9900004F04CFA1B4B18602C211B4804F076FA7B
:10B9A0001A4B18600C211A4804F040FA194B186021
:10B9B000C121194804F06AFA184B18601C21184874
:10B9C00004F034FA174B18600621174804F05EFAA9
:10B9D000164B1860164B00225A60164B01221A7043
:10B9E00008BD00BF246E0020348B0020148D002081
:10B9F000E06D0020188D0020686E0020308B002044
:10BA00002C3E0108EC8A0020383E0108008B002003
:10BA1000443E01083C8B0020503E01084C8B002026
:10BA20005C3E0108C08A0020683E0108E08A0020D0
:10BA3000F08A0020388B002008B51849184B186888
:10BA400004F045FA1749184B186804F040FA1749F2
:10BA5000174B186804F03BFAFFF74EFEFFF730FF74
:10BA6000144B1B7833B1144B1B689B7A013BDBB240
:10BA7000022B0FD91149124B186804F03FFA1149F3
:10BA8000114B186804F03AFA1049114B186804F089
:10BA900035FA08BDFFF774FEECE700BFE48A00202A
:10BAA000E08A0020508B00204C8B0020048B00206B
:10BAB000008B0020388B0020348B0020C48A0020AB
:10BAC000C08A0020408B00203C8B0020F08A0020A0
:10BAD000EC8A002000B583B003F07CFE174B009386
:10BAE000174B184A18490020FDF7FEFD0EE0134BD6
:10BAF0000193164B0093164B164A17490020FDF789
:10BB0000F3FD04F041F90120FCF744FC00F0EAFDEC
:10BB1000124C84ED000A03F0FFFF00F0E3FDD4EDCA
:10BB2000007A30EE670A094B83ED000AF7EE007ADF
:10BB3000B4EEE70AF1EE10FAD9DCE2E7783D01084D
:10BB4000383D01083C3D0108A43E01082C8D002031
:10BB5000D83D0108DC3D0108C83E0108308D0020B9
:10BB600000B583B0164B0093164B174A17490020B7
:10BB7000FDF7BAFD0CE0124B0193154B0093154BEA
:10BB8000154A16490020FDF7AFFD0120FCF702FC25
:10BB900000F0A8FD124C84ED000A04F07BFF00F0D9
:10BBA000A1FDD4ED007A30EE670A094B83ED000A5F
:10BBB000F7EE007AB4EEE70AF1EE10FADBDCE4E728
:10BBC000783D0108383D01083C3D0108003F01086F
:10BBD000388D0020D83D0108DC3D0108283F0108D0
:10BBE0003C8D002000B583B000F0EEFF174B0093B2
:10BBF000174B184A18490020FDF776FD0CE0134B4F
:10BC00000193164B0093164B164A17490020FDF777
:10BC10006BFD0A20FCF7BEFB00F064FD134C84EDC5
:10BC2000000A02F035FE00F0EDFF00F05BFDD4ED00
:10BC3000007A30EE670A094B83ED000AF2EE047ACF
:10BC4000B4EEE70AF1EE10FAD9DCE2E7783D01083C
:10BC5000383D01083C3D0108643F0108208D00206B
:10BC6000D83D0108DC3D01088C3F0108248D0020EF
:10BC700008B5A82000F04EFC00F0B2FD08BD0000A1
:10BC800010B59CB0254C0DF1540CA646BEE80F0033
:10BC9000ACE80F009EE807008CE80700002115A81B
:10BCA000FCF743FB1E4B18600DF1380C04F11C0E21
:10BCB000BEE80F00ACE80F009EE807008CE8070024
:10BCC00000210EA8FCF731FB164B18600DF11C0C7F
:10BCD00004F1380EBEE80F00ACE80F009EE8070044
:10BCE0008CE80700002107A8FCF71FFB0E4B18602B
:10BCF000EE4604F1540CBCE80F00AEE80F009CE8DF
:10BD000007008EE8070000216846FCF70EFB074B92
:10BD1000186004F0E3FD1CB010BD00BF283C010812
:10BD2000288D0020348D00201C8D0020408D0020A7
:10BD300008B572B6FFF79CFFFFF714FE00F04CF851
:10BD4000FFF79EFF62B608BD08B5FFF775FE00F06D
:10BD50007DF908BD00B583B0164B0093164B174A0A
:10BD600017490020FDF7C0FC0CE0124B0193154B66
:10BD70000093154B154A16490020FDF7B5FC01202C
:10BD8000FCF708FB00F0AEFC124C84ED000AFFF754
:10BD9000DBFF00F0A7FCD4ED007A30EE670A094B18
:10BDA00083ED000AF7EE007AB4EEE70AF1EE10FA3E
:10BDB000DBDCE4E7783D0108383D01083C3D010843
:10BDC000C83F0108448D0020D83D0108DC3D010832
:10BDD000F43F0108488D00202DE9F04F2DED068B32
:10BDE000ADF51D7D4FF0B80B5A4600216EA807F047
:10BDF000EDFB784B7D934FF07F537E939FED768ADA
:10BE00008DED7F8A9FED759A8DED809A07258DF8CF
:10BE10000852DFED738ACDED838A4FF08243889319
:10BE2000704B8A93704B8B938DF834526F4B8E937B
:10BE300004268DF84C624FF0060A8DF84DA20127BA
:10BE40008DF84E7202248DF85442DFF8FC81CDF853
:10BE5000588297976EA804F011FA654B1860979472
:10BE600000248DF84E426EA804F008FA614B186069
:10BE70005A46214640A807F0A9FBF0EE00AACDEDF6
:10BE80004FAA8DED508A8DED529A8DF85051CDED1F
:10BE9000558A594B5A93594B5B938DED5C8A9FEDB4
:10BEA00058AA8DED5DAA8DF87C51DFED569ACDED47
:10BEB000609A8DF894618DF895A18DF896714FF088
:10BEC00003098DF89C91CDF8A081CDF8A4915A4634
:10BED000214612A807F07AFBCDED21AA8DED228A2A
:10BEE0008DED249A8DF89850CDED278A464B2C93F2
:10BEF0008DED2FAA8DF8C450CDED329A8DF8DC600F
:10BF00008DF8DDA08DF8DE708DF8E490CDF8E88036
:10BF10003B968DF83C408DF83D403C4B109311947E
:10BF20000CAF3B4B93E8070087E807008DF82440EF
:10BF30008DF82540374A0A920B9406AE03F10C02A5
:10BF400007CA86E8070003AD03F1180207CA85E8AF
:10BF500007006C46243393E8070084E8070040A8F4
:10BF600004F08CF92C4B186012A804F087F92B4BC5
:10BF700018600FA804F098FD294B1860384604F0AB
:10BF800093FD284B186009A804F08EFD264B18601D
:10BF9000304604F089FD254B1860284604F084FDE6
:10BFA000234B1860204604F07FFD224B1860C1210E
:10BFB000214803F03BFF214B18600C21204803F07F
:10BFC00065FF204B18600DF51D7DBDEC068BBDE8AF
:10BFD000F08F00BF000040406F12833A00606A4655
:10BFE00000401C460AD7233D00C0DA450000C84285
:10BFF000548D0020588D00200000A0410000A0407A
:10C0000000409C470000FA4300008841B86B0020C4
:10C01000983C0108986A0020508D00204C8D00202B
:10C020005C8D0020608D0020708D00206C8D0020C4
:10C03000688D0020648D0020503E0108448F002050
:10C04000443E0108488F0020B0630020F8B54E4CF4
:10C0500021464E4B186803F03AFF23783BBB4C4B0C
:10C06000186804F003F94B4B186804F0FFF84A4BCA
:10C07000186804F0FBF8494B186804F0F7F8424BD5
:10C080005B7A002B3ED0012B42D03F4B9B7A022B98
:10C0900044D0032B48D03C4BDB7A042B4AD0052BF1
:10C0A0005DD03F493F4B186803F028FFF8BD384E7C
:10C0B000306804F0DFF8374F386804F0DBF8364DAD
:10C0C000286804F0D7F8304CD4F8013000EE103A6C
:10C0D000386804F03FF9D4F8013000EE103A3068C7
:10C0E00004F038F9D4F8053000EE103A286804F06E
:10C0F00031F9D4F8013000EE103A284B186804F0FA
:10C1000029F9BCE73E21284B186804F0EFFCBCE796
:10C110004E21254B186804F0E9FCB6E72D21234B8E
:10C12000186804F0E3FCB6E75A21204B186804F0C5
:10C13000DDFCB0E7B4211E4B186804F0D7FCB42135
:10C140001C4B186804F0D2FC00211B4B186804F04B
:10C15000CDFC0021194B186804F0C8FCA1E72D2183
:10C16000134B186804F0C2FC2E21124B186804F01F
:10C17000BDFC8721104B186804F0B8FC87210F4BD9
:10C18000186804F0B3FC8CE7748D0020488F002001
:10C19000548D0020588D0020508D00204C8D0020A3
:10C1A000808D0020448F00205C8D0020608D002059
:10C1B000708D00206C8D0020688D0020648D002023
:10C1C00010B50C4C2046F5F7FDFA02212046F5F794
:10C1D00076FC10212046F5F772FC074C2046F5F757
:10C1E000F1FA02212046F5F76AFC10212046F5F706
:10C1F00066FC10BDB0630020D863002000B58BB092
:10C200000123069300230793C36913F0010F0CBFAA
:10C210000123002304930E230993436B5B010193D5
:10C2200002680B4B9A420DD00A4A1378591C1170C0
:10C2300005930123089369460068F5F727FA0BB0C8
:10C240005DF804FB044A1378591C1170F0E700BF35
:10C25000B0630020FA000020508F002070B582B03B
:10C2600005460E4631462846F5F716FC48B36B46A0
:10C27000154A31462846F5F76AFB002400E00134F0
:10C28000124B1B78A342EDD9114B53F824301A6896
:10C29000AA42F4D10C4A11685A6B9142EFD1D3F8FB
:10C2A000392072B1084A126983F83820084D1846BF
:10C2B00069462C30F4F75CFD55F82400D0F839308D
:10C2C000984702B070BD00BF988F0020948F002067
:10C2D000548F002030B585B00446314B1B7873B1C4
:10C2E0002F4B93F800C0BCF10F0F2FD92D4B0093AB
:10C2F0002D4B2E4A2E490020FDF7F6F9F6E7FFF701
:10C300005FFF284B00932B4B2B4A2C490020FDF755
:10C31000EBF9E5E701339C451AD9294A52F8232065
:10C32000506BA1688842F5D1116822689142F1D121
:10C330001C4B029304F108030193231D00931A4B35
:10C340001A4A20490020FDF7CFF9F1E70023E2E780
:10C35000412006F083FE05464122002107F036F910
:10C3600062686A600023082129756B75AB75EB75EF
:10C3700023682B60EA61A3686B63E368C5F8393012
:10C380002369C5F83D302846FFF738FF044A137883
:10C39000591C11700A4A42F82350284605B030BD96
:10C3A000948F0020783D0108D83D0108DC3D01084C
:10C3B0005C400108383D01083C3D0108344001085B
:10C3C000548F0020B440010810B52DED028B82B0CF
:10C3D0000446F0EE408A00F085F9B0EE408A20680D
:10C3E000F5F79CFAD8B900F07DF930EE480AB4EEC2
:10C3F000E80AF1EE10FAF2DD1A4B01931A4C2368A9
:10C4000000931A4B1A4A1B490020FDF76DF9236867
:10C4100001332360002002B0BDEC028B10BD00F0A0
:10C4200061F930EE488A144B83ED008A214651F8B9
:10C43000040B04F1200304F12402F5F7F1F908B923
:10C440000120E8E7074B0193074C23680093074B53
:10C45000074A0A490020FDF747F9236801332360A2
:10C460000020D8E7783D01084C8F002000410108EA
:10C47000044101080C410108B48F00205C4101080F
:10C480004B1EDBB2072B0AD900B583B0054B0093D6
:10C49000054B064A06490020FDF726F9F6E74161FB
:10C4A000704700BF783D0108D83D0108DC3D010818
:10C4B0008441010808B50021FFF7D0FE08BD08B58A
:10C4C0000121FFF7CBFE08BD0E4B1B78C3B982B02C
:10C4D0000C4B01221A700C4B5B680193019A0B4BB9
:10C4E0001B689A4203D20A4A136801331360064B51
:10C4F0005A68064B1A60034B00221A7002B070474C
:10C50000704700BFF88F0020001000E0E88F002087
:10C51000EC8F002008B5124AD2F8FC3043F080734B
:10C52000C2F8FC300F4B002159601A6842F001023A
:10C530001A600D4B03FB00F00C4B18600C4BA3FB77
:10C5400000239B090B4A13600B4BA3FB0030800CAC
:10C550000A4B18600A4B1960FFF7B6FF08BD00BF11
:10C5600000ED00E0001000E040420F00D08F0020FE
:10C57000D34D6210D48F002083DE1B43D88F002060
:10C58000EC8F002000B52DED028B83B00D4B5B6866
:10C590000193019B02689B1A07EE903AF8EE677AC6
:10C5A000094B93ED007AB8EE477A87EE878A019BB4
:10C5B0000360FFF789FFB0EE480A03B0BDEC028BC1
:10C5C0005DF804FB001000E0D08F00202DE9F04161
:10C5D00082B0274B5B680193FFF776FF254B1C6801
:10C5E00000266508E3071B1B65F10005DB186D419C
:10C5F0001C1945F10005019BE41845F100071E4B8D
:10C600001C605F601D4B1D682A4633462046394634
:10C61000F4F72CFA1A4A10605160A5FB003205FBB2
:10C620000125E41A67EB0505164B1C605D60DFF819
:10C630006480C8F80000144B1F683A463346204611
:10C640002946F4F713FA80B2A8F8040007FB00F0BB
:10C65000201A65F100010D4B186059600C4B1A68E7
:10C660003346F4F703FAA8F8060002B0BDE8F081FB
:10C67000001000E0EC8F0020E08F0020D08F002021
:10C68000B88F0020C08F0020D48F0020C88F0020DA
:10C69000D88F0020F08F002008B5FFF797FF0E4BD2
:10C6A0009A8800EE102AB8EEC00ADFED0C7A60EE30
:10C6B000277A93ED007AB8EE470A30EE270ADB8836
:10C6C00007EE903AF8EEE77A9FED057A67EE877A03
:10C6D00030EE270A08BD00BFF08F00206F12833AAA
:10C6E000BD37863508B5FFF771FF0B4A116893888F
:10C6F0004FF47A7000FB013300EE103AB8EE400AB6
:10C70000D38807EE903AF8EEE77A9FED047A67EE69
:10C71000877A30EE270A08BDF08F00206F12833A27
:10C720000A4B5A68094B5B689B1A07EE903AB8EEC1
:10C73000677A074BD3ED007AF8EE677A67EE807A76
:10C74000B4EEE77AF1EE10FAECD47047001000E096
:10C75000D08F002008B50146002300E00133074ACE
:10C7600012789A4209D9064A52F82300C2888A42AE
:10C77000F4D18268002AF1D0904708BD24900020AF
:10C78000FC8F00200146002305E0036903B19847B0
:10C7900010BD0133DBB20E4A12789A4217D90D4A06
:10C7A00052F8230002688A42F3D110B54C6C02792A
:10C7B0009442EAD00133DBB2054A12789A42E7D9B3
:10C7C000044A52F8230002688A42F3D1EEE7704728
:10C7D000259000202890002008B5FFF7D3FF08BD62
:10C7E00008B5FCF77FFD08BD08B5036803F14042BA
:10C7F000B2F5005F0FD903F13F4202F57F02B2F5B7
:10C80000806F17D9A3F14023A3F58033B3F5006FF0
:10C8100010D9002008BDF8F7E7F90E4B9B68C3F369
:10C8200082230D4AD35C1BB9012303FB00F0F1E71F
:10C830000223FAE7F8F7E8F9064B9B68C3F3822373
:10C84000054AD35C1BB9012303FB00F0E2E7022396
:10C85000FAE700BF00380240903D010808B50146E4
:10C86000002301E00133DBB20B4A12789A4212D95D
:10C870000A4A52F8230002688A42F3D191F81CE078
:10C8800042684FEA920C012202FA0CF29645E9D175
:10C89000436903B1984708BD3090002034900020D0
:10C8A000836801684A680132B3FBF2F307EE903AFD
:10C8B000F8EE677A67EE807A0B68FCEEE77AC3EDF4
:10C8C0000B7A836801684A680132B3FBF2F307EE22
:10C8D000903AF8EE677A27EE800ABCEEC00A81ED46
:10C8E000030A7047436863B903681B68D3ED0B7A8A
:10C8F000F8EE677A27EE800ABCEEC00A83ED0D0AD7
:10C900007047042B0ED0082B19D003681B68D3ED99
:10C910000B7AF8EE677A27EE800ABCEEC00A83ED48
:10C92000100A704703681B68D3ED0B7AF8EE677A3C
:10C9300027EE800ABCEEC00A83ED0E0A704703683A
:10C940001B68D3ED0B7AF8EE677A27EE800ABCEE0F
:10C95000C00A83ED0F0A704738B51C4B1B780F2BAC
:10C9600000D9FEE705461C2006F078FB04460023AC
:10C97000036043608360C36003614361836128682F
:10C9800020606B686360AB68E360EB6823612B69D0
:10C9900063616B69A361FFF727FFA060616820688E
:10C9A000F9F734F994ED030A2046FFF779FF94ED87
:10C9B000040A2046FFF796FF044A1378591C1170A9
:10C9C000034A42F82340204638BD00BF3090002083
:10C9D0003490002010B5044690F800210146D0F8AC
:10C9E0000401F9F7CDFDD4F804319B6B1A68136884
:10C9F00023F00803136010BD70B582B0214B1D7881
:10CA0000022D1DD9204B0093204B214A21490020A3
:10CA1000FCF76AFEF6E70133DBB29D4213D91E4AEA
:10CA200052F82320D2F8041162689142F3D1164BD8
:10CA30000093164B164A19490020FCF755FEF6E7FD
:10CA400004460023E9E74FF4867006F007FB06462C
:10CA50004FF48672002106F0B9FD6368C6F8043110
:10CA6000237886F80031A368C6F808316A1C054BA4
:10CA70001A70094B43F825603046FFF7ABFF30468C
:10CA800002B070BD74900020783D0108D83D0108C7
:10CA9000DC3D0108C84101087890002000420108EF
:10CAA00038B50C46002301E00133DBB2154A92F899
:10CAB00000C09C4525D91D46134A52F82320D2F8C0
:10CAC00004118142F0D1D2F808313BB19847224697
:10CAD00000210D4B53F8250006F078FD0A4C54F860
:10CAE000251091F80021D1F80401F9F749FD54F817
:10CAF0002530D3F804319B6B1A68136823F00803C0
:10CB0000136038BD74900020789000208446002384
:10CB1000174A12789A422AD910B582B01C46154A93
:10CB200052F82310D1F80401604506D00133DBB27E
:10CB30000F4A12789A42F1D817E091F80021F9F7DC
:10CB40001FFD0C4B53F82430D3F804319B6B1A684B
:10CB5000136823F008031360074B01930094074BFD
:10CB6000074A08490020FCF7BFFD02B010BD70471E
:10CB70007490002078900020783D01080041010861
:10CB8000044101083C42010810B584B004AB03E93C
:10CB90000300FEF789FB064C2060064B0093064B12
:10CBA000064A07490020FCF79FFD206804B010BD2D
:10CBB00084900020783D0108383D01083C3D010883
:10CBC000844201087047000000B587B0002300933D
:10CBD00001930293039304930593074B0093082357
:10CBE0000193064B02936846FFF7B6FE044B1860AC
:10CBF00007B05DF804FB00BF286B00206F12833A7A
:10CC00008890002038B5002440E095ED000A284BBC
:10CC10001868FFF767FE2B79062B0BD8DFE803F0C7
:10CC2000040B121920272E009FED220A204B1868B2
:10CC3000FFF736FE38BD9FED200A1D4B1868FFF741
:10CC40002FFEF7E79FED1D0A194B1868FFF728FE26
:10CC5000F0E79FED1B0A164B1868FFF721FEE9E786
:10CC60009FED180A124B1868FFF71AFEE2E79FEDD6
:10CC7000160A0F4B1868FFF713FEDBE79FED130A48
:10CC80000B4B1868FFF70CFED4E70134042CD1D805
:10CC90000F4B53F824506B79042BF6D8AB79002B4B
:10CCA000B3D19FED0C0A024B1868FFF71BFEECE7AF
:10CCB000889000209D9DFA3A934ADF3A32E5C63AC1
:10CCC00041C8BB3A052FA73A09F2943AFAA9843A27
:10CCD0008C90002000000000F6EE007A60EE277ACB
:10CCE00010EE103A074AA2EB630307EE103A67EE24
:10CCF000277A67EE277AB7EE080A30EE670A27EE42
:10CD0000000A7047865A375F10B52DED048B044634
:10CD1000D0F8EC3093ED009A5C4A82ED009A93EDE6
:10CD2000018A5B4A82ED008AD3ED028A594AC2ED3C
:10CD3000008AD3ED039A584BC3ED009A69EE097A45
:10CD400028EE080A77EE807A28EEA80A77EE807A35
:10CD500029EEA90A37EE800AFFF7BEFF4F4B83ED9D
:10CD6000000A00230BE0D4F8EC2002EB8302D2EDA2
:10CD7000007A67EE807AC2ED007A0133DBB2032BD2
:10CD8000F1D9474B93ED6F7A28EE077AD4F800215A
:10CD9000F6EE007A27EE277A82ED047A93ED6F7A29
:10CDA00028EE877AD4F8002127EE277A82ED057ADB
:10CDB00093ED6F7A29EE477AD4F8002127EE277A8F
:10CDC00082ED0A7A93ED6F7A29EE877AD4F8002102
:10CDD00027EE277A82ED0B7A93ED6F7A69EEC79A88
:10CDE000D4F8002169EEA79AC2ED109A93ED6F7AFC
:10CDF00029EE479AD4F8002129EE279A82ED119A5C
:10CE000093ED6F7A68EE878AD4F8002168EEA78ADE
:10CE1000C2ED168A93ED6F7A28EE478AD4F8002186
:10CE200028EE278A82ED178AD4F8F82093ED747AD9
:10CE3000D2ED1C6AC6EE877AC2ED1C7AD4F8F820CF
:10CE400093ED747AD2ED236AC6EE877AC2ED237A27
:10CE5000D4F8F83093ED1C7ADFED127AB4EEE77A6D
:10CE6000F1EE10FA01DDC3ED1C7AD4F8F83093ED41
:10CE7000237ADFED0C7AB4EEE77AF1EE10FA01DDF9
:10CE8000C3ED237ABDEC048B10BD00BF34930020AA
:10CE90003C930020449300204C93002050930020AA
:10CEA0003091002000401C4638B504469022D0F84E
:10CEB000F8100848F3F75CFF48252A46D4F81C11FF
:10CEC0000548F3F755FF2A46D4F80C110348F3F749
:10CED0004FFF38BDFC000020E8900020A09000200B
:10CEE0002DE9F84F044600F1780500F18007394636
:10CEF000284604F06FFA84F8C800B4F87830A4F833
:10CF0000A830B4F85A30A4F8AA3004F1580A04F151
:10CF1000A80842465146284604F022FB84F8C8007F
:10CF2000B4F8A830A4F8B030B4F88230A4F8B23025
:10CF300004F1B0094A463946404604F011FB84F832
:10CF4000C800B4F89030A4F8A030B4F89230A4F837
:10CF5000A23004F1A0052A4604F19001484604F0ED
:10CF6000A9FC84F8C8004946284604F099FB84F8D7
:10CF7000C800D4F8EC30D3ED007AC44AC2ED007A90
:10CF800093ED016AC24A82ED006AD3ED026AC14A9A
:10CF9000C2ED006A93ED037ABF4B83ED007AB4F8DB
:10CFA0007830A4F8B8300123A4F8BA3066EE075AF6
:10CFB00027EEA65A75EEC55AD4F82C3175EEA55A4F
:10CFC000C3ED005A67EE865A26EE875A75EE855AEB
:10CFD000D4F82C3175EEA55AC3ED015A67EEA77A45
:10CFE00026EE066A77EEC67A66EEA66A77EEE67AEF
:10CFF00027EE077AD4F82C3177EE877AC3ED027AE0
:10D00000002512E0D4F82C3103EB850393ED000AE0
:10D01000B0EEC00A04F0BAFD05F160029F4B03EBCD
:10D02000820383ED010A0135EDB2022DEAD9B4F88D
:10D030004830A4F8C0304FF0010BA4F8C2B004F19E
:10D04000B80504F1C0063246294604F1480004F050
:10D050001DFA84F8C800B4F8C030A4F8A830A4F8C9
:10D06000AAB042463146484604F07AFA84F8C8002D
:10D07000A4F8B8B0B4F8C030A4F8BA3029463046A5
:10D0800004F0A8F984F8C800DFF810B20BF5E072DC
:10D090004146284604F064FA84F8C8009BED727A91
:10D0A000DBED737AF6EE006A67EEA66AB4EEE67A16
:10D0B000F1EE10FA02D501228BF83821B4EEE77AAE
:10D0C000F1EE10FA45DD754B93F83831002B40D066
:10D0D000724B93F83931DBB1704AD2F84031D2F853
:10D0E0004411013341F10001C2F84031C2F844114A
:10D0F0006A4BD3F84021D3F84431332A73F100034B
:10D100000CD30023654A82F8383184F82C3046E08D
:10D11000624B00200021C3E95001E9E7227B604D0A
:10D120002B8803FB02F2D4F8EC10D4F8E800F3F7F4
:10D130001FFE227B2B8802FB03F303FB02F2D4F8D1
:10D14000FC10D4F8F800F3F713FE012384F82C3018
:10D150009AE0DFED546A67EEA66AB4EEE67AF1EE85
:10D1600010FA0FDD4D4B93F838315BB137EEC77ACB
:10D17000DFED4D6A67EEA67AC7EE276A474BC3ED2F
:10D18000676A04E0454B4FF07E52C3F89C21434B45
:10D1900000200021C3E95001002384F82C30B4F8AA
:10D1A0005830A4F8A830B4F88230A4F8AA30424627
:10D1B0003946504604F0D4F984F8C80004F19807C1
:10D1C0003A464946404604F0CBF984F8C8000023AB
:10D1D0000EE0D4F81C2102EB8302304991ED677A0E
:10D1E000D2ED007A67EE877AC2ED007A0133DBB2C6
:10D1F000B4F89820B4F89A1001FB02F29342E8DBED
:10D20000042201E00132D2B2052A1DD80023022BEC
:10D21000F8D8D4F81C1102EB4200184401EB80014D
:10D2200002F15C0C1D4800EB8C00D0ED016ADFEDD3
:10D230001F7A86EEA77AD1ED007A67EE877AC1ED84
:10D24000007A0133DBB2E2E7B4F89830A4F8B830E2
:10D250000123A4F8BA302A463146384604F080F952
:10D2600084F8C8000D4B93F83831002B4DD1D4F819
:10D27000BC300022DA6004F13002294604F13800A3
:10D2800004F018FB84F8C800BDE8F88F3093002044
:10D2900038930020409300204893002030910020D4
:10D2A0005E930020CDCCCC3D6666663FDA0FC93F69
:10D2B0000133DBB2052BDAD8D4F8BC10980001EBAF
:10D2C000830191ED007A124AD2ED6F7ADFED116A97
:10D2D00067EEA67AB4EEE77AF1EE10FA01DDC1ED61
:10D2E000007AD4F8BC20024492ED007A0849D1EDCE
:10D2F0006F7ADFED096A67EEA67AB4EEE77AF1EEAF
:10D3000010FAD5D5C2ED007AD2E70423D2E700BFE8
:10D31000309100200AD7233C0AD723BC10B52DED4D
:10D32000048B0446D0F8EC3093ED009A39EE099A5C
:10D330002E4A82ED009A93ED018A38EE088A2C4A33
:10D3400082ED008AD3ED029A79EEA99A294AC2EDBC
:10D35000009AD3ED038A78EEA88A274BC3ED008AA2
:10D36000827B264B1B8802FB03F3027B03FB02F24A
:10D370000021D0F80C0106F029F9D4F80C31F1EEB7
:10D38000697AC3ED007AD4F80C31C3ED018AD4F880
:10D390000C31B1EE497A83ED027AD4F80C3183ED89
:10D3A000038AD4F80C3183ED068AD4F80C3183ED6E
:10D3B000079AD4F80C31C3ED088AD4F80C31C3EDC8
:10D3C000099AD4F80C3183ED0C9AD4F80C31B1EEF3
:10D3D000488A83ED0D8AD4F80C31C3ED0E7AD4F867
:10D3E0000C31C3ED0F8ABDEC048B10BD14930020EB
:10D3F000189300201C930020209300205E930020AF
:10D4000038B504462F4B01221A7083ED6C0AC3ED28
:10D410006D0A83ED6E1A2C4AC3F8CC21002283F8E2
:10D42000382100200021C3E95001C3E95201F7EE81
:10D43000007AF4EEE71AF1EE10FA01DDF0EE671A69
:10D44000204DC5ED741A85ED642A032300220621C0
:10D45000281D00F029FD05F5E4730122114605F5AC
:10D46000E07004F023FA002309E0164AD2F8EC2019
:10D4700002EB830204EB8301096811600133032B83
:10D48000F3DD104C114BC4F8D030114BC4F8D4303C
:10D49000104BC4F8D830104BC4F8DC30012384F8AA
:10D4A0002E3084F82F3090252A460C49D4F80401F8
:10D4B000F3F75EFC2A460A49D4F8FC00F3F758FC5F
:10D4C00038BD00BF3091002077CC2B32A9CE0008A8
:10D4D00009CD00081DD30008E1CE0008A0420108D4
:10D4E000FC00002010B52DED068BF0EE61AAB0EE29
:10D4F00042AAF0EE629A804C84ED6F3A94ED589A0D
:10D5000030EE490A84ED5B0A94ED598A70EEC80A40
:10D51000C4ED5C0AD4ED5A8A31EE681A84ED5D1AC6
:10D52000F6EE008A20EE280A20EE039A734B83ED74
:10D53000009A60EEA80A20EE838A714B83ED008A80
:10D5400021EE281A61EE038A6E4BC3ED008A902209
:10D550006D49D4F80401F3F70BFCD4F80431F1EE73
:10D56000497AC3ED017AD4F80431F1EE486AC3ED8B
:10D57000026AD4F80431B1EE687A83ED037AD4F804
:10D58000043183ED069AD4F80431C3ED088AD4F847
:10D590000431C3ED096AD4F8043183ED0C8AD4F860
:10D5A000043183ED0D7AD4F8043183ED0F9AD4F869
:10D5B0000431C3ED128AD4F8043183ED138AD4F810
:10D5C0000431C3ED147AD4F84821D4F84C31134314
:10D5D00005D1C4ED5EAA84ED5FAAC4ED609A464B06
:10D5E00093ED5E7AD3ED647A27EE277A93ED6F6A36
:10D5F00077EE866A87EE260A66EE2AAA8AEEA67A71
:10D6000030EE070A83ED5E0AD3ED5F5A67EEA55A46
:10D6100085EEA67A26EE0AAACAEE265A37EE257AB3
:10D6200083ED5F7AD3ED605A67EEA55AC5EEA67A10
:10D6300026EE296AC6EE265A77EEA57AC3ED607A01
:10D6400020EE000A27EE077A30EE070A67EEA77A87
:10D6500030EE270AFFF740FBB0EE408A2B4B83EDFC
:10D66000000A00230FE0244903F15E0201EB82026D
:10D67000D2ED007A8A6802EB830268EE277AC2ED67
:10D68000007A0133DBB2022BEDD91B4C94ED5B0A1F
:10D6900020EE000AD4ED5C7A67EEA77A30EE270A16
:10D6A000D4ED5D7A67EEA77A30EE270AFFF714FB18
:10D6B000B7EE007AC7EE007AC4ED657AC7EE086A65
:10D6C000C4ED666A9FED127AF4EEC77AF1EE10FAB5
:10D6D00024D5DFED107AF4EEE76AF1EE10FA1DDDE5
:10D6E000DFED0D7AF4EEE76AF1EE10FA16D50122BD
:10D6F00084F8392116E000BF3091002024930020E7
:10D70000289300202C930020A042010810930020B1
:10D710009A99993ECDCC1441CDCC24417E4B002228
:10D7200083F839217C4CD4ED6C7A94ED6F7AD4F87F
:10D73000183167EE877AC3ED007AD4ED6C7A94EDF8
:10D740006F7AD4F8183167EE877AC3ED077AD4ED93
:10D750006C7A94ED6F7AD4F8183167EE877AC3ED5E
:10D760000E7AD4ED6C7A94ED6F7AD4F8183167EEB6
:10D77000877AC3ED157AD4ED6D7A94ED6F7AD4F88B
:10D78000183167EE877AC3ED1C7AD4ED6D7A94ED8B
:10D790006F7AD4F8183167EE877AC3ED237AD4F81C
:10D7A0001C21D4F8B8311360D4F81C211361D4F8CB
:10D7B0001C31D4F8B8211A62201D00F0F9FE63680C
:10D7C000D3ED000AC4ED540AD3ED017AC4ED557AC5
:10D7D00093ED027A84ED567A93ED030A84ED570AAD
:10D7E0001A69C4F860215B69C4F864310023C4F885
:10D7F000683120EE800A27EE877A30EE070A60EE65
:10D80000A00A67EEA77A70EEA70A70EEA00AF7EEFC
:10D81000008A70EEE80A30EE000A04F00FFA9FED7D
:10D820003F8A20EE080A84ED6A0AD4ED540A94ED8A
:10D83000550A20EE800A94ED567AD4ED577A27EEF9
:10D84000277A30EE070A60EEA00A67EEA77A70EE3C
:10D85000A70A70EEA00A70EEE80A30EE000A04F0A3
:10D86000EDF920EE080A84ED690AD4ED557A94EDBD
:10D87000570A67EE807A94ED540A94ED567A20EEBA
:10D88000070A77EEC07AB8EE000A27EE800A04F0A5
:10D89000A9F920EE080A84ED680A94ED6A7AD4EDBD
:10D8A000767A77EE677ADFED1E6AF4EEE67AF1EECD
:10D8B00010FA23DDB4F9D431013BA4F8D431164B6E
:10D8C000B3F9D42107EE902AF8EEE77ADFED156A76
:10D8D00067EEA67A77EE277AC3ED6B7A83ED767AD8
:10D8E000D3F84821D3F84C11013241F10001C3F8BB
:10D8F0004821C3F84C11BDEC068B10BDDFED0A6A60
:10D90000F4EEE67AF1EE10FAD9D5034AB2F9D43141
:10D910000133A2F8D431D2E730910020E12E6542E4
:10D92000000034430000B443000034C3D0ED017A5A
:10D9300090ED0D7AD0ED0E6A37EE267AF6EE006A9B
:10D9400027EE267A67EE877A90ED197A67EE877A66
:10D95000C0ED137A7047D0ED0D7A90ED117A27EE75
:10D96000877AB5EEC07AF1EE10FA26DDF5EEC07AD0
:10D97000F1EE10FA1CDD90ED087AB4EEE77AF1EEE4
:10D9800010FA1ADAD0ED076A37EE266AB4EEE76AC3
:10D99000F1EE10FA0FDB76EEE77A77EE277A87EE74
:10D9A000A67AD0ED137A67EE877AC0ED137A7047C6
:10D9B000F1EE677ADFE70023C3647047D0ED116AA8
:10D9C00090ED137A36EE877A1F4B83ED007AD0ED17
:10D9D000107A76EEA77A90ED126A77EE867A1B4B74
:10D9E000C3ED007AF5EEC07AF1EE10FA28DD90ED85
:10D9F000036AB4EEE76AF1EE10FA0AD5D0ED0D7ABB
:10DA000066EEA76AF5EEC06AF1EE10FA01DD0023BA
:10DA1000C364D0ED067AB4EEE77AF1EE10FA03DDD6
:10DA20000023C364C0ED117AF1EE677AB4EEE77AB1
:10DA3000F1EE10FA03D50023C364C0ED117A7047EC
:10DA4000F1EE677AD3E700BF54930020589300208B
:10DA5000D0ED027A90ED0C7AD0ED0B6A37EE667A53
:10DA600067EE877AD0ED196A87EEA67A80ED127A92
:10DA7000704790ED126AD0ED197A26EE276A90ED84
:10DA80000A7A77EE877AC6EE276A90ED166A27EE55
:10DA9000067A87EE276A76EE867AC0ED127A7047AC
:10DAA00090ED146AD0ED197A26EE276A90ED097A86
:10DAB00077EE877AC6EE276A90ED156A27EE067A2A
:10DAC00087EE276A76EE867AC0ED147A704790ED7D
:10DAD000147AD0ED037AB4EEE77AF1EE10FA01DDB4
:10DAE000C0ED147A90ED147AF1EE677AB4EEE77A2D
:10DAF000F1EE10FA01D5C0ED147A704790ED147A6A
:10DB0000B0EEC77AD0ED037ADFED1D6A67EEA67A34
:10DB1000B4EEE77AF1EE10FA2BD4D0ED177AB0EE2E
:10DB2000E77ADFED186AB4EEE67AF1EE10FA20D467
:10DB3000D0ED0B6A77EEE67AF0EEE77AC7EE876A09
:10DB4000DFED117AF4EEE76AF1EE10FA12DD836E82
:10DB5000C26E013342F100028366C266816EC36EFB
:10DB600040F2F512914273F1000302D3012380F8D1
:10DB70007030704700220023C0E91A23EEE700BF8F
:10DB80006F12833A17B7D1383333733F38B5054630
:10DB90000C467822002105F019FD23462A46203440
:10DBA000D3F800E0D3F804C09868D968C2F800E060
:10DBB000C2F804C09060D16010331032A342EFD19C
:10DBC000186859689B6810605160936005F16000A7
:10DBD000FEF7D8FC38BD10B52DED028B0446F0EEF3
:10DBE000408AB0EE608A90F91430002B71DB04F1AA
:10DBF0006000FEF7C7FC84ED190AC4ED0B8A84EDC2
:10DC0000178A78EE680AC4ED0D0AF5EEC00AF1EE47
:10DC100010FA61DDF0EE607A94ED047AB4EEE77A02
:10DC2000F1EE10FA73D5D4ED007A60EEA77AC4ED68
:10DC3000107AD4ED017A60EEA77A60EE277AC4ED0F
:10DC4000137AD4ED027A94ED0E7A70EEC70A67EE7D
:10DC5000A00AC0EE807AC4ED127A237D13F0040F7F
:10DC60003DD1237D13F0200F3DD1237D13F0020F12
:10DC70003DD1237D13F0400F3DD1237D13F0010FE3
:10DC80003DD1D4ED137A94ED117A77EE877AC4ED15
:10DC9000117A94ED107A77EE877A94ED127A77EE16
:10DCA000877AC4ED147A237D13F0100F2BD1204610
:10DCB000FFF70DFFE36A236394ED140A84ED150A60
:10DCC000A36CA365636BA363E36CE363BDEC028B9E
:10DCD00010BDFFF713FF8AE7F1EE607A9CE720465C
:10DCE000FFF724FEBDE72046FFF735FEBDE72046DF
:10DCF000FFF7AEFEBDE72046FFF7BBFEBDE72046BF
:10DD0000FFF75CFEBDE72046FFF7CAFECFE7002322
:10DD10002365E364CEE70000034690B14FF6FF7041
:10DD200009E013F8012B4240D2B2074931F8122022
:10DD300082EA102061464A1E1FFA82FC0029F0D1B7
:10DD400070474FF6FF7070478C010020D8B138B58E
:10DD50000C460546022918D9023989B2FFF7DCFFC3
:10DD60002B19C2B213F8023C9A4201D0002038BDF0
:10DD7000C0F30F202C4414F8013C984201D000203D
:10DD8000F5E70120F3E7002070470020EFE70000EF
:10DD900070B5044600250574827B424E338803FB30
:10DDA00002F24168D0F8F400F2F7E2FFA27B338878
:10DDB00003FB02F22946606805F008FCA27B338869
:10DDC00002FB03F303FB02F22946D4F8180105F025
:10DDD000FDFB227B338802FB03F3A27B03FB02F2F1
:10DDE0002946D4F80C0105F0F1FB294601E0013188
:10DDF000C9B2A37B8B422AD9D4F8F4304FEA810C04
:10DE000003EB8102D2ED007AF5EE407AF1EE10FAE2
:10DE1000EDD0227C03EB8203C3ED007A626A237C9F
:10DE2000D154A069D4F80C2194F80CE0257C6369E6
:10DE30005B5C05FB0E3303F18043013B02EB830384
:10DE4000604402681A60237C01332374CFE7002307
:10DE50000FE0E069616A11F803C0D4F8181102FB01
:10DE6000033201EB820200EB8C0001681160013388
:10DE7000DBB2227C9A42ECD892B2A4F87820237BC1
:10DE8000A4F87A30A4F88030A4F88220A4F8902076
:10DE9000A4F89220A4F89830A4F89A20A4F8482076
:10DEA00070BD00BF5E9300202DE9F04704460D468B
:10DEB00091461E46DFF8B8830423A8F80030EB4BE8
:10DEC00008221A80017380F80D908673002707746A
:10DED000304605F0C3F860613246394605F076FBFE
:10DEE000B8F800A006FB0AFA504605F0B7F8A061A2
:10DEF0005246394605F06AFBB8F800A006FB0AFA5C
:10DF0000504605F0ABF8E0615246394605F05EFB3D
:10DF1000B8F800A005FB0AFA504605F09FF8206209
:10DF20005246394605F052FB304605F097F86062DC
:10DF30003246394605F04AFBB8F8000005FB00F010
:10DF400005F08CF82060B8F8002005FB02F2394695
:10DF500005F03CFBB8F800A006FB0AFA504605F0B5
:10DF60007DF860605246394605F030FBB8F800A0F5
:10DF700009FB0AFA504605F071F8A060524639468E
:10DF800005F024FBB8F800A005FB0AFA504605F09E
:10DF900065F8C4F8E8005246394605F017FBD4F896
:10DFA000E8300122217B04F1300003F07FFCB8F857
:10DFB000008005FB08F8404605F050F8C4F8EC0076
:10DFC0004246394605F002FBD4F8EC300122217BB1
:10DFD00004F1380003F06AFCB9F1000F40F04A8107
:10DFE000DFF88C82B8F8007006FB07F7384605F0BA
:10DFF00035F8C4F8F4003A46002105F0E7FAD4F801
:10E00000F4300122A17B04F1480003F04FFCB8F882
:10E01000007005FB07F705FB07F7384605F01EF80B
:10E02000C4F8F8003A46002105F0D0FA217BD4F874
:10E03000F8300A4604F1500003F038FCB8F80070DC
:10E0400005FB07F705FB07F7384605F007F8C4F8A6
:10E05000FC003A46002105F0B9FA217BD4F8FC30E7
:10E060000A4604F1580003F021FCB8F8007005FBE3
:10E0700007F705FB07F7384604F0F0FF8246C4F8BF
:10E080000001384604F0EAFFC4F804013A460021D2
:10E09000504605F09BFAB8F8002005FB02F205FB9C
:10E0A00002F20021D4F8040105F090FA217BD4F8A3
:10E0B00000310A4604F1600003F0F8FB217BD4F83C
:10E0C00004310A4604F1680003F0F0FBB9F1000FD7
:10E0D00040F0E680664FB7F800A00AFB06F909FB9E
:10E0E00005F9484604F0BAFF8046C4F80C010AFB63
:10E0F00005F006FB00F004F0B1FFC4F810014A4639
:10E100000021404605F062FA3A8805FB02F206FB60
:10E1100002F20021D4F8100105F058FAD4F80C31BD
:10E12000227BA17B04F1780003F0C0FBD4F810310E
:10E13000A27B217B04F1800003F0B8FBB7F80080DC
:10E1400005FB08F808FB05F8404604F087FFC4F813
:10E1500014014246002105F039FA217BD4F814312C
:10E160000A4604F1880003F0A1FBB7F8008006FB23
:10E1700008F808FB06F8404604F070FFC4F81801E0
:10E180004246002105F022FAA17BD4F818310A4654
:10E1900004F1900003F08AFB398801FB05F505FBCB
:10E1A00006F6304604F05AFFC4F81C01324600213E
:10E1B00005F00CFAD4F81C31A27B217B04F1980005
:10E1C00003F074FB267B3F8806FB07F707FB06F589
:10E1D000284604F043FF8046C4F82001284604F096
:10E1E0003DFFC4F82401284604F038FFC4F8280194
:10E1F000384604F033FFC4F82C01384604F02EFFF3
:10E20000C4F83001B1B243460A4604F1A00003F05D
:10E210004DFB217BD4F824310A4604F1A80003F019
:10E2200045FB217BD4F828310A4604F1B00003F005
:10E230003DFBD4F82C310122217B04F1B80003F01E
:10E2400035FBD4F830310122217B04F1C00003F00A
:10E250002DFB002384F8283084F8293084F82A30F4
:10E2600084F82B3084F82C30BDE8F0875C930020D4
:10E270005E930020164B1F8809FB07F7384604F011
:10E28000EDFEC4F8F0003A46002105F09FF9D4F8FD
:10E29000F0300122617B04F1400003F007FB9FE6B0
:10E2A000B8F8002005FB02F202FB09F9484604F029
:10E2B000D5FEC4F808014A46002105F087F9D4F8D4
:10E2C0000831627B217B04F1700003F0EFFA01E773
:10E2D0005E93002038B50446C37B63B1FFF758FD59
:10E2E000627B0E4B1B8803FB02F2A168D4F8F0009E
:10E2F000F2F73EFD38BD827B084D2B8803FB02F20E
:10E300004168D0F8F400F2F733FDA27B2B8803FBC1
:10E3100002F20021606805F059F9E1E75E93002000
:10E3200090F82830B3BB70B50446437B43B3037BFE
:10E33000A0F8B8300126A0F8BA6000F1B8052A4666
:10E3400000F13001603003F00BF984F8C800237B42
:10E35000A4F8C030A4F8C26004F1C006324604F14B
:10E36000400104F1700003F0FBF884F8C80004F1E8
:10E3700038023146284603F09DFA84F8C80070BD83
:10E3800000F1380200F13001603003F0E9F884F860
:10E39000C800F4E77047F8B590F8293003B1F8BD2C
:10E3A000044600F1600600F168073946304603F084
:10E3B00011F884F8C80004F158052A4604F1500108
:10E3C000304603F0CDF884F8C800B4F85830A4F80B
:10E3D000A830B4F86A30A4F8AA3004F1A80632468E
:10E3E0003946284603F0BCF884F8C8002A4604F1F0
:10E3F0008801304603F05EFA84F8C800CFE72DE9C3
:10E40000F84390F82A300BB1BDE8F883044600F1D8
:10E41000780600F180073946304602F0DBFF84F8C9
:10E42000C800B4F87830A4F8A830B4F85A30A4F88A
:10E43000AA3004F1580804F1A8052A46414630469E
:10E4400003F08EF884F8C800B4F8A830A4F8B0300F
:10E45000B4F88230A4F8B23004F1B006324639463E
:10E46000284603F07DF884F8C800B4F89030A4F88A
:10E47000A030B4F89230A4F8A23004F1A0094A46C2
:10E4800004F19001304603F015FA84F8C8003146D3
:10E49000484603F005F984F8C800B4F85830A4F8E9
:10E4A000A830B4F88230A4F8AA302A46394640464B
:10E4B00003F056F884F8C80004F198023146284663
:10E4C00003F04EF884F8C8009EE790F82B3003B1B3
:10E4D00070472DE9F0410446B0F87830A0F8B83024
:10E4E0000126A0F8BA6000F1380700F1B8052A4605
:10E4F0003946783003F034F884F8C800B4F848306E
:10E50000A4F8C030A4F8C26004F1C008424629460D
:10E5100004F1480002F0BAFF84F8C800B4F898305B
:10E52000A4F8B830A4F8BA602A46414604F198002D
:10E5300003F016F884F8C80004F130022946384682
:10E5400003F0B8F984F8C800BDE8F081F8B590F898
:10E550002C3003B1F8BD0446B0F89830A0F8A830CC
:10E56000B0F87A20A0F8AA20A0F8B030B0F85A305D
:10E57000A0F8B23000F1A8073A4600F178019830CF
:10E5800002F0EEFF84F8C80004F1580504F1B0066B
:10E5900032462946384602F0E3FF84F8C80004F109
:10E5A00050023146284602F071FF84F8C800D1E7D6
:10E5B00038B50446FFF78EFED4F8CC300BB12046B8
:10E5C00098472046FFF7ACFED4F8D0300BB1204678
:10E5D00098472046FFF7DFFED4F8D4300BB1204631
:10E5E0009847237C0BB9E37BCBB92046FFF707FFA5
:10E5F000D4F8D8300BB1204698472046FFF765FF86
:10E60000D4F8DC300BB1204698472046FFF79EFF38
:10E61000D4F8E0300BB120469847002319E0227B64
:10E62000204D2B8803FB02F2D4F8EC10D4F8E8005C
:10E63000F2F79EFB227B2B8802FB03F303FB02F223
:10E64000D4F8FC10D4F8F800F2F792FBE0E70133BD
:10E65000DBB2227B9A4214D9D4F8F81002FB0332C1
:10E6600001EB820292ED007A216A01EB8301D1ED88
:10E67000007AB4EEE77AF1EE10FAE8D5C2ED007A4E
:10E68000E5E7084B1B8803FB02F2D4F8E81020688A
:10E69000F2F76EFBD4F8E4300BB1204698472068BF
:10E6A00038BD00BF5E930020F0EE405AB5EEC00AC0
:10E6B000F1EE10FA1ED9F6EE007A20EE270A9FED51
:10E6C0000F6A25EE866A60EE007A77EEE57A70EEE4
:10E6D000006A87EEA67A30EE470AB4EEE76AF1EEFA
:10E6E00010FAF0D4B1EE467AB4EEE77AF1EE10FA11
:10E6F000E9DC70479FED020A704700BF6F12833A52
:10E7000000000000B4EEE00AF1EE10FA07D4B4EE17
:10E71000C10AF1EE10FA04DDB0EE410A7047B0EE26
:10E72000600A7047FDEEC07A0C4BC3ED007AB8EE7C
:10E73000E77A30EE470A0A4B83ED000AB6EE007A1C
:10E74000B4EEC70AF1EE10FA04DD17EE903A013389
:10E75000024A1360014B1868704700BF64930020A1
:10E760006093002010B52DED048B044690ED009AC7
:10E7700069EE097AD0ED018A28EEA80A77EE807A50
:10E7800090ED028A28EE080A37EE800AFFF78CFF28
:10E79000C9EE007AC4ED007AC8EE807AC4ED017A41
:10E7A000C8EE007AC4ED027A2046BDEC048B10BDA1
:10E7B000D0ED017A91ED027A67EE877A90ED027AD8
:10E7C000D1ED016A27EE267A77EEC77AC2ED007A9C
:10E7D000D0ED027A91ED007A67EE877A90ED007ABB
:10E7E000D1ED026A27EE267A77EEC77AC2ED017A7A
:10E7F000D0ED007A91ED017A67EE877A90ED017A9B
:10E80000D1ED006A27EE267A77EEC77AC2ED027A5A
:10E810007047D0ED007A91ED000A67EE807A90EDB6
:10E82000010A91ED017A20EE070A77EE807A90EDE9
:10E83000020A91ED027A20EE070A37EE800A70474D
:10E8400010B50446102004F009FC00230360436067
:10E850008360C360A368C360238803B96423038013
:10E8600063684360638803B9642303812388038159
:10E87000034A1378591C1170024A42F8230010BD54
:10E88000689400206893002003880381704700008B
:10E8900010B5002404E053680BB1D06898470134E8
:10E8A000064B1B78A34208D9054B53F82420138943
:10E8B000002BF0D0013B1381F1E710BD68940020DC
:10E8C0006893002008B5002210210248F3F756FF94
:10E8D00008BD00BF0000024008B501221021024817
:10E8E000F3F74CFF08BD00BF0000024008B500224E
:10E8F00001210248F3F742FF08BD00BF00040240B7
:10E9000008B5012211460248F3F738FF08BD00BFE1
:10E910000004024000B587B08DF80F004FF47A7301
:10E92000009301230DF117020DF10F010448006857
:10E93000F6F7EDFB9DF8170007B05DF804FB00BF8C
:10E940006C94002038B50D46144640F08000FFF767
:10E95000E1FF06E05520FFF7DDFF05F8010B013C64
:10E96000E4B2002CF6D138BD10B50C46FFF7D2FF4B
:10E970002046FFF7CFFF10BD10B50C4640F08000D9
:10E98000FFF7C8FF5520FFF7C5FF207010BD00003E
:10E9900030B52DED048B8BB00446CB4B93E80300D0
:10E9A0000890ADF82410090C8DF8261000238DF87E
:10E9B0002730FDF771FEC54B83ED000AFDF76CFEB5
:10E9C000C24BD3ED007A30EE670AF2EE087AB4EE6D
:10E9D000E70AF1EE10FA0ADC9FEDBD0AFDF7A0FE92
:10E9E000002323636362A362E3620025E1E0B94B85
:10E9F0006362B94BA362E362B84B2363B84BA36174
:10EA0000B84B0093B84BB94AB9490020FAF76CFEED
:10EA100094ED0C7ADFEDB76AC6EE877AC4ED087A1A
:10EA20000BB0BDEC048B30BD9DF823301B021BB234
:10EA30009DF82220134307EE103AAF4BD3ED006A46
:10EA4000B8EEC77A27EE267A84ED037AD4ED097AF8
:10EA500037EE877A84ED097A9DF825301B021BB2C8
:10EA60009DF82420134307EE103AB8EEC77A27EE3C
:10EA7000267A84ED047AD4ED0A7A37EE877A84ED2B
:10EA80000A7A9DF827301B021BB29DF826201343FB
:10EA900007EE903AF8EEE77A67EEA67AC4ED057ACB
:10EAA00094ED0B7A77EE277AC4ED0B7AE5E000233C
:10EAB000022B0DD89A1C04EB820251680AAA02EBC1
:10EAC000830242F8141C42F8201C0133DBB2EFE74A
:10EAD000B0EE688A78EEC86A884BC3ED006A0023FE
:10EAE0003BE00133DBB2022B24D819469A1C04EB1D
:10EAF0008202D2ED017A0AAA02EB830212ED057AB4
:10EB0000F4EEC77AF1EE10FA04DD0AAA02EB8302F2
:10EB100042ED057A0AAA02EB810212ED087AF4EEC0
:10EB2000C77AF1EE10FADCD50AAA02EB810141EDB9
:10EB3000087AD6E7F0EE498ACCE70AAA02EB83020C
:10EB400052ED057A12ED087A77EEC77A6C4A02EB3D
:10EB50008302C2ED007A0133DBB2022BEDD9F6EE6F
:10EB6000007AF4EEE76AF1EE10FA00F39980644B54
:10EB700093ED007ADFED637AB4EEE77AF1EE10FA06
:10EB800000F38E8093ED017AB4EEE77AF1EE10FA9D
:10EB900000F3868093ED027AB4EEE77AF1EE10FA94
:10EBA0007EDC9FED590AFDF7BBFD0135ADB2B0EE3D
:10EBB000689A41F26F739D427CD8FFF783FE9220E2
:10EBC000FFF7A8FE062208A91220FFF7BBFEFFF7F9
:10EBD00083FE9DF821301B021BB29DF820201343B9
:10EBE00000EE103AB8EEC00A484AD2ED007A20EEA4
:10EBF000270A84ED000A9DF823301B021BB29DF802
:10EC000022100B4307EE103AD2ED006AB8EEC77A35
:10EC100027EE267A84ED017A9DF825301B021BB27F
:10EC20009DF82420134307EE903AF8EEE77A67EE5A
:10EC3000A67AC4ED027A20EE000A27EE077A30EEBB
:10EC4000070A67EEA77A30EE270A02F0F9FFF0EE26
:10EC5000408AD4ED0C7A77EE807AC4ED0C7AFFF717
:10EC600045FE082208A90020FFF76CFEFFF748FECA
:10EC70009DF820300F2B3FF4D7AE002D3FF417AF97
:10EC8000B4EEE89AF1EE10FA01D5B0EE689AB4EE5F
:10EC9000E88AF1EE10FA01DDB0EE688A002322E77F
:10ECA000104B00931A4B1B4A1B490020FAF71CFD1E
:10ECB000B0EE689AD4ED0C6A9FED187AC6EE877AAA
:10ECC000C4ED0C7A002339E0C83C0108C894002048
:10ECD0000AD7A33BAC38223BB016CE393F161B41B6
:10ECE00000002042783D0108D83D0108DC3D0108C4
:10ECF00030430108C3F51C4190030020B494002068
:10ED0000B89400209A99193E6F12033A8C030020A0
:10ED10000041010804410108684301080080BB4527
:10ED200003F1080204EB8202D2ED016A1FED057ABD
:10ED3000C6EE877AC2ED017A0133DBB2022BEFD93E
:10ED4000FFF7C0FDA220FFF7E5FD022208A922205F
:10ED5000FFF7F8FDFFF7C0FD9DF820209DF821305A
:10ED60005B0943EAC203B3F5806F01DBA3F50063DF
:10ED700007EE903AF8EEE77AB4EE007A67EE877A1B
:10ED8000B3EE077A77EE877AC4ED067A2D4A1388B8
:10ED9000013313802C4B93ED007AF6EE007AB4EE3B
:10EDA000E77AF1EE10FA3FF709AED4ED0C7A9FED59
:10EDB000277A77EEC77AF0EEE77AB6EE007AF4EECD
:10EDC000C77AF1EE10FA3FF7F9AD214B93ED007AD7
:10EDD000DFED207AB4EEE77AF1EE10FA3FF7EEAD10
:10EDE00093ED017AB4EEE77AF1EE10FA3FF7E6AD73
:10EDF00093ED027AB4EEE77AF1EE10FA3FF7DEAD6A
:10EE0000D4ED097AF0EEE77A9FED137AF4EEC77A43
:10EE1000F1EE10FA3FF7D2ADD4ED0A7AF0EEE77AD0
:10EE2000F4EEC77AF1EE10FA3FF7C8ADD4ED0B7AE5
:10EE3000F0EEE77AF4EEC77AF1EE10FA3FF7BEADE6
:10EE4000E6E500BFB0940020B4940020CDCC1C4176
:10EE5000B89400209A99193E0AD7233C70B52DED3D
:10EE6000028B82B0FFF72EFD8020FFF753FD552067
:10EE7000FFF750FD5520FFF74DFD514C2070FFF777
:10EE80002BFD9FED508AB0EE480AFDF749FCFFF7D5
:10EE900019FD8020FFF73EFD5520FFF73BFD552073
:10EEA000FFF738FD2070FFF717FDB0EE480AFDF7B9
:10EEB00037FCFFF707FDB6217E20FFF755FDFFF772
:10EEC0000BFD9FED410AFDF72BFCFFF7FBFC8020BB
:10EED000FFF720FD5520FFF71DFD5520FFF71AFD18
:10EEE0002070FFF7F9FCB0EE480AFDF719FCFFF7B8
:10EEF000E9FC8020FFF70EFD5520FFF70BFD5520A4
:10EF0000FFF708FD2070FFF7E7FCB0EE480AFDF7B9
:10EF100007FC23781E2B03D12C4B00221A7011E022
:10EF20002B4B00932B4B2C4A2C490020FAF7DCFB8F
:10EF3000FF2041E0A2782A49087802430A70013391
:10EF4000224A1370214B1B78052B34D8FFF7BAFCEB
:10EF50001E4D2B78234C03EB4303E2185178E05C01
:10EF6000FFF702FDFFF7B8FC9FED168AB0EE480AE6
:10EF7000FDF7D6FBFFF7A6FC2B7803EB4303E05C21
:10EF800040F08000FFF7C6FC5520FFF7C3FC55207A
:10EF9000FFF7C0FC0A4E3070FFF79EFCB0EE480A47
:10EFA000FDF7BEFB2B7803EB430214446178327803
:10EFB0009142BFD1C3E7002002B0BDEC028B70BD0F
:10EFC000C49400206F12833A0AD7A33DCC9400204A
:10EFD000783D0108D83D0108DC3D0108984301084F
:10EFE000B29400200044010870B52DED028B82B070
:10EFF000FFF77CFC494C21460020FFF7BDFCFFF7E2
:10F000007FFC9FED478AB0EE480AFDF789FBFFF7CA
:10F010006DFC21460020FFF7AFFCFFF771FCB0EE5E
:10F02000480AFDF77DFBFFF761FCB6211420FFF7CE
:10F030009BFCFFF765FC9FED3B0AFDF771FBFFF7BB
:10F0400055FC21460020FFF797FCFFF759FCB0EE76
:10F05000480AFDF765FBFFF749FC21460020FFF752
:10F060008BFCFFF74DFCB0EE480AFDF759FB237807
:10F070000F2B03D12C4B00221A7019E02B4B00935D
:10F080002B4B2C4A2C490020FAF72EFBFF2041E0A5
:10F09000013BDBB22B7003EB4303284A13449B78FC
:10F0A000274A11780B4313701F4A137801331370EA
:10F0B0001D4B1B78052B2CD8FFF718FC1A4D2B780D
:10F0C000204C03EB4303E2185178E05CFFF74CFC63
:10F0D000FFF716FC9FED128AB0EE480AFDF720FB01
:10F0E000FFF704FC0D4E2B7803EB43033146E05C45
:10F0F000FFF742FCFFF704FCB0EE480AFDF710FBF7
:10F100002B7803EB43021444617832789142BFD1EB
:10F11000CAE7002002B0BDEC028B70BDC494002091
:10F120006F12833A0AD7A33DCC940020783D0108A2
:10F13000D83D0108DC3D0108CC430108004401082A
:10F14000B29400201444010838B50D46114B1860E4
:10F15000114C00232370FFF781FE237818432070A1
:10F16000FFF742FF23781843207075B90B4B0C4A08
:10F170005A620C4A9A62DA620B4A1A630B4A1A62A2
:10F180000B4A9A61044B187838BD0448FFF700FC1D
:10F19000F8E700BF6C940020B29400207094002027
:10F1A000AC38223BB016CE393F161B41C48B813F91
:10F1B0000000204238B50546FFF784FB9220FFF798
:10F1C000A9FB734C062221461220FFF7BBFBFFF779
:10F1D00083FB63781B021BB2227813436D4A1380B2
:10F1E00007EE903AF8EEE77A6B4991ED007A67EE18
:10F1F000877A95ED087A67EE877AC5ED007AE3782D
:10F200001B021BB2A07803431380D1ED006A07EE06
:10F21000903AF8EEE77A67EEA67A67EE277AC5EDC0
:10F22000017A63791B021BB221790B43138007EE2D
:10F23000903AF8EEE77A67EEA67A67EE277AC5EDA0
:10F24000027AFFF753FB082221460020FFF77AFBE2
:10F25000FFF756FB23780F2B2BD0FFF733FBA220B1
:10F26000FFF758FB4A4C022221462220FFF76AFB97
:10F27000FFF732FB227863785B0943EAC203454A11
:10F280001380B3F5806F02DBA3F500631380414B5D
:10F29000B3F9003007EE903AF8EEE77AB4EE007A70
:10F2A00067EE877AB3EE077A77EE877AC5ED077A4D
:10F2B00038BD3A4B1B78002B3AD0E3781B021BB2C7
:10F2C000A1780B4333490B803548D0ED006A07EE37
:10F2D000903AB8EEE77A27EE267AD5ED097A37EE3E
:10F2E000677A85ED037A63791B021BB220790343A9
:10F2F0000B8007EE903AB8EEE77A27EE267AD5ED46
:10F300000A7A37EE677A85ED047AE3791B021BB23D
:10F31000A27913430B8007EE903AF8EEE77A67EE96
:10F32000A67A95ED0B7A77EEC77AC5ED057A94E764
:10F33000174AD3781B021BB291780B4315490B80F7
:10F340001748D0ED006A07EE903AB8EEE77A27EE5C
:10F35000267A85ED037A53791B021BB21079034399
:10F360000B8007EE903AB8EEE77A27EE267A85ED25
:10F37000047AD3791B021BB2927913430B8007EEF8
:10F38000903AF8EEE77A67EEA67AC5ED057A64E77B
:10F39000A8940020A49400208C0300209403002053
:10F3A00090030020014B1B6858637047E06A0020FF
:10F3B00070B52DED028B8AB00646002407940894A0
:10F3C00009940023049305934FF07E530693019410
:10F3D0000294039421E0354D2846FFF7EBFE95EDAE
:10F3E000027ADDED077A77EEC77ACDED077A95EDF3
:10F3F000017ADDED087A77EE877ACDED087A95ED22
:10F40000007ADDED097A77EE877ACDED097A9FED06
:10F41000280AFDF785F90134E4B2632CDBD9002317
:10F420000CE00AAA02EB830252ED036A9FED217AF7
:10F43000C6EE877A42ED037A0133DBB2022BF0D9B4
:10F4400007A8FFF78FF904A907A8FFF7E2F902F070
:10F450009DFBB0EE408A01AA04A907A8FFF7A8F90E
:10F4600001A8FFF77FF9F6EE007A28EE278AB0EEC2
:10F47000480A02F019FB86ED000A002410E00AABEE
:10F4800003EB840353ED098AB0EE480A02F044FB13
:10F49000013406EB840368EE808AC3ED008AE4B28F
:10F4A000012CECD90AB0BDEC028B70BD7094002029
:10F4B0006F12833A0000C84270B52DED068B86B0FE
:10F4C00004460D46164690ED040A9F4BD3ED007A94
:10F4D00070EE677AF0EEE77A9FED9C7AF4EEC77AE9
:10F4E000F1EE10FA22DCD0ED057A994B93ED007A1B
:10F4F00077EEC77AF0EEE77A9FED947AF4EEC77A6A
:10F50000F1EE10FA12DCD0ED067A924B93ED007A10
:10F5100077EEC77AF0EEE77A9FED8C7AF4EEC77A51
:10F52000F1EE10FA02DC0378002B6ED09FED8AAA70
:10F5300080EE0A0A02F06EFAB0EE409A94ED050AE7
:10F5400080EE0A0A02F066FAF0EE408A94ED060AAE
:10F5500080EE0A0A02F05EFAF0EE40AA94ED040A88
:10F5600080EE0A0A02F010FAB0EE408A94ED050A25
:10F5700080EE0A0A02F008FAF0EE409A94ED060ACC
:10F5800080EE0A0A02F000FA69EE2A6A28EE297A69
:10F5900027EE007A36EE877A704B83ED007A28EEFC
:10F5A000887A6F4B83ED007A29EE006A6AEE885AFA
:10F5B00025EEA97A36EE476A6A4B83ED006A29EE9A
:10F5C000297A27EE007A37EE657A674B83ED007A69
:10F5D00029EE289A654B83ED009A28EE408A66EE64
:10F5E000A96A38EE668A624B83ED008A68EEC07ABB
:10F5F000604BC3ED007A604BC3ED009A68EEAA8AB7
:10F600005E4BC3ED008A00232370002310E005EB5E
:10F610008302D2ED007A04EB830292ED017A67EE69
:10F62000877A06AA02EB830242ED037A0133DBB24A
:10F63000022BECD9DDED037A484B93ED006A27EEFF
:10F64000867A9DED045A464BD3ED002A65EE226A78
:10F6500037EE267ADDED055A424B93ED003A65EE22
:10F66000836A37EE267A85ED007A3F4BD3ED006A48
:10F6700027EEA67A3D4BD3ED003A65EE234A37EEEE
:10F68000247A3B4B93ED004A65EE844A37EE247AA8
:10F6900085ED017A374B93ED007A67EE877A364B2A
:10F6A000D3ED004A25EE245A77EE857A334B93ED5D
:10F6B000005A65EE855A77EEA57AC5ED027A0023E9
:10F6C00009E006EB8302116806AA02EB830242F806
:10F6D000181C0133DBB2022BF3D99DED002A26EE74
:10F6E000026ADDED015A62EEA52A36EE226ADDEDF0
:10F6F000027A23EE273A36EE036A86ED006A66EE5A
:10F70000826A63EEA53A76EEA36A24EE274A76EE85
:10F71000846AC6ED016A27EE027A64EEA54A37EEE6
:10F72000247A25EE275A37EE057A86ED027A226989
:10F73000054B1A606269064B1A60A269054B1A6094
:10F7400006B0BDEC068B70BD249600206F12833A84
:10F750001C96002020960020E12E6542F0950020A6
:10F76000F4950020F8950020FC95002000960020DC
:10F7700004960020089600200C9600201096002089
:10F7800010B50F4CDFED0F0A0F4B93ED070A204623
:10F79000FEF721FA94ED140AFEF7C4FF00EE100AFA
:10F7A0009FED0A1ADFED0A0AB8EEC00AFEF7AAFFBB
:10F7B000BCEEC00A10EE103A98B2FFF7F3FD10BD90
:10F7C0007895002000002042709400200000804FB7
:10F7D000000000002E4B93F880300BB12D4870478D
:10F7E00030B52DED028B91B0294B012283F880209A
:10F7F00000212948F6F70AFA01212848FFF7A4FC5E
:10F800000028F9D1264BB7EE008A83ED018A83EDFB
:10F81000028A83ED038ADFED238AC3ED048AC3EDF8
:10F82000058AC3ED068A01251D7000240C940D94F1
:10F830000E940F940CA8FFF7BBFDB0EE682AF0EE13
:10F84000481A9FED191ADFED190AB2EE040A0CA846
:10F85000FDF7D6FD2C22214601A803F0B7FE144B7C
:10F860000193144B0293144B04938DF81850134BCF
:10F87000079301A91248FEF789F9054B114A9A62CC
:10F880001148FCF77FFE034811B0BDEC028B30BD80
:10F89000EC9400203C950020E06A00209C69002048
:10F8A000D094002000000000002474496F12833AB5
:10F8B00000007A440000A0410000FA440000964392
:10F8C0007895002096430B3C7095002092ED026ADB
:10F8D00066EE067AF6EE006A76EEE77A92ED037A45
:10F8E00067EE075A77EEE57AD0ED005A67EEA57A13
:10F8F000D2ED014A66EE245A92ED005A27EE054AEF
:10F9000075EEC45A90ED014A65EE845A77EEA57AF9
:10F9100027EE247A26EE056A37EE067A90ED026A23
:10F9200027EE067A77EE877A77EEA77AC1ED007A2E
:10F93000D2ED015AD2ED027A25EEA77AD2ED004A35
:10F9400092ED035A24EE856A37EE067A90ED006A4E
:10F9500027EE067A25EEA56A36EEC66A25EE054A3A
:10F9600036EE446A90ED014A26EE046A37EE067AD6
:10F9700067EE857A65EEA45A77EEE57A90ED026A35
:10F9800067EE867A37EE277A37EE077A81ED017ACD
:10F99000D2ED015A92ED037A65EE877A92ED005A24
:10F9A00092ED026A65EE064A77EEE47AD0ED004AFF
:10F9B00067EEA47A27EE067A25EE855A37EE057AA9
:10F9C00090ED015A27EE057A77EE877A65EEA55A13
:10F9D00076EEE56A26EE066A76EEC66A90ED027A63
:10F9E00066EE876A77EEA67A77EEA77AC1ED027A9D
:10F9F000704792ED026A66EE067AF6EE006A76EEDF
:10FA0000E77A92ED037A67EE075A77EEE57AD0ED62
:10FA1000005A67EEA57AD2ED014A66EE245A92EDBD
:10FA2000005A27EE054A75EE845A90ED014A65EEBC
:10FA3000845A77EEA57A27EE247A26EE056A37EE09
:10FA4000467A90ED026A27EE067A77EE877A77EEAD
:10FA5000A77AC1ED007AD2ED015AD2ED027A25EEF5
:10FA6000A77AD2ED004A92ED035A24EE856A37EE6A
:10FA7000467A90ED006A27EE067A25EEA56A36EE04
:10FA8000C66A25EE054A36EE446A90ED014A26EE36
:10FA9000046A37EE067A67EE857A65EEA45A77EE49
:10FAA000A57A90ED026A67EE867A37EE277A37EE0E
:10FAB000077A81ED017AD2ED015A92ED037A65EE73
:10FAC000877A92ED005A92ED026A65EE064A77EE69
:10FAD000A47AD0ED004A67EEA47A27EE067A25EEE6
:10FAE000855A37EE457A90ED015A27EE057A77EE82
:10FAF000877A65EEA55A76EEE56A26EE066A76EE18
:10FB0000C66A90ED027A66EE876A77EEA67A77EE9D
:10FB1000A77AC1ED027A704770B586B000230393CF
:10FB20000493564B05935648FCF72CFD554E86ED35
:10FB3000000A554BD3ED007A37EE800A83ED000AB8
:10FB4000524D2846FFF736FBD5ED027AF1EE677A83
:10FB50004F4CC4ED177A6B6823662B686366D5ED4E
:10FB6000057AF1EE677AC4ED147A2B696365EB6868
:10FB7000A36504F15C0204F150014648FFF79CFCC8
:10FB800096ED003AD4ED192A94ED182AD4ED171AFF
:10FB900094ED161AD4ED150A94ED140AFDF7A2FCA3
:10FBA0003D4B0FCB84E80F00224604F12C013B486B
:10FBB000FFF78CFE224604F138013948FFF786FE34
:10FBC000224604F144013748FFF780FE2246694689
:10FBD00003A8FFF70EFF002327E02D4A03F11601CB
:10FBE00002EB810191ED017A06A901EB830151ED50
:10FBF000067A37EE677A2349D1ED007A27EE277A25
:10FC0000D2ED0A6A77EEA67A87EE276A191D02EB13
:10FC1000810292ED007A66EE876A86EEA77A76EE2A
:10FC2000077AC2ED007A0133DBB2022BD5D9184C2A
:10FC3000224604F11C0104F11000FFF747FE1A4BA5
:10FC400093ED6A0A84ED1C0AD3ED690AC4ED1B0A20
:10FC5000D3F8A021A266D3F8AC31636700F060F856
:10FC6000124B1B6813F0010F05D0104A13680133C3
:10FC7000136006B070BDFFF783FDF6E7C3F51C41C6
:10FC8000709500201896002028960020709400207F
:10FC9000EC940020D0940020809200202844010899
:10FCA000344401084044010830910020149600209B
:10FCB00000B583B0054B0093054B064A064900206A
:10FCC000F9F712FD03B05DF804FB00BF783D0108B1
:10FCD00000410108044101084C44010838B50E4BAD
:10FCE00018680378A52B00D038BD3021FEF72EF818
:10FCF0000028F9D0084B1C68084D04F1300EAC46C2
:10FD000020686168A268E368ACE80F0010346546BB
:10FD10007445F4D1E8E700BF8C9600202C960020B3
:10FD2000044A10EE103AC2F8063010EE903AC2F8CB
:10FD3000023070477496002010B586B004AB0024E2
:10FD4000049405940B4A059293E80300FCF71CFF0A
:10FD5000094B18600194029403940523ADF8043014
:10FD6000064B029301A8FEF76BFD054B1860054892
:10FD700006B010BDDDFC00088C960020B1FC000828
:10FD8000909600202C96002038B50C4C5A232370F6
:10FD900016212046FDF7C0FFE082094DAE46A4467D
:10FDA000BCE80F00AEE80F009CE803008EE80300FB
:10FDB00018212846FCF706FF38BD00BF74960020C6
:10FDC0005C96002010B582B00446212103F0ECFCC3
:10FDD0001F2801D802B010BD044B01930094044BBE
:10FDE000044A05490020F9F77FFCFEE7783D010849
:10FDF000D83D0108DC3D010888440108884200D153
:10FE0000704700B585B0054B029301910090044BFB
:10FE1000044A05490020F9F767FCFEE7783D010830
:10FE2000D83D0108DC3D0108AC440108F8B50546A1
:10FE30000F46FFF7C7FF144C2646A46A74B1294643
:10FE40002046F1F741F80028F6D194F82110384601
:10FE5000FFF7D4FF012384F82C3012E0302003F0A8
:10FE6000FDF8B0623022002103F0B0FBB36A83F8E2
:10FE700021702946B06A03F039FC012386F82C3042
:10FE8000B46A2046F8BD00BF98030020F8B50E46BE
:10FE9000FFF7CCFF07460C2003F0E0F805460024EE
:10FEA000046044608460067144B17B6A6BB11A4699
:10FEB0009B68002BFBD195602846F8BD304603F0C7
:10FEC000CDF845F824000134EEE77D62F4E710B583
:10FED0000446C07900B910BD0B466179227954F807
:10FEE00021101846F0F744FF637901336371002352
:10FEF0006371E379013BE3710120ECE770B50546DE
:10FF00000E46426A0F4B1A600FE0A37995F8212044
:10FF1000314654F82300F0F72BFF0023A371E37957
:10FF20000133E371A268074B1A60064B1C683CB1B1
:10FF3000E379012BE9D100226271013BE371E4E72F
:10FF4000012070BD9496002000B585B0D0F8A8318E
:10FF500019680A4A91420ED0022209490291DB69CE
:10FF600001930092074B084A08490020F9F7BCFBAF
:10FF700005B05DF804FB0122EFE700BFB06300208D
:10FF8000783D01080041010804410108D0440108FE
:10FF900030B585B00C4609794A1ED2B290F8AE3120
:10FFA000012B57D05DB2002D00F0BC80023BDBB2CC
:10FFB000012B00F2B780032A14D821685F4B9942C5
:10FFC0000DD01346042102F20122A2605C4A0125F1
:10FFD000555480F8AD3180F8AC1100230FE0134682
:10FFE0000121F0E74B1FDBB2256854498D4201D057
:10FFF0000321E8E70021E6E701251FE00133514A2C
:020000040801F1
:1000000012789A4240F297804F4A52F82320D2F851
:10001000A821106821688842F0D1516BA2689142F2
:10002000ECD14A4B00934A4B4A4A4B490020F9F71E
:100030005BFB2268414B9A42DED00225434B029380
:100040000195A3680093424B424A44490020F9F7C6
:100050004BFBF3E790F8AF31012B13D0032A2AD8DA
:100060002168364B994223D01346032102F2052220
:10007000A260334A0125555480F8AD3180F8AC11A7
:10008000002325E0032A09D821682C4B994202D08D
:1000900013460821EAE713460621E7E74B1FDBB2C8
:1000A000256826498D4201D00921DFE70721DDE7D8
:1000B00013460021DAE74B1FDBB225681F498D424A
:1000C00001D00521D2E70221D0E701251EE001334E
:1000D0001C4A12789A422ED91B4A52F82320D2F891
:1000E000A821106821688842F1D1516BA268914221
:1000F000EDD1164B0093164B164A17490020F9F71D
:10010000F3FA22680D4B9A42DFD002250F4B02937F
:100110000195A36800930E4B0E4A10490020F9F791
:10012000E3FAF3E7094B0093094B0A4A0C49002014
:10013000F9F7DAFAF6E705B030BD00BFB06300208A
:10014000CC960020C896002098960020783D0108A3
:10015000D83D0108DC3D01080C4501087C4501083B
:10016000A845010838B50546D0F83D40D4F8B4019B
:10017000FEF78AFB04F5DC70FCF704FA84ED6F0AE5
:100180006188218095F82C3095F82D2042EA0322D1
:10019000628007EE902AF8EE677ADFED2F6A67EE4D
:1001A000A66AC4ED016AD4ED027A9FED2C7A27EE9F
:1001B000877A95F82E0095F82F3043EA00231BB27A
:1001C00007EE903AF8EEE77A9FED256A67EE867AB9
:1001D00077EE277AC4ED027AB4F90C3007EE903A44
:1001E000F8EEE77A9FED1F7A27EE877A95F83000D0
:1001F00095F8313043EA00231BB207EE903AF8EE4F
:10020000E77A9FED196A67EE867A77EE277AFDEE38
:10021000E77A17EE903AA38195F83230A373521A19
:10022000B2F5805F10DD6369013B636163694FF480
:10023000B47202FB03F307EE903AF8EEE77A77EE3A
:10024000A67AC4ED047A38BD12F5805FEEDA6369F0
:1002500001336361EAE700BFACFF333D9899193E73
:100260003433A340D0CCCC3D6666663F002380F893
:10027000B0317047012380F8B031704770B584B059
:1002800005464FF4E07002F0E9FE04464FF4E072D8
:10029000002103F09BF995F89C3084F8AE3104F10D
:1002A000180305F1940292E8030083E8030095F82F
:1002B000B43084F8AF3105F1100104F13000FDF7DE
:1002C00065FC05F13C0104F1A800FDF75FFC05F1B8
:1002D000680104F59070FDF759FC2B6823626B6888
:1002E0006362EB68E362AB68A36205F1A006314686
:1002F0002046FFF74DFE134BC5F8AC30C5F8B040B3
:100300003046FBF7E7FFC4F8A801002301930293EE
:1003100003936423ADF804300B4B0293039401A8BC
:10032000FEF78EFAC4F8B4012046FFF7A3FF074A90
:100330001378591C1170064A42F82340204604B035
:1003400070BD00BF6501010849FF0008C896002084
:100350009896002080ED660A7047000070B52DED7C
:10036000028B002553E0B1EE400A5DE0237F012BB4
:100370000AD0D4ED047AF0EE400AB0EE670A04F534
:100380009070FDF728FC56E0236AD3ED007AF2E77F
:10039000636AD3ED007AF0EE400AB0EE670A04F12A
:1003A000A800FDF718FCA37F13F0010F04D0E36A47
:1003B000D3ED007A30EE270AE37E012B5AD0E37F9B
:1003C000012B5AD09FED711ADFED710AFEF79AF9F1
:1003D000FDEEC07A17EE902A94F8AC1194F8ADC1F6
:1003E0004FEA4C00C2F3072601EB811E694B7344B0
:1003F00003EB4C0E8EF8246000F1010E734483F879
:10040000242094F8B031002B00F09C800135624B21
:100410001B78AB4240F2A480604B53F8254094ED2A
:10042000660AA37E012B9ED0637E13F0040F02D0D8
:10043000237E042B9AD0637E13F0020FB3D0237E69
:1004400013F0060FAFD0A37F13F0020F04D0A36AFE
:10045000D3ED007A30EE270A637F012B98D0E37E3C
:10046000012B02D0D4ED027A95E7D4ED027AF1EEB9
:10047000677A90E7B1EE400AA1E794ED027AF1EED7
:10048000087A87EE276ADFED467A60EE277A67EE14
:10049000867A9FED447A26EE077A27EE067A77EE83
:1004A000877ADFED416A60EE266A66EE806A77EE53
:1004B000A67AC4ED687AD4ED696AF7EE005AF4EED4
:1004C000E56AF1EE10FABFF67DAFF5EEC07AF1EE17
:1004D00010FA3FF577AFF4EEE56AF1EE10FA7FF52A
:1004E00071AF67EEA67A9FED2E8A26EE088A77EE28
:1004F000677AB5EEC00AF1EE10FA10D428EE080AB9
:100500009FED2A7A67EE877A30EE670A01F098FB52
:1005100030EE486ADFED267A86EE270A52E7F1EEE2
:10052000488A28EE088A9FED217A67EE877A38EEAE
:10053000670A01F085FB78EEC08ADFED1D7A88EE50
:10054000A70A3FE701EB81112031124B1944043116
:100550000844002341F81C3043608360C36055E7C2
:10056000002400E00134092C0CD8124B1B5D002B39
:10057000F8D004EB8413B7EE000A06481844FBF7E2
:1005800023FFEFE7BDEC028B70BD00BF000080468B
:10059000000080C6C8030020C8960020989600205E
:1005A000CFC9DA35635A1A35D6D98A34D6D98A35BD
:1005B000D6D90A35CC96002003780A7802700B70E1
:1005C0007047000070B5002677E094F82830012BC2
:1005D00012D094ED030A04F59870FDF7FCFAF0EEE2
:1005E000400A94F82A3013F0020F79D0636BD3EDF0
:1005F000007A70EE270A73E0E36A93ED000AEAE7F7
:10060000236B93ED000A7BE094F8253013F0010F83
:1006100040F08880FDEEE00A10EE903A1BB294F8AC
:100620002620012A00F08780494D2A78022161F3B3
:1006300047122A70D2B26FF384022A70D2B201211B
:1006400061F301022A7007EE903AF8EEE77A17EEAE
:10065000903AC5F801300A236B710023AB71072172
:10066000D4F8B001FBF70CFFD4F8B0312868586219
:10067000A988AA79198583F82A20D4F8B00100F155
:1006800028012530FFF798FFD4F8B00100F12701C9
:100690002630FFF791FFD4F8B00100F12A0129308C
:1006A000FFF78AFF94F8AC31002B47D09FED290A61
:1006B000D4F8B001FBF788FE0136274B1B78B34214
:1006C00044D9264B53F82640D4ED6A0A94F82530D5
:1006D00013F0040F04D094F82430042B3FF475AFCA
:1006E00094F8253013F0020F8ED094F8243013F0D4
:1006F000060F89D094F82830012B81D094ED020A9E
:1007000004F59870FDF767FAF0EE400A94F82A3085
:1007100013F0010F3FF478AFA36BD3ED007A70EEC6
:10072000270A71E794ED030A04F14000FDF753FA3C
:10073000F0EE400A6EE75B421BB275E7D4F8B001F9
:10074000072200212430F0F713FBAFE770BD00BF94
:10075000D4960020CDCC4C3EEC960020DC960020B8
:1007600031EE601A30EE600A01238340013B07EE50
:10077000903AF8EEE77A60EE277A87EE817AFCEE1F
:10078000C77A17EE903A98B27047000008B5044651
:10079000D0F8B85148E094F83030012B0CD094EDEB
:1007A000007AF0EE400A9FED4B0A27EE000A04F5AE
:1007B0009470FDF710FA42E0D4F8A03193ED007A7E
:1007C000EFE7D4F8A43193ED007A53E0F0EE400A5D
:1007D00094ED080A04F13800FDF7FDF964E0B1EE8C
:1007E000400A65E0BBEE020A0C20B3EE021AFBEEF3
:1007F000020AFFF7B5FF94F8B43143B90C20B3EE09
:10080000021AFBEE020A9FED340AFFF7A9FF030A62
:1008100085F82A3085F82B00B6EE000A2846FBF74B
:10082000D3FD0120F7F7B6FD94ED6C0A94F82D3056
:1008300013F0040F03D094F82C30042BABD094F8B1
:100840002D3013F0020F1FD094F82C3013F0060F48
:100850001AD094F8323013F0020F05D0D4F8A83132
:10086000D3ED007A30EE270A94F83030012BA8D06F
:1008700094ED027AF0EE400A9FED160A27EE000A88
:1008800004F1B000FDF7A7F994F8323013F0010F2E
:1008900005D0D4F8AC31D3ED007A30EE270A94F8C5
:1008A0002D3013F0010F91D194F82E30012B96D0FA
:1008B000FBEE027AB4EEE70AF1EE10FA92D9F3EE0B
:1008C000027AB4EEE70AF1EE10FA8DDBB0EE670AB9
:1008D0008AE700BFE12E65420000000030B58BB012
:1008E00047F26843089300238DF82430154B1B789A
:1008F0002BB300251FE00023ADF800300A22694623
:10090000284602F095FB694608A802F0CFFE0DF1DB
:10091000040C0D4C0FCCACE80F0094E807008CE8F9
:1009200007000A4B53F8251001A8F7F7FEFC084B07
:1009300043F825000135034B1B78AB42DBD80BB0E5
:1009400030BD00BF10970020D03C0108F096002079
:100950000097002038B500253FE094F82430012BA3
:1009600016D0B4F90C3000EE103AB8EEC00A04F517
:100970009470FDF730F9F0EE400A94F8263013F049
:10098000020F3CD0236BD3ED007A70EE270A36E0DD
:10099000A36A93ED000AEAE7E36A93ED000A3EE0FA
:1009A00094F8213013F0010F4AD1FDEEE00A10EE69
:1009B000903A1BB294F82220012A4ED0314A126894
:1009C0002432D4F8A811C969A1F5207122F8113098
:1009D00094F8A431002B43D001352B4B1B78AB424C
:1009E00047D92A4B53F82540D4ED680A94F82130B2
:1009F00013F0040F03D094F82030042BADD094F8FA
:100A0000213013F0020FCBD094F8203013F0060FF2
:100A1000C6D094F82430012BBED094ED020A04F520
:100A20009470FDF7D8F8F0EE400A94F8263013F0F1
:100A3000010FB5D0636BD3ED007A70EE270AAFE7F4
:100A4000B4F90C3000EE103AB8EEC00A04F13800E8
:100A5000FDF7C1F8F0EE400AA7E75B421BB2ADE735
:100A6000D4F8A831DB69A3F52073002122F8131014
:100A7000B2E703B938BD9FED060A024B1868FBF7D1
:100A8000A3FCF7E72497002011970020149700207B
:100A9000CDCC4C3E08B5FFF761FCFFF75BFFFFF7DD
:100AA00091FD00F03DF808BD38B50546142002F070
:100AB000D5FA04460023036043608360C36003618A
:100AC0002B7883726868E060A9682161F5F79EF869
:100AD000044A1378591C1170034A42F823402046F7
:100AE00038BD00BF3697002038970020837A012B4D
:100AF0000AD0022B0ED01BB100290FDBC18070473A
:100B0000B429F9DDB421F9E7B1F5877FF4DD4FF4BD
:100B10008771F3E76429EFDD6421EFE70021EDE75A
:100B200038B5002574E0B4F902304FF47A7000FB58
:100B300003F38C4880FB03201844DB17C3EBA010A1
:100B4000EFF7A0FC0022884BEFF750FBEFF716FF02
:100B5000864B23F8150070E0B4F904304FF47A7036
:100B600000FB03F37F4880FB03201844DB17C3EB33
:100B7000A010EFF787FC00227B4BEFF737FBEFF776
:100B8000FDFE7A4B23F815005AE0042B08D0082B01
:100B90000DD0E3681B68754A32F915201A6436E0F7
:100BA000E3681B68714A32F915209A632FE0E36805
:100BB0001B686E4A32F91520DA6328E02378012B8E
:100BC00062D02378022B78D02378BBB9B4F90630F1
:100BD0004FF47A7000FB03F3654880FB0320184450
:100BE000DB17C3EBE010EFF74DFC00225E4BEFF795
:100BF000FDFAEFF7C3FE5D4B23F815002369002BC8
:100C000074D1E3681B68594A32F915205A630135DB
:100C1000584B1B78AB4240F2A380574B53F825400A
:100C2000002CF4D0A37A012BC8D0022B77D0002B54
:100C3000EDD12378012B3FF476AF2378022B8BD0B4
:100C40002378BBB9B4F906304FF47A7000FB03F394
:100C5000444880FB03201844DB17C3EBA010EFF7D8
:100C600011FC0022404BEFF7C1FAEFF787FE3F4B34
:100C700023F815002369002B87D1E3681B683B4AE2
:100C800032F915205A63C2E7B4F902304FF47A7092
:100C900000FB03F3364880FB03201844DB17C3EB4B
:100CA000E010EFF7EFFB00222F4BEFF79FFAEFF783
:100CB00065FE2E4B23F8150083E7B4F904304FF49A
:100CC0007A7000FB03F32A4880FB03201844DB17EB
:100CD000C3EBE010EFF7D6FB0022234BEFF786FAC9
:100CE000EFF74CFE214B23F815006DE7042B08D0DD
:100CF000082B0DD0E3681B681C4A32F915201A64D2
:100D000085E7E3681B68194A32F915209A637EE784
:100D1000E3681B68154A32F91520DA6377E72389FF
:100D200003EB83039B009BB203F5FA731BB20F4ADC
:100D300022F8153022691AB9E2681268536366E72F
:100D4000042A05D0082A07D0E268126813645EE717
:100D5000E268126893635AE7E2681268D36356E761
:100D600038BD00BFB7600BB600407F402897002019
:100D700049D6B9F236970020389700200278044B04
:100D80001A8042785A8082789A80C278DA807047D6
:100D90005897002010B582B0094B00241C605C609D
:100DA0009C60DC60074B1868FBF714FE064B009351
:100DB000064B074A07492046F8F796FC02B010BDDB
:100DC000589700206C970020783D010800410108E9
:100DD000044101080C46010808B5044B1868FDF7EA
:100DE00053FD034B1868FFF7C9FF08BD6897002043
:100DF0006C97002010B586B00E4B059304900A2422
:100E00008DF80C4003A8FBF7F7FD0B4B186000238F
:100E1000009301930293ADF80040084B019368469C
:100E2000FDF70EFD064B1860064B01221A700648AE
:100E300006B010BDD90D01086C970020950D010872
:100E400068970020549700205897002003461046CA
:100E500005E013F8011B4140044A505C614601F172
:100E6000FF3C1FFA8CFC0029F3D17047284601088B
:100E700088B138B50C46054602290ED90139FF2242
:100E800089B2FFF7E3FF2C4414F8013C834214BFFE
:100E90000020012038BD002070470020FAE7000044
:100EA000034698B1481E99B110B413F8011B514084
:100EB000C9B2084C34F8111081EA122201460138F7
:100EC0000029F2D110465DF8044B70474FF6FF72CF
:100ED0001046704728470108D8B170B50C46064641
:100EE000022918D98D1E0D4B1A882946FFF7D8FF05
:100EF000C2B2735D9A4201D0002070BDC0F30F20D2
:100F0000344414F8013C984201D00020F5E7012058
:100F1000F3E7002070470020EFE700BF52060020F3
:100F200000B583B0074B1868FBF754FD064B0093E0
:100F3000064B074A07490020F8F7D6FB03B05DF8D7
:100F400004FB00BF0C980020783D01080041010817
:100F50000441010828490108002860D010B5044662
:100F60002F4B0068186022791A712378A52B00D0C6
:100F700010BD05212046FFF77BFF01280AD0284B32
:100F8000B3F801300933E018E35CA52BF0D1FFF78B
:100F9000E3FFEDE7617809312046FFF79DFF012867
:100FA000EDD1A279637943EA02231D4AA2F8053004
:100FB00040F20232934210D0B3F5417FDFD1184B9B
:100FC000D4F80700D4F80B10D4F80F20C3F80700AA
:100FD000C3F80B10C3F80F20D1E7114BD4F807006A
:100FE000D4F80B10D4F80F20D4F813C0C3F81300B2
:100FF000C3F81710C3F81B20C3F81FC0D4F817009C
:10100000D4F81B10D4F81F20C3F82300C3F827100E
:10101000C3F82B20B4F82320A3F82F20AFE77047A4
:1010200070970020F0B53B4AB2F907103A4B19808F
:10103000B2F909105980517B1971917B5971B2F83D
:101040000F201FFA82FEDA80D1B212F0200F14D0E6
:1010500092B21A8111F0100F13D02F4BDA885A81F7
:101060002D4BB3F842601889B3F80AC0B3F8445066
:10107000B3F846400123002220E0274B00221A81CA
:10108000E8E7254B00225A81EAE7034206D02B42CB
:1010900004D1214911440F7F01370F7713EA0C0F58
:1010A00008D0234206D11C49114491F82C70013715
:1010B00081F82C705B009BB2013292B20F2A13D8D8
:1010C000111F89B20129F5D91EEA030FDDD0334281
:1010D000DBD10342D9D113EA0C0FD6D10E4911440A
:1010E0000F7B01370F73D0E70B4B03F13C0E9C468F
:1010F000BCE80F00AEE80F00BCE80F00AEE80F0040
:10110000BCE80F00AEE80F009CE807008EE807007F
:10111000F0BD00BF709700209497002008B5054BE4
:101120001868FDF7B1FB044B1868FFF715FFFFF7D0
:1011300079FF08BD909700200C98002000B587B07B
:101140000E4B0593049080238DF80C3003A8FBF719
:1011500053FC0B4B186000230093019302931E2352
:10116000ADF80030074B019302906846FDF768FB2D
:10117000054B1860054807B05DF804FB1D11010818
:101180000C980020210F01089097002094970020D0
:10119000002301E00133DBB2042B0DD8074931F9FC
:1011A0001320002AB8BF524292B2B2F5257FF1D97E
:1011B000002221F81320EDE7704700BF10980020AF
:1011C000F8B504460378427843EA0223C3F30A03DE
:1011D000A3F580634F4DAB8043788278DB0843EA08
:1011E0004213C3F30A03A3F58063EB808378C278CC
:1011F0009B0943EA8203027943EA8223C3F30A0389
:10120000A3F580632B804179530843EAC113C3F3EC
:101210000A03A3F580636B80037C427C43EA0223CC
:10122000C3F30A03A3F580632B81FFF7B1FF637952
:10123000C3F30113EB7263799B09AB72A379E27973
:1012400043EA0223AB81237A627A43EA0223EB81E9
:10125000237B2B74637B6B74A37BE27B43EA0223C7
:101260009C466B82DAB213F0200F14D01FFA8CF177
:10127000A98212F0100F12D0264B5A8ADA82254B1F
:10128000B3F85A60988ADC8AB3F85C50B3F85EE031
:101290000123002222E01F4B00219982E9E71D4B28
:1012A0000022DA82EBE7034208D02B4206D119492B
:1012B000114491F82870013781F82870234209D031
:1012C00013EA0E0F06D11349114491F83870013713
:1012D00081F838705B009BB2013292B20F2A12D8AB
:1012E000111F89B20129F5D91CEA030FDBD0334263
:1012F000D9D10342D7D12342D5D1064911440F7E1B
:1013000001370F76CFE7034948228818EFF730FD01
:10131000F8BD00BF1098002000B583B090220021D6
:10132000084802F053F9084B1868FBF753FB074BCA
:101330000093074B074A08490020F8F7D5F903B096
:101340005DF804FB10980020A8980020783D010863
:1013500000410108044101085849010808B5044B3F
:101360001868FDF791FA034B1868FFF729FF08BDCD
:10137000A0980020A898002000B587B00F4B0593D7
:10138000049012238DF80C3003A8FBF735FB0C4BAF
:10139000186000230093019302930A23ADF80030F4
:1013A000084B01936846FDF74BFA074B1860074B53
:1013B00001221A70064807B05DF804FB5D130108AE
:1013C000A898002019130108A0980020A4980020D4
:1013D000109800202DE9F04F02884B88D0F804C007
:1013E0004F684088934283B04CD1B1F800E0864505
:1013F00048D14FEA9E089C000EF0030E08FB04F94A
:101400004FEA8E021D01DB004FEA890907EB040A4F
:101410004FEA081B019200933B46B8F1000F1DD024
:1014200000990CF110023944404652F8106C1E60CD
:1014300052ED037A1E19C6ED007A52F8086C0E6060
:1014400052ED017A0E1901382B4402F11002C6ED5B
:10145000007A2944E9D1DC4409EB0703BEF1000F0F
:1014600009D07246614651F8040B1860013A2344D2
:10147000F9D1019B9C4404375745CDD1002003B0DE
:10148000BDE8F08F6FF00200F9E700BFF0B4D1E9DA
:1014900000470368D0F804C05668A3425DD11268C3
:1014A00093425AD10388448804FB03F4A50832D040
:1014B0000CF1100107F1100206F11003284612ED9D
:1014C000047A51ED047A77EEC77A013843ED047A55
:1014D00012ED037A51ED037A77EEC77A01F110012C
:1014E00043ED037A12ED027A51ED067A77EEC77A70
:1014F00002F1100243ED027A51ED057A12ED057A00
:1015000077EEC77A03F1100343ED057AD7D12B01AB
:101510009C441F441E4414F003041BD0DCED007AED
:1015200097ED007A77EEC77A013CC6ED007A11D0CC
:10153000DCED017A97ED017A77EEC77A012CC6EDE2
:10154000017A07D0DCED027A97ED027A77EEC77A5E
:10155000C6ED027A0020F0BC70476FF00200FAE797
:101560002DE9F04F45880B8806884768546848681D
:101570008BB0AB4209910496498840F08A80158867
:10158000B54240F0868052888A4240F082804FEA1D
:101590009308011D1601089107EB0811C2EB827C2C
:1015A000019106FB08F195000391D2004FEA8C01EE
:1015B00003F003099B0007F1100B04EB050A0791E8
:1015C00002920693ABF110030593079BDDF820E030
:1015D00003EB0A0CDFED317AB8F1000F53D0029B18
:1015E0004446C11802465B4692ED006A13ED047A48
:1015F00053ED034A53ED026A91ED005A53ED015A3F
:10160000571927EE067A97ED006A77EE277A26EECD
:10161000246A4F1936EE276A26EE857AD7ED007ACE
:1016200037EE067A67EEA57A013C3244314477EE14
:10163000877A03F11003D7D1039B019A1844B9F1BB
:10164000000F0BD04B46D0ED006AB2EC017A27EECA
:10165000267A013B284477EE877AF4D1ECEC017AC4
:10166000D44570460EF1040EB4D1019A069B114682
:1016700019449B44049B0191013BAA44049304D068
:10168000099B58689EE7059AD9E718460BB0BDE854
:10169000F08F6FF002000BB0BDE8F08F000000008B
:1016A0002DE9F04F438804884E68D0F8049087B045
:1016B0009C420193039640F0EA800A884B8893424B
:1016C00040F0E5809C4240F0E28005900CB34FF082
:1016D0007E5B671E46F804BB1BD04FF00108BA00C2
:1016E00006EB020A4FEA88053046002101F06EFF42
:1016F0000AEB05062A4600215046B8F1000F00F01B
:10170000CB8001F063FF013F08F1010846F804BBFC
:10171000E5D1019B002B00F0B5809D0009EB05028F
:10172000CC460292DDF80C902A1D04922F469E466C
:101730000026029BDCED006AB442A3EB070B00F02D
:10174000A1809FED597A324663460BE0F4EE477A6A
:10175000F1EE10FA02F10102C8BFB0EE677AA242C0
:101760002B4414D0D3ED007AF5EEC07AF1EE10FAE6
:10177000B1EE676AEADCB4EE476AF1EE10FA02F104
:101780000102C8BFB0EE467AA2422B44EAD1B5EEC0
:10179000407AF1EE10FA75D0F5EE406AF1EE10FAEB
:1017A00070D07246634693ED007AC7EE267A013A0E
:1017B000E3EC017AF7D101994B4693ED007AC7EE3D
:1017C000267A0139E3EC017AF7D103984FEA8608CB
:1017D000B14239D0DBED006A5A467346E246BAECB4
:1017E000017AD2ED007A26EE877A013B77EEC77A4E
:1017F000E2EC017AF3D1019BBB440246CA46BAEC43
:10180000017AD2ED007A26EE877A013B77EEC77A2D
:10181000E2EC017AF3D1284401318C42C344D7D1A0
:10182000049BBEF1010E06F101069C44A7F10407DA
:10183000A9447FF47EAFF5EE406AF1EE10FA06D0CF
:10184000002007B0BDE8F08FBB442844E4E7059BC7
:10185000019A5B68D3ED007AF5EE407A02FB04F260
:10186000F1EE10FA144608BF043307D0E8E7F3ECB2
:10187000017AF5EE407AF1EE10FAE1D10EF1010EA7
:101880007445F4D16FF0040007B0BDE8F08F6FF03D
:10189000020007B0BDE8F08F5646013F46F804BB92
:1018A0007FF41BAF35E700BF0000000001804280DD
:1018B00043607047F0B4D1E900470368D0F804C032
:1018C0005668A3425DD1126893425AD10388448876
:1018D00004FB03F4A50832D00CF1100107F110024B
:1018E00006F11003284612ED047A51ED047A77EEE2
:1018F000877A013843ED047A12ED037A51ED037AC9
:1019000077EE877A01F1100143ED037A12ED027A46
:1019100051ED067A77EE877A02F1100243ED027AF2
:1019200051ED057A12ED057A77EE877A03F110030F
:1019300043ED057AD7D12B019C441F441E4414F07B
:1019400003041BD0D7ED007A9CED007A77EE877AFE
:10195000013CC6ED007A11D0DCED017A97ED017AF9
:1019600077EE877A012CC6ED017A07D0DCED027A9A
:1019700097ED027A77EE877AC6ED027A0020F0BC06
:1019800070476FF00200FAE7DFED1F7A20EE270ABA
:10199000B5EEC00AF1EE10FAFDEEC07A04D517EEEE
:1019A000903A013B07EE903AF8EEE77A9FED177A0E
:1019B00030EE670A20EE070AFCEEC07A17EE903A86
:1019C0009BB2B3F5007F1AD207EE903AF8EE677A31
:1019D000591C30EE670A0E4AF7EE007A02EB8303D9
:1019E00002EB810293ED007AD2ED006A77EEC07AC5
:1019F00020EE260A67EE877A37EE800A704730EECF
:101A0000470A01210023E6E783F9223E0000004453
:101A10007C490108DFED217A20EE270AF5EE007AF5
:101A200030EE270AB5EEC00AF1EE10FAFDEEC07AEC
:101A300004D517EE903A013B07EE903AF8EEE77ABC
:101A40009FED177A30EE670A20EE070AFCEEC07AA7
:101A500017EE903A9BB2B3F5007F1AD207EE903A98
:101A6000F8EE677A591C30EE670A0E4AF7EE007AF4
:101A700002EB830302EB810293ED007AD2ED006A60
:101A800077EEC07A20EE260A67EE877A37EE800A74
:101A9000704730EE470A01210023E6E783F9223E32
:101AA000000000447C49010810EE103A184A23F067
:101AB000004393421BDDB3F1FF4F02DB30EE400ADF
:101AC000704700B583B0684600F0AEFB00F003003D
:101AD0000128DDED010A9DED000A0CD0022812D08C
:101AE00070B1012001F092F803B05DF804FBDFED66
:101AF000090A00F0CFBC01F089F8B1EE400AF3E723
:101B000000F0C8FCF0E700F0C5FCB1EE400AEBE7DE
:101B1000D80F493F0000000010EE103A194A23F098
:101B2000004393421CDDB3F1FF4F02DB30EE400A6D
:101B3000704700B583B0684600F076FB00F0030004
:101B40000128DDED010A9DED000A0ED0022813D018
:101B500070B100F09FFCB1EE400A03B05DF804FBE9
:101B6000DFED090A002001F051B800F093FCF4E722
:101B7000012001F04BF8F0E7012001F047F8B1EE49
:101B8000400AEAE7D80F493F0000000008B52DEDF4
:101B9000028BB0EE408A00F075F8B4EE488AF1EEA0
:101BA00010FAF0EE408A0AD6B0EE480A01F050F979
:101BB000F7EE007AB4EEE70AF1EE10FA04DCB0EECC
:101BC000680ABDEC028B08BD01F008FABDEC028B7F
:101BD000034621221A600248BDE8084001F086B998
:101BE000F83C010808B52DED028BB0EE408A00F0FC
:101BF0006DF9B4EE488AF1EE10FAF0EE408A0AD69A
:101C0000B0EE480A01F024F9F7EE007AB4EEE70AE4
:101C1000F1EE10FA04DCB0EE680ABDEC028B08BDF0
